S0200000656D6265646465645F686F73745F5457522D4B36354631382E73726563CF
S113000000000320D5D00000C77400002F75000045
S1130010A7750000EB7500001796000000000000B3
S113002000000000000000000000000097AD000088
S1130030BBB600000000000049D10000D12200003E
S1130040FDE4000005E500000DE5000015E50000F5
S11300501DE5000025E500002DE5000035E5000064
S11300603DE5000045E500004DE5000055E50000D4
S11300705DE5000065E500006DE5000075E5000044
S11300807DE50000D5E60000D5E60000D5E60000D9
S1130090D5E60000D5E60000D5E60000D5E6000070
S11300A085E500008DE5000095E500009DE5000074
S11300B0A5E50000ADE50000D5E60000B5E50000CB
S11300C0BDE50000C5E50000CDE50000D5E5000074
S11300D0DDE50000E5E50000EDE50000D5E6000003
S11300E0D5E60000D5E60000D5E60000D5E6000020
S11300F0D5E60000D5E60000D5E60000D5E6000010
S1130100D5E60000D5E60000D5E60000D5E60000FF
S1130110D5E60000912B0000D5E60000D5E60000EE
S1130120D5E60000D5E60000D5E600001BB80000C7
S1130130D5E60000D5E60000D5E60000D5E60000CF
S1130140D5E60000F5E50000C5200000FDE500004F
S1130150D5E60000D5E60000D5E60000D5E60000AF
S1130160D5E60000D5E6000005E6000013210000F6
S11301701D210000272100000DE6000015E6000007
S1130180312100001DE6000025E600002DE60000F8
S113019035E600003DE6000045E60000D5E6000037
S11301A0D5E60000D5E60000D5E600004DE60000E7
S11301B0D5E60000D5E6000055E600005DE6000047
S11301C065E600006DE6000075E600007DE60000CF
S11301D0D5E60000D5E60000D5E60000D5E600002F
S11301E0D5E60000D5E60000D5E60000D5E600001F
S11301F0D5E60000D5E60000D5E60000D5E600000F
S1130200D5E60000D5E60000D5E60000D5E60000FE
S11303F0D5E60000D5E60000D5E60000FFFFFFFFCC
S1130400FFFFFFFFFFFFFFFFFFFFFFFFFEFFFFFFF9
S11304100EB430B5040003A805002900200001F043
S1130420EDF830BC5DF810FB30B595B004000D005C
S1130430684601F0EFF85A208DF80400A4208DF8E6
S113044005000C20ADF8060007208DF80A000020F6
S11304508DF80B0000208DF80C0002208DF80D00A3
S11304600DF10E00E4B204600DF1120000210160F0
S1130470042201A9684601F0DBF8BDF806200DF15D
S11304800A01684601F0D4F8BDF80000ADF8080090
S11304900DF13600012101600BA901A800F045FC13
S11304A0002801D0012017E00DF13601086800286A
S11304B00FD19DF83500286001202968884208D2B0
S11304C00BA911EB8002D2F80A1045F82010401C49
S11304D0F3E70DF13601086815B030BD30B595B0BD
S11304E004000D00684601F095F85A208DF80400C8
S11304F0A4208DF805000C20ADF806000C208DF822
S11305000A0000208DF80B0000208DF80C0002205A
S11305108DF80D000DF10E00E4B204600DF112002F
S11305200560042201A9684601F082F8BDF806209E
S11305300DF10A01684601F07BF8BDF80000ADF842
S113054008000DF13600012101600BA901A800F09B
S1130550ECFB002801D0012002E00DF1360108680F
S113056015B030BD00B591B0684601F053F85A207B
S11305708DF80400A4208DF805000420ADF80600D1
S11305800B208DF80A0000208DF80B0000208DF858
S11305900C0000208DF80D00042201A9684601F02A
S11305A047F8BDF806200DF10A01684601F040F84D
S11305B0BDF80000ADF808000DF13600012101601E
S11305C00BA901A800F0B1FB002801D0012002E032
S11305D00DF13601086811B000BD00B591B0684650
S11305E001F018F85A208DF80400A4208DF80500B5
S11305F00420ADF806000D208DF80A0000208DF8C7
S11306000B0000208DF80C0000208DF80D00042252
S113061001A9684601F00CF8BDF806200DF10A01A5
S1130620684601F005F8BDF80000ADF808000DF1CA
S11306303600012101600BA901A800F076FB002817
S113064001D0012002E00DF13601086811B000BDAF
S113065000B591B0684600F0DDFF5A208DF8040023
S1130660A4208DF805000420ADF8060001208DF8C3
S11306700A0000208DF80B0000208DF80C000020EB
S11306808DF80D00042201A9684600F0D1FFBDF8E1
S113069006200DF10A01684600F0CAFFBDF800000B
S11306A0ADF808000DF13600012101600BA901A885
S11306B000F03BFB002801D0012002E00DF13601DF
S11306C0086811B000BD30B591B004000D00684653
S11306D000F0A0FF4FF40070B5FBF0F101FB1051E6
S11306E000290AD0B5F5007F04D915F50070450A34
S11306F06D0202E04FF4007005005A208DF80400EA
S1130700A4208DF805000C20ADF8060002208DF819
S11307100A0000208DF80B0000208DF80C00022048
S11307208DF80D000DF10E0004600DF1120005604E
S1130730042201A9684600F07BFFBDF806200DF1F4
S11307400A01684600F074FFBDF80000ADF8080027
S11307500DF13600012101600BA901A800F0E5FAB2
S1130760002805D0DFF8C00CFFF752FE012010E08E
S11307700DF136010868002804D1DFF8EC0BFFF70F
S113078047FE03E0DFF8A00CFFF742FE0DF136014F
S1130790086811B030BD30B591B004000D00684652
S11307A000F038FF5A208DF80400A4208DF80500CD
S11307B00820ADF8060008208DF80A0001208DF805
S11307C00B0000208DF80C0001208DF80D000DF1B8
S11307D00E000560042201A9684600F029FFBDF857
S11307E006200DF10A01684600F022FFBDF8000062
S11307F0ADF808000DF136000121016022000BA9BB
S113080001A800F017FC002801D0012000E000201E
S113081011B030BD70B590B004000D0016006846EC
S113082000F0F8FE5A208DF80400A4208DF805008D
S11308300C20ADF8060004208DF80A0001208DF884
S11308400B0000208DF80C0002208DF80D000DF136
S11308500E0004600DF112000660042201A968462E
S113086000F0E6FEBDF806200DF10A01684600F02E
S1130870DFFEBDF80000ADF808000DF136000121DF
S113088001602A000BA901A800F088FA002801D011
S1130890012002E00DF13601086810B070BD70B59A
S11308A090B004000D001600684600F0B3FE5A2014
S11308B08DF80400A4208DF805000C20ADF8060086
S11308C003208DF80A0000208DF80B0000208DF81D
S11308D00C0002208DF80D000DF10E0004600DF1E6
S11308E012000660042201A9684600F0A1FEBDF8CA
S11308F006200DF10A01684600F09AFEBDF80000DA
S1130900ADF808000DF13600012101602A000BA9A1
S113091001A800F0F5FA002801D0012002E00DF151
S11309203601086810B070BD70B590B004000D00B9
S11309301600684600F06EFE5A208DF80400A420CC
S11309408DF805001020ADF8060005208DF80A008A
S113095000208DF80B0000208DF80C0003208DF88A
S11309600D000DF10E0004600DF1120006600DF192
S113097016000560042201A9684600F059FEBDF87E
S113098006200DF10A01684600F052FEBDF8000091
S1130990ADF808000DF13600012101600BA901A892
S11309A000F0C3F9002801D0012002E00DF1360166
S11309B0086810B070BD30B591B004000D006846F1
S11309C000F028FE5A208DF80400A4208DF80500BC
S11309D00C20ADF8060006208DF80A0000208DF8E2
S11309E00B0000208DF80C0002208DF80D000DF195
S11309F00E0004600DF112000560042201A968468E
S1130A0000F016FEBDF806200DF10A01684600F05C
S1130A100FFEBDF80000ADF808000DF1360001210D
S1130A2001600BA901A800F080F9002801D0012081
S1130A3002E00DF13601086811B030BD70B590B018
S1130A4004000D001600684600F0E4FD5A208DF8FD
S1130A500400A4208DF805001020ADF8060009203C
S1130A608DF80A0000208DF80B0000208DF80C0092
S1130A7003208DF80D000DF10E0004600DF112003D
S1130A8005600DF116000660042201A9684600F015
S1130A90CFFDBDF806200DF10A01684600F0C8FD3F
S1130AA0BDF80000ADF808000DF136000121016029
S1130AB00BA901A800F039F9002801D0012002E0B7
S1130AC00DF13601086810B070BD30B591B0040066
S1130AD00D00684600F09EFD5A208DF80400A42005
S1130AE08DF805000C20ADF806000A208DF80A00E8
S1130AF000208DF80B0000208DF80C0002208DF8EA
S1130B000D000DF10E0004600DF1120005600422C9
S1130B1001A9684600F08CFDBDF806200DF10A011C
S1130B20684600F085FDBDF80000ADF808000DF141
S1130B303600012101600BA901A800F0F6F8002895
S1130B4001D0012002E00DF13601086811B030BD7A
S1130B50F0B591B004000D0016001F00684600F0C7
S1130B6059FD5A208DF80400A4208DF80500052DA8
S1130B7003D31420ADF8060002E01020ADF80600FF
S1130B800E208DF80A0000208DF80B0000208DF84F
S1130B900C00052D03D304208DF80D0002E0032082
S1130BA08DF80D000DF10E0004600DF112000560CA
S1130BB00DF1160006600DF11A000760042201A968
S1130BC0684600F035FDBDF806200DF10A016846BF
S1130BD000F02EFDBDF80000ADF808000DF1360060
S1130BE0012101600BA901A800F09FF8002801D0A1
S1130BF0012002E00DF13601086811B0F0BDF0B536
S1130C0095B004000D0016001F00684600F002FDB8
S1130C105A208DF80400A4208DF805000C20ADF8AE
S1130C2006000F208DF80A0000208DF80B0000202C
S1130C308DF80C0002208DF80D000DF10E000460FB
S1130C400DF112000560042201A9684600F0F0FCD1
S1130C50BDF806200DF10A01684600F0E9FCBDF874
S1130C600000ADF808000DF13600012101600BA968
S1130C7001A800F05AF8002801D001200AE00DF183
S1130C803E01086830600DF14201086838600DF1DA
S1130C903601086815B0F0BDF0B591B004000D0040
S1130CA016001F00684600F0B5FC5A208DF80400B9
S1130CB0A4208DF805001020ADF8060010208DF852
S1130CC00A0000208DF80B0000208DF80C00032092
S1130CD08DF80D000DF10E0004600DF11200066098
S1130CE00DF116000760042201A9684600F0A0FC7B
S1130CF0BDF806200DF10A01684600F099FCBDF824
S1130D000000ADF808000DF13600012101602A0051
S1130D100BA901A800F0F4F8002801D0012002E09A
S1130D200DF13601086811B0F0BD70B504000D0076
S1130D300026032000F01AFB002801D001202CE03B
S1130D406088811D2000DFF84C2812689047DFF886
S1130D504808A17910EB810050F8041CDFF83C0826
S1130D60FFF756FB0320060076B2012E01DA0120BC
S1130D7013E000F014FB002804D03000461E40B2FB
S1130D800128F1DA280000F051FB0221DFF81008F5
S1130D90DFF8002812689047002070BD2DE9F04765
S1130DA08CB004000D0016000027D4F80E805FF00C
S1130DB00009684600F02EFC2020B8FBF0F101FB8E
S1130DC01081002904D05FEA5810401C070002E09B
S1130DD05FEA58100700032000F0C8FA002801D089
S1130DE001208AE06088811D2000DFF8A8271268AE
S1130DF09047DFF8A407A17910EB810050F8041C98
S1130E00DFF89807FFF704FB00F0C9FA012801D1C5
S1130E10012072E0280000F009FB0221DFF88007BE
S1130E20DFF87027126890475A208DF80400A52037
S1130E308DF80500002F55D0B8F1210F11D32020D3
S1130E40ADF806000020202808DA19F8061001AAD7
S1130E508218917119F10109401CF4E7B8F12008D6
S1130E6010E04046ADF806000020404508D219F8CD
S1130E70061001AA8218917119F10109401CF4E7C6
S1130E8000208046684600F0C5FB042201A968469C
S1130E9000F0CEFBBDF806200DF10A01684600F013
S1130EA0C7FBBDF80000ADF80800BDF80600811DC1
S1130EB001A8DFF8E026126890475FF0030A5FFAA2
S1130EC08AFABAF1000F01D1012016E000F067FAA6
S1130ED0002805D05046B0F1010AC0B20028EED176
S1130EE07F1EA7E7280000F0A1FA0221DFF8B00670
S1130EF0DFF8A0261268904700200CB0BDE8F08708
S1130F002DE9F0438BB004000D0016000027D4F83F
S1130F100E805FF00009684600F07CFB2020B8FBDF
S1130F20F0F101FB1081002904D05FEA5810401C45
S1130F30070002E05FEA58100700032000F016FAE9
S1130F40002801D0012072E06088811D2000DFF8B4
S1130F50442612689047DFF84006A17910EB81001F
S1130F6050F8041CDFF83406FFF752FA00F017FAC1
S1130F70012801D101205AE0280000F057FAD5F8E1
S1130F800A00002802D0D5F80A0050E00221DFF858
S1130F901006DFF800261268904701A8282100F007
S1130FA093FB002F38D0B8F1210F16D3414601A886
S1130FB000F095FA002801D0012038E00020202814
S1130FC008DA01A94118897909F8061019F101090B
S1130FD0401CF4E7B8F1200815E0414601A800F0F0
S1130FE07EFA002801D0012021E00020404508D2EB
S1130FF001A94118897909F8061019F10109401C61
S1131000F4E7002080460221DFF89405DFF8842508
S1131010126890477F1EC4E7280000F007FA0221F7
S1131020DFF87C05DFF86C251268904700200BB0D0
S1131030BDE8F0832DE9F0478CB004000D001600E4
S11310400027D4F80A805FF00009684600F0E2FA4D
S11310502020B8FBF0F101FB1081002904D05FEAE5
S11310605810401C070002E05FEA581007000320F4
S113107000F07CF9002801D0012088E06088811DFF
S11310802000DFF8102512689047DFF80C05A179DD
S113109010EB810050F8041CDFF80005FFF7B8F9E5
S11310A000F07DF9012801D1012070E0280000F052
S11310B0BDF90221DFF8E804DFF8D824126890476C
S11310C05A208DF80400A5208DF80500002F53D078
S11310D0B8F1210F0CD32020ADF8060020220DF129
S11310E00A01300000F056F8B8F1200820360AE072
S11310F04046ADF8060042460DF10A01300000F00A
S113110049F800208046684600F084FA042201A9C8
S1131110684600F08DFABDF806200DF10A01684614
S113112000F086FABDF80000ADF80800BDF806002E
S1131130811D01A8DFF85C24126890475FF0030A60
S11311405FFA8AFABAF1000F01D101201FE000F022
S113115026F98146B9F1000F02D0B9F1030F00D18D
S113116005E05046B0F1010AC0B20028E8D1B9F157
S1131170030F01D07F1EA9E7280000F057F90221D0
S1131180DFF81C04DFF80C241268904700200CB030
S1131190BDE8F08710B40023934204D204785C5471
S11311A0401C5B1CF8E710BC704770B504000D00D0
S11311B02E00E4B2032C0BD13068B0F5964F31D237
S11311C04FF461403060DFF8DC03FFF721F929E0D8
S11311D0E4B2042C26D130687E2806D27D2030600B
S11311E0DFF8C403FFF714F91CE03068FB2806D2CB
S11311F0FA203060DFF8B403FFF70AF912E0306830
S1131200B0F5FA7F07D84FF4FA703060DFF8A00326
S1131210FFF7FEF806E04FF47A703060DFF89403CD
S1131220FFF7F6F870BD38B504000D00DFF8880349
S11312300078E4B2A04204D1DFF87C0300780328EC
S11312400FD1DFF874030470FFF78CF9002804D180
S1131250DFF86803FFF7DCF803E0DFF86403FFF767
S1131260D7F8E4B2012C0CD1DFF85803C94908605F
S1131270DFF85403DFF854130860280000F058FC2A
S113128026E0E4B2022C0AD1DFF84403C149086025
S1131290D048CE490860280000F087FC18E0E4B28A
S11312A0032C09D1CC48BB490860CC48C749086025
S11312B0280000F0AAFE0BE0E4B2042C08D1C848D0
S11312C0B4490860C748C1490860280000F0CBFC55
S11312D031BD30B585B001A80021002200230EC025
S11312E00C3800208DF8000000208DF8010000F07B
S11312F0B0FF04000D00BC4800F0C6FF24184D41A7
S11313000221BA48A34A12689047642000F0C5FF3E
S11313109DF800005A280CD000F09BFFA94208D881
S113132001D3A04205D201216846A84A1268904719
S1131330EEE79DF800005A2801D0012011E00121B8
S11313400DF10100A14A126890479DF80100A728F9
S113135001D0012005E0082101A89C4A12689047A9
S1131360002005B030BD00009CD9000038B5040051
S11313700125E4B2EDB2AC420CD3FFF7AAFF00287A
S113138006D1EDB229009A48FFF742F8002005E0A3
S11313906D1CEEE79748FFF73BF8012032BD38B5E6
S11313A000208DF8010000208DF8000000F051FFAE
S11313B004000D00904800F067FF24184D4164209C
S11313C000F06BFF9DF801005A280DD000F041FF9A
S11313D0A94209D801D3A04206D201210DF101008E
S11313E07A4A12689047EDE79DF801005A2801D027
S11313F0012017E001216846744A126890479DF85D
S11314000000A12801D100200CE09DF80000A328D1
S113141001D1032006E09DF80000A22801D101209B
S113142000E0012032BD00003CE200007CB5060073
S11314300020ADF804000020ADF8020000208DF873
S1131440000000208DF8010000F003FF04000D00EF
S1131450694800F019FF24184D41642000F01DFF75
S11314609DF800005A280CD000F0F3FEA94208D8D9
S113147001D3A04205D201216846544A126890471C
S1131480EEE79DF800005A2801D0012026E0012152
S11314900DF101004D4A126890479DF80100A428FF
S11314A01BD1022101A8494A1268904702210DF17B
S11314B00200464A126890475A203070A420707087
S11314C0BDF804007080BDF80200B0807188B01DC2
S11314D03E4A12689047002000E0012076BDF0B536
S11314E083B006000F000020ADF804000020ADF822
S11314F0020000208DF8000000208DF8010000F0AB
S1131500A8FE04000D003C4800F0BEFE24184D4126
S1131510642000F0C2FE9DF800005A280CD000F0B0
S113152098FEA94208D801D3A04205D201216846F9
S1131530264A12689047EEE79DF800005A2801D029
S1131540012026E001210DF10100204A1268904794
S11315509DF80100A5281BD1022101A81B4A12688D
S1131560904702210DF10200184A126890475A2050
S11315703070A5207070BDF804007080BDF80200C2
S1131580B0803900B01D114A12689047002000E075
S11315900120FEBD5C04FF1F58C40000A8DD00004C
S11315A03A5600000CCE000034CE00005CCE0000A1
S11315B084CE0000ACCE0000E405FF1FD4CE0000B2
S11315C04CE20000531B00007F1B00006004FF1F5F
S11315D0C91B0000071C0000372000004D2000003C
S11315E0BB1C00009B1F000080841E0072270000AB
S11315F08CD0000054C50000404B4C0002B502469C
S11316006B46012102487844801D00F083FE02BD30
S1131610C9C7000010B50400002C06D130222749A8
S1131620274800F011FFC046C0460020208010BDAE
S11316307FB504000D001600002C06D137221F4987
S11316401F4800F001FFC046C046002D06D13822D5
S11316501A4919A000F0F8FEC046C046684600F0DA
S11316608DFF00208DF80B002088019041F22100AD
S1131670009000208DF80A0000208DF8080000205A
S11316808DF80900002E13D001F03AF869460D4890
S1131690006800F060FF320029000A48006800F08A
S11316A07BFF0848006800F095FF019001F02FF8D7
S11316B0019820807FBD000073726300C8C20000DF
S11316C088E200008CE60000002201F039B80268CC
S11316D0531C036011707047012110F01F029140E8
S11316E0DFF87C2A40B2430942F82310704710B552
S11316F00400200040B2FFF7EFFF10BD10B450F813
S1131700213033F47023D2B2140414F4702423432C
S113171040F8213010BC7047016270474A0103D57C
S1131720026852F080620260426831F080631A43BA
S113173042607047826A0A4382627047826A8A43BF
S113174082627047C9B2002907D002685200520869
S113175002600268D202FCD406E0026852F0004241
S113176002600268D202FCD57047C079704770B538
S1131770002400250020DFF8EC19086001F01AF8B5
S113178001F0CEF801F09FF800F03CFD00F081F884
S113179000F0C5F800F017F9002000F0E7F8DFF8D2
S11317A0C80900F07AFD00F04AFD0026642E07D235
S11317B0022001F097F8002800D0641C761CF5E79D
S11317C03D2C15D301F0EAF9DFF8A00901F0FCFA89
S11317D0EFF31080050072B6DFF894395FF48012DD
S11317E05FF48031DFF8840901F052FB85F310883F
S11317F00A220421DFF87C09FFF780FF3B20FFF772
S113180076FF0A220A21DFF86C09FFF777FF3B20F5
S1131810FFF76DFF70BDDFF860090068C0F3036077
S1131820401CDFF858190968B1FBF0F0704700203C
S1131830DFF84C190860DFF84C09006830F44030D8
S1131840DFF840190860DFF83C09006850F4A02074
S1131850DFF8301908600920DFF824190860DFF880
S11318602809006850F48020DFF81C190860DFF8AC
S11318701C09006850F00040DFF810190860DFF818
S11318800C09006830F44020DFF8001908600120DA
S11318907047E0B5684601F0AEFD4FF4614000903A
S11318A001208DF8080001208DF80900022000F0C5
S11318B01FF802006946DFF8D808806801F0AEFC22
S11318C0DFF8D00890F90400FFF711FF042000F0BE
S11318D00FF802006946DFF8B808006901F09EFCC1
S11318E04FF40051DFF8A808006901F0A2FD07BD1C
S11318F010B50400002C06D0022C08D003D3042C0D
S113190008D007D309E0DFF87408006806E0FFF7A1
S113191082FF03E0FFF77FFF00E0002010BD10B559
S1131920DFF874088468DFF8740802F01EF80120F8
S1131930DFF8681808700120DFF8601808730120C8
S1131940DFF858184873DFF85808DFF85018486073
S1131950FFF761FF0200DFF84418200001F085FF63
S1131960DFF84008DFF84018C86010BD10B5040067
S1131970DFF8380802F0C5FDFFF74DFF0200DFF87D
S11319802C18DFF82C0850F8240002F074FD002312
S11319900FF26122DFF81C18DFF8140850F8240055
S11319A002F0BFFF1020DFF8101808710020DFF8E4
S11319B0081888600020DFF8001808730020DFF89A
S11319C0F817086010BD10B586B0DFF8F00704689A
S11319D002A803F010FA01208DF80C00DFF8E007EC
S11319E002900820DFF8DC1708650920DFF8D41717
S11319F0486540F22310DFF8CC17886440F22130A8
S1131A00DFF8C017C8640020DFF8B81781F8980021
S1131A100020DFF8B01781F899000021DFF8A8074B
S1131A2000F0F2FD0021DFF8A40700F0EDFD08202E
S1131A30DFF8901708600920DFF888174860FFF77F
S1131A40EAFE020002A9200003F06EF90121200041
S1131A50FFF778FE4FF480412000FFF75FFEDFF8C8
S1131A607017200003F0E3F90020DFF8581781F81D
S1131A7038000820DFF84C17C86300208DF80400F4
S1131A80DFF84007806CDFF84C1711EA80400090C3
S1131A9000208DF8050001236A460821200003F088
S1131AA042FA4FF480712000FFF744FE0020DFF873
S1131AB0141781F840000820DFF808174864002252
S1131AC00921200003F0E6F9DFF80C0790F9000083
S1131AD0FFF702FEDFF8040790F90000FFF7FCFDB2
S1131AE0DFF8FC0690F90000FFF7F6FD06B010BD24
S1131AF010B50400DFF898068068807D002807D0C0
S1131B00DFF88C068068FFF730FE2070012000E0CB
S1131B10002010BD80B500208DF800000122694628
S1131B20DFF86C06806801F0BAFC9DF8000002BD85
S1131B3038B504004FF47A7000FB04F5FFF76BFE30
S1131B4003002A000121DFF85006806801F046FFF7
S1131B5031BD38B504000D00DFF84C0604600020E8
S1131B60DFF844164860DFF840068560DFF8381671
S1131B70DFF82406806802F07BF8002032BD38B517
S1131B8004000D000020DFF820160860DFF81806B6
S1131B904460DFF814068560DFF80C16DFF8F805FA
S1131BA0806802F065F8002032BD10B50400FFF72C
S1131BB032FE02004FF47A7000FB04F1DFF8F00506
S1131BC0006802F0D2FC10BD38B504000D000020FE
S1131BD0DFF8E4154871DFF8E0050461DFF8D805A3
S1131BE04561DFF8D415DFF8C805006802F0DEFDB2
S1131BF0002032BD30B4002A03D10124DFF8E455BB
S1131C002C7030BC704770B504000D004FF6FF76A1
S1131C100120DFF8A4154871DFF89C050461DFF8A2
S1131C2098054561DFF89025DFF88815DFF8800511
S1131C30006802F0A8FE0020DFF8A8150870DFF89D
S1131C40A4050078002803D1761EB6B2002EF6D182
S1131C50B6B2002E01D1052004E00020DFF884157F
S1131C600870002070BD38B50400002520007D38C0
S1131C7008D07D3809D0FA380AD0FA380BD0FA38AF
S1131C800CD00DE0002005000AE00120050007E06B
S1131C900220050004E00320050001E00420050003
S1131CA0052D09D2DFF82805052101FB0501DFF820
S1131CB00C05006803F0BBF831BDF0B583B0040037
S1131CC00D0000272600AF4220D2E81B092806D2C7
S1131CD0E81BDFF8F0144864E819C71B04E0082087
S1131CE0DFF8E014486408374FF47A7001900096E6
S1131CF0DFF8D004C36CDFF8F0240921002000F0E1
S1131D0009F8DFF8C004406C8619DCE700F03CF900
S1131D100020FEBD2DE9F04F87B004000D00160031
S1131D201F00DDF84080DDF84490DFF89004E4B251
S1131D3050F82400029028008DF8040030780399AC
S1131D4060F3555103917068039960F31341039153
S1131D50049810F06040B904C900C908084304900D
S1131D60039830F48010039003A80090B8F1000F9A
S1131D7032D000200099886000200099C8600020BB
S1131D8083465FFA8BFB7068834525D25FFA8BFB31
S1131D901BF8082011005FFA8BFBBBF1040F0CDA6F
S1131DA0DBF10302D2B2D20011FA02F21000009A5F
S1131DB092681043009A90600BE0DBF10702D2B204
S1131DC0D20011FA02F21000009AD2681043009A6D
S1131DD0D0601BF1010BD4E7009A2900C9B2029824
S1131DE003F00DF900281FD1012010FA05F1029823
S1131DF0FFF7A0FC4946DFF8D00300F02AFC824636
S1131E005FFA8AFABAF1030FF4D0012010FA05F14F
S1131E100298FFF793FC5FFA8AFABAF1000F01D037
S1131E20052002E0002000E0012007B0BDE8F08FAB
S1131E302DE9F04186B00400DFF88003E4B250F8E5
S1131E402460306BB16A084000900098002864D088
S1131E500120DFF8701309688840050000982842C3
S1131E604ED0DFF8680300F034FC01AADFF8540315
S1131E700168C9B2300003F04CF9002840D15FF08A
S1131E80000800200700FFB20198C0F30340874216
S1131E9036DAFFB2002F0BD0022F11D00CD3042F4F
S1131EA016D011D3062F1BD016D3072F1CD01FE03A
S1131EB09DF80F0080461BE09DF80E00804617E059
S1131EC09DF80D00804613E09DF80C0080460FE05D
S1131ED09DF8130080460BE09DF81200804607E051
S1131EE09DF81100804603E09DF810008046FFE74E
S1131EF0E4B221004046C0B200F02FF87F1CC2E7D4
S1131F000120B0494968884005000098284202D061
S1131F10AD4800F0DEFB009830634FF6024130001C
S1131F20FFF7FAFB06B0BDE8F08138B50400A3481A
S1131F30E4B250F824504FF602412800FFF7ECFBBE
S1131F4031BD38B504009D48E4B250F824504FF632
S1131F5002412800FFF7E0FB31BD9A4A994B93F800
S1131F6098309A1882F85800964A92F89820521C91
S1131F70944B83F89820934A92F8982012F03F02E9
S1131F80904B83F89820704700208E4981F8980080
S1131F9000208C4981F899007047F8B504000D00C1
S1131FA000264FF6FF77F6B2AE4225D27F1EBFB2AF
S1131FB0002F21D0834890F89900824991F8981015
S1131FC08842F0D07F487F4991F89910081890F81A
S1131FD05800F6B230557B4890F89900401C794976
S1131FE081F89900761C774890F8990010F03F002A
S1131FF0744981F89900D6E7BFB2002F03D1FFF7E7
S1132000E2FC052000E00020F2BD10B584B004001D
S1132010684601F0F0F9009401208DF808000120D1
S11320208DF80900FFF7F7FB02006946584800697C
S113203001F0F4F81FBD38B504000D002A0021009A
S11320405348006901F015FA002032BDF0B40200D3
S11320504FF6FF736548006810F58070644C24687F
S1132060001B4FF48074B0FBF4F505FB14058D429E
S113207003D25B1E9BB2002BECD19BB2002B01D18F
S113208005201DE0002088420ED25A4C2468584D89
S11320902D6845194FF48076B5FBF6F707FB165704
S11320A03C5D8454401CEEE75148006808184FF426
S11320B08074B0FBF4F505FB14054D480560002061
S11320C0F0BC704780B54C480078800604D54B4876
S11320D00078C0B200F001F801BD46490968484AD9
S11320E011604749096800290FD0454909683F4AEA
S11320F0126850543D490968491C4FF48072B1FB81
S1132100F2F303FB121339490B6000213C4A1160BE
S1132110704780B50020FFF78BFE01BD80B500201D
S1132120FFF703FF01BD80B50020FFF70AFF01BDE3
S113213080B50020FFF77CFE01BD70B504000D00E2
S113214016003000461E002807D00122290010483E
S1132150806801F08EF96D1CF3E7300070BD00005B
S113216000E100E000D0004020A107003800FF1F7C
S11321706B66656B00900440448004408804FF1F34
S113218048800440048004403480044000700440CB
S1132190F8DF0000DCE400009CE30000E0C1FF1F66
S11321A0A08601000100100004C2FF1F14C2FF1F1B
S11321B05CE2000038C2FF1F20C2FF1FE4E40000FD
S11321C048E801000808FF1F1008FF1F2808FF1F28
S11321D06804FF1F0000FC1F6656000056570000ED
S11321E076660000D9C7FF1F4808FF1F64C2FF1F9F
S11321F068C3FF1F6404FF1F04A00E4007A00E4025
S113220060C2FF1F0020364908607FF07F403549D7
S113221008600020344908600720344908603448C5
S11322200068C0003349B0FBF1F03349086032481C
S11322300068002802D101202F49086070472B480C
S11322400068C008C00029490860002026490860C9
S11322507047F0B4224B1B681A00234B1B68DB4306
S11322601B021B0A1C001E4B1B689A42F2D116006B
S113227000273F0647EA16273606002536196F4120
S113228030003900F0BC70471B490968A1FB00010C
S1132290C00840EA4170C90870472DE9F041804602
S11322A0FFF7D7FF06000F0013480068A0FB0801E2
S11322B0C00840EA4170C908841951EB0705FFF7CB
S11322C0C8FFA942FBD301D8A042F8D3BDE8F081EE
S11322D003480068401C0249086070470000000081
S11322E07CC4FF1F14E000E018E000E010E000E010
S11322F08804FF1F40420F0080C4FF1F70B50446CE
S11323001E000846154604D015F8011BA047761E8A
S1132310FAD170BD2DE9F04784B08246894614464F
S11323201F46E84607E00123224649465046FFF788
S1132330E5FF8146641C207810B904B0BDE8F0873D
S11323402528F0D16078A41C2528014618D05828E7
S11323505CD063280ED0642818BF692814D06F2875
S113236054D0702858D073285DD0752818BF7828A9
S11323704CD0E0E73868386050F8041B3860C9B2C4
S11323804846D0478146D6E73868386050F8045B41
S11323903860002D03D52D214846D047814664205E
S11323A06F2808BF082205D040F02001782914BF07
S11323B00A2210220B216428AC4603D1002D48BF09
S11323C0CCF1000CBCFBF2F502FB15CC0CF1300691
S11323D05FFA86FC4B1EBCF13A0FA4BFA0F1510674
S11323E0B44403F808C019465FEA050C01D001297A
S11323F0E8DA68460D184846D1F10B09C2D015F841
S1132400011BD047B9F10109F9D1BBE7396839603B
S113241051F8045B3960C3E73868386050F8045BEE
S113242038607820BCE73868386050F8045B38605E
S1132430284603F0E7F806004846A3D015F8011B28
S1132440D047761EFAD19DE780B503460FF20C0003
S113245003F0F4F8BDE8014003F002B925733A250E
S113246064202573202D2D20617373657274696F48
S11324706E206661696C65640A000000010C01F15C
S1132480804111F58E210A68012383401A430A60B2
S11324907047C0B2002801D0022000E00320C0B27F
S11324A07047C0B2002801D0022000E00020C0B272
S11324B0704710B44B7A0C7A240714F0405454EA51
S11324C083738C7A53EA8463CC7A240614F0807480
S11324D023431A0082600B68436052F000738360E8
S11324E04B680360826010BC70473EB504000D0069
S11324F02868009068680190687AFFF7D2FF8DF829
S11325000800287AFFF7C5FF8DF80900A87A8DF82E
S11325100A00E87A8DF80B0069462000FFF7C9FF2E
S113252037BD3EB504000D0028680090686801902E
S113253000208DF80800287AFFF7ABFF8DF809001A
S113254000208DF80A00E87A8DF80B006946200017
S1132550FFF7AFFF37BD38B504000D000C48FFF797
S11325608DFF287B002804D129002000FFF7BDFF40
S113257003E029002000FFF7D4FF31BD30B404008C
S113258004480FC8250085E80F0030BC70470000E0
S113259012003C105CE0000010B4002A08D011F0D6
S11325A00304002C04D00C780470491C521EF4E778
S11325B00B00042A04D31C6804601B1D121FF8E7D7
S11325C01900002A04D00C780470491C521EF8E744
S11325D010BC704701000B6818008B68C3F30173CB
S11325E01A00022A03D3000C0004000C00E080B29D
S11325F080B2704710B5101A73EB01014C4CD4E94A
S1132600002303F031F810BD38B504000D00002C90
S113261006D14C2247494848FFF716FFC046C0463A
S11326204348D0E90023002B08D1002A06D14FF4F7
S11326307A70FFF729FE3E4AC2E900016570002066
S1132640207000200021C4E9020100202061002044
S113265032BDF8B506000F00002E06D16E223549B2
S11326603548FFF7F1FEC046C0467078002808D010
S113267072B67078401E70700020307062B6002010
S113268026E0002F01D1022022E03078002812D069
S1132690FFF7DFFD04000D0022002B00D6E9020144
S11326A0FFF7A8FF3169814211D272B60020307061
S11326B062B602200CE017F1010F08D072B60120B7
S11326C0307062B6FFF7C5FDC6E902013761032029
S11326D0F2BD10B50400002C06D1A52215491648F8
S11326E0FFF7B2FEC046C0466078FF2801D1012042
S11326F005E072B66078401C607062B6002010BDC0
S113270072B60E480068401C0C49086070470B48BC
S11327100068022804D200200849086062B604E078
S113272006480068401E0549086070470000000024
S11327300008FF1F1CBF000034E40000C8C1FF1FD5
S113274000B500BF130096469446103928BFA0E890
S11327500C50FAD85FEA417C28BF0CC048BF40F84F
S1132760042BC90728BF20F8022B48BF00F8012B0F
S113277000BD5AA670B504000D001600002E06D147
S1132780C62247494748FFF75FFEC046C04614EBE0
S113279085003188018070BD10B450F8213033F4C5
S11327A0E063D2B2140214F4E064234340F821300D
S11327B010BC704780B50320ADF80000BDF80000E0
S11327C050F02000ADF800003748006850F478500D
S11327D035490860032210213448FFF7DDFF032246
S11327E011213248FFF7D8FF032219212F48FFF7A0
S11327F0D3FF032218212D48FFF7CEFF6A4612218A
S11328002A48FFF7B7FF6A4613212848FFF7B2FFAB
S1132810042212212548FFF7BFFF04221321234875
S1132820FFF7BAFF02220B212148FFF7B5FF02226E
S11328300C211F48FFF7B0FF02220D211C48FFF7AF
S1132840ABFF02220E211A48FFF7A6FF01221C212A
S11328501848FFF7A1FF01221D211648FFF79CFF2E
S1132860012204211448FFF797FF01220521124891
S1132870FFF792FF012204210E48FFF78DFF01228A
S11328800A210C48FFF788FF02221E210948FFF79E
S113289083FF02221F210748FFF77EFF01BD0000CE
S11328A05CBD0000ECE400003880044000D004402B
S11328B000C004400090044000A004400069C840E7
S11328C010F00100704780B52248006800906A4605
S11328D00421214802F063FF6A460A211E4802F0DF
S11328E05EFF01BD10B50400012C0AD104211A4871
S11328F0FFF7E4FF002801D1012000E00020C0B26E
S11329000DE0022C0AD10A211348FFF7D7FF002853
S113291001D1012000E00020C0B200E0002010BD81
S113292080B50E48006800906A461C210A4802F0EF
S113293036FF6A4605210A4802F031FF6A461D2126
S1132940054802F02CFF6A460421054802F027FFDF
S113295001BD000084E6000000F00F4088E600009E
S113296040F00F40012110F01F029140DFF8F423E2
S113297040B2430942F82310704710B440B2002813
S113298009D50A01DFF8E03340B210F00F04E31870
S113299003F8042C04E00A01DFF8D03340B2C25437
S11329A010BC70470EB430B5040003A8050029001C
S11329B02000FEF723FE30BC5DF810FB2DE9F04744
S11329C004000D00160001275FF0000A012D0AD053
S11329D05DD3032D23D014D3052D42D030D3072D3E
S11329E055D053D353E0B146B9F1000F08D0D9F80C
S11329F00000400A82464946504600F00BF90700A1
S1132A0045E0B146B9F1000F08D0D9F80000400AFA
S1132A1082464946504600F05DF9070037E0B1466A
S1132A20DFF84C03D9F8001008180830C9F808007A
S1132A30B9F1000F03D0DFF83C03C9F8080026E021
S1132A40B146B9F1000F02D0CB48C9F80800D9F853
S1132A500000400A82464946504600F0DBF8070071
S1132A6015E0B0464FF40060C8F800004FF4007061
S1132A70C8F80400012088F810004FF40070C8F86A
S1132A8008004FF40070C8F80C0000E0FFE73800BD
S1132A90C0B2BDE8F0872DE9F84304000D0016002C
S1132AA00027B046B146280001280ED0072812D0CE
S1132AB008281AD009284FD00A2855D00B285BD0F3
S1132AC0112825D012282CD05EE00020AB490870D4
S1132AD00020070058E0002E06D00120A749087006
S1132AE099F80000A64908704EE0A4480078002830
S1132AF00DD0B8F80000000AB8F80010C0B20028E1
S1132B0005D19B4AC0B2801846F20B0211543BE037
S1132B10002E05D09A48007889F8000000200700AC
S1132B2032E0002E17D0B8F80000000AC0B2002826
S1132B300FD1B8F8001011F47F418D4AC0B2821849
S1132B4046F20B039A5C1143A8F8001000210F0011
S1132B5001E005210F0017E0002E04D03100200011
S1132B6002F066FE07000FE0002E04D031002000C2
S1132B7002F065FE070007E0002E04D031002000BB
S1132B8002F069FE0700FFE73800C0B2BDE8F28337
S1132B9080B57748006803F049FD01BD10B582B0E7
S1132BA0784800788DF800009DF80000040003F0D8
S1132BB04AFEFEF73CFE00207349087000206F496E
S1132BC0087000206A4948600020694908606F481D
S1132BD000F0A0F86D4802F015FD6D49C1F80C0431
S1132BE0634A6C49002004F0C9F8002804D16948FC
S1132BF0006840685E4948600421200040B2FFF745
S1132C00BCFE200040B2FFF7ADFE5948006804F056
S1132C10EEFA13BD2DE9F84304000D006F685FF070
S1132C200008AE6842463900300004F04DFC5A4EAC
S1132C30706800280FD03068A0420AD1B768D6F86F
S1132C400480D5F808903A004146484604F070FCE8
S1132C5001E00C36ECE72000002806D011280DD046
S1132C6016281FD0172821D031E05520A96881F8F3
S1132C70FE01AA20A96881F8FF0128E0AF6817F5D2
S1132C80BE704349D1F80C1401604448404991F89E
S1132C901C1450F82180404602F0B4FC17F5CE71A4
S1132CA0086014E0A86800F035F810E03B483849A3
S1132CB091F81C1450F82170380002F0A3FC8046EF
S1132CC0D5F8089042463900484604F031FC00200B
S1132CD0BDE8F283F8B504000D0000261B27BC42B2
S1132CE016D3EFF31080060072B64FF40073214A36
S1132CF02B480068E11B4FF4007C0CFB01012948C0
S1132D0000F01CF9002801D000F027F886F31088A1
S1132D100020F2BD10B58CB0040023480A9023486B
S1132D200990234808905FF480200790214806907A
S1132D30214805905FF400100490782003901F4808
S1132D4002900020019000200090012345221C499C
S1132D50200004F029FC0CB010BD80B51948FFF721
S1132D6021FE01BD00E100E018ED00E000E400E018
S1132D70C018FF1FD078FF1FD07AFF1FCD78FF1F28
S1132D80CA78FF1FF2D90000CC78FF1FD47CFF1F44
S1132D90D07CFF1F7800FF1FB0C400004CE000008F
S1132DA03400FF1F3800FF1FF0DD0000D0E20000F8
S1132DB0C4E20000B8E20000ACE200003CE0000025
S1132DC0B0BC000018DA000070B50400002C01D17A
S1132DD004204AE0DFF838020068000E10F00F0605
S1132DE0F6B20F2E03D15FF40010050006E0DFF801
S1132DF06802F6B230F81600800205000020206058
S1132E0065600420A0604FF48050E0604FF480704F
S1132E10DFF8641291F9001088406061DFF85C0209
S1132E200078C0B2A06100202061200000F03CF9CD
S1132E30002813D00020DFF864120860DFF8600275
S1132E40DFF858124860DFF85C02DFF8501288603F
S1132E50DFF84802E061200000F008F85FF0A050BD
S1132E6020624FF480506062002070BD38B50400C9
S1132E70002C01D104200AE0E0690500686800F034
S1132E80B8F8A86800F0EAF802202860002032BDF3
S1132E902DE9F04F89B004000D0016001F006A46AA
S1132EA02900200000F02DF9049B320029002000A5
S1132EB000F00BF98346BBF1000F01D058463AE00D
S1132EC000980500019880467019401E8146B9FBA0
S1132ED0F8F008FB1090002807D0B9FBF8F0401C6C
S1132EE0824608FB0AF0401E8146A9451FD32802EA
S1132EF0000A50F01060DFF86C12096808603800AE
S1132F0000F027F98346BBF1000F01D0584612E0C8
S1132F10200000F07FF883462069002801D0206952
S1132F208047BBF1000F02D118EB0505DDE7200057
S1132F3000F0A6F8584609B0BDE8F08F2DE9F0413D
S1132F4088B004000D0016001F00002E01D10420DB
S1132F504CE06A462900200000F0D3F8039B3A00B5
S1132F602900200000F0B1F88046B8F1000F01D02C
S1132F7040463BE000980500002F33D03068DFF86E
S1132F80E41109684860361D0398042808D1280212
S1132F90000A50F0C060DFF8CC110968086010E046
S1132FA0039808280DD13068DFF8B81109688860E3
S1132FB0361D2802000A50F0E060DFF8A811096805
S1132FC00860200000F026F880462069002801D01F
S1132FD020698047B8F1000F04D10398451903987C
S1132FE03F1AC9E7200000F04BF8404608B0BDE89E
S1132FF0F08170B504000C255C4E2A0031002000DD
S113300004F096FA601C5A49086070BD0000000084
S11330104C80044070B504007020564908702000AC
S113302000F042F80600002E01D0300013E05148B1
S11330304F49096888474F4800780500A80601D51C
S1133040672008E0E80601D5682004E0E80701D518
S1133050692000E0002070BDACD1000070B5040010
S11330601425454E2A003100200004F061FA601C4A
S11330704249086070BD0000280002402B00024055
S113308038B50400200000F00FF80500002D03D12E
S11330903B483A490968884731BD00009CC1FF1F7D
S11330A01CC1FF1F5CC1FF1F0100002901D10420C6
S11330B00AE0C8690200C869002804D01068022820
S11330C001D1002000E06D20704730B40400002CD2
S11330D001D1042013E0581E014202D1581E0242BD
S11330E001D065200BE02068814205D32068656823
S11330F028185518A84201D2662000E0002030BCF0
S113310070472DE9F04104000D001600002C01D198
S113311004201CE020275FF00008424639003000FC
S113312004F0D2F92068281A3060E06870606068A2
S1133130A168B0FBF1F0B0600820F06010203061AD
S1133140102070610820B0610420F0610020BDE807
S1133150F08101000448814201D06B2000E000208E
S11331607047000090E600006B66656B00E30000AA
S113317014C1FF1F0000024004DE000018C1FF1F3D
S113318004F00140010C01F1804111F58E210A681F
S1133190012383401A430A60704770B50400052672
S11331A000200500B54207D2DFF8940550F8250049
S11331B0A04201D06D1CF5E7B54208D39F22DFF889
S11331C08415DFF88405FFF73FF9C046C0462800A0
S11331D070BD01000A8C4B8C92B29A4207D20A8CC1
S11331E0CB6913FA82F24B8CD21A100004E00A8CD9
S11331F092B24B8CD21A1000704738B504002000EC
S1133200FFF7E7FFE169491E884202D1012005006A
S113321001E0002005002800C0B232BD2DE9F047CE
S113322004000D001600002D08D1C622DFF8141585
S1133230DFF81805FFF708F9C046C04628680028DB
S113324008D1C722DFF8FC14DFF80405FFF7FCF807
S1133250C046C046DFF8FC04844201D1082019E0CE
S1133260DFF8F404844201D1082013E0DFF8EC0411
S1133270844201D101200DE0DFF8E404844201D14D
S1133280012007E0DFF8DC04844201D1012001E0E1
S11332905FF0FF30A979884208DAC922DFF8A41464
S11332A0DFF8C404FFF7D0F8C046C046DFF8A40432
S11332B0844201D1082019E0DFF89C04844201D142
S11332C0082013E0DFF89404844201D101200DE0CA
S11332D0DFF88C04844201D1012007E0DFF8840484
S11332E0844201D1012001E05FF0FF30E979884296
S11332F008DACA22DFF84C14DFF87004FFF7A4F8E8
S1133300C046C04600275FF000085FF00009286847
S11333100001B6FBF0F00700BFB2002F01D101207D
S11333200700700129680901B0FBF1F0BFB2B0EBEE
S1133330471A7000BFB2790111FA8AF1B0FBF1F0BB
S11333402968401A814628686421B0FBF1F0032102
S11333504843484502D240F2F5304AE02000FFF7E6
S11333601CFFDFF80C1451F82000FFF70BFFE07886
S113337010F0F300E070207810F0E001380080B223
S1133380000A084320706770A07A10F0E0001AF079
S11333901F010843A072A07810F0EF00804618F0D7
S11333A0FC08287950EA0800A070207810F0DF00AB
S11333B06979490111F0200108432070A879E0746B
S11333C0E8796075207C50F088002074607C50F0AF
S11333D0C0006074E0788046287A002801D058F054
S11333E00808687A002801D058F0040884F803809B
S11333F00020BDE8F08710B50400002C09D140F28C
S11334004512DFF84013DFF84403FFF71DF8C04608
S1133410C0465FF4E130206000202071002060711C
S11334200020A0710120E071002020720020607251
S113343010BD02780A430270C2780B0A1A43C270A4
S113344082790B0C1A438271427C0B0E1A4342742C
S1133450704702788A430270C2780B0A9A43C2709A
S113346082790B0C9A438271427C0B0E9A4342740C
S1133470704713005A1E002B06D003791B06FCD597
S11334800B78C371491CF4E7704710B400239342CE
S113349003D25C5CC4715B1CF9E710BC7047130079
S11334A05A1E002B06D0837D002BFCD0C3790B70F1
S11334B0491CF4E7704710B40023934203D2C47943
S11334C05C545B1CF9E710BC7047F8B504000D00B0
S11334D0207900070BD5E079686A002807D0AB6A29
S11334E040F2F13229002000D5F824C0E0472079C9
S11334F0800673D5E078800670D5A07D0700FFB202
S1133500002F2AD02869002827D02869FFB2B842A2
S113351001D22E6900E03E00F6B23200E9682000D4
S1133520FFF7C9FFE868F6B23018E8602869F6B218
S1133530801B2861BF1B28690028E0D1022085F880
S11335402D00686A0028DAD0AB6A40F2EB32290019
S11335502000D5F824C0E047D1E7A869002835D079
S11335603800471EC0B2002838D02800FFF745FEB7
S113357000280AD0686A002807D0AB6A4FF47C722E
S113358029002000D5F824C0E0472800FFF735FEC5
S113359000280AD0688C401CE969884202D10020C6
S11335A0688402E0688C401C6884288CE179AA69EC
S11335B080B28154288C401CE969884202D10020E1
S11335C02884CDE7288C401C2884C9E72869002872
S11335D004D15FF402212000FFF73BFF20790006AD
S11335E051D5E07800064ED55A48844201D10820CE
S11335F015E05948844201D1082010E0574884421C
S113360001D101200BE05648844201D1012006E09B
S11336105448844201D1012001E05FF0FF30217D54
S1133620471AFFB2002F2ED0686800282BD0686894
S1133630FFB2B84201D26E6800E03E00F6B232003A
S113364029682000FFF721FF2868F6B230182860A7
S11336506868F6B2801B6860BF1B68680028E0D108
S1133660002085F82C00E07810F07F00E070686A94
S11336700028D6D0AB6A40F2EA3229002000D5F8FF
S113368024C0E047CDE7F1BD80B53A480068002882
S113369007D140F2C3322B493748FEF7D5FEC04666
S11336A0C046344801682B48FFF70FFF01BD80B5C1
S11336B0FFF7EAFF01BD80B52E484068002807D116
S11336C040F2D2321F492D48FEF7BEFEC046C04626
S11336D0284841682048FFF7F8FE01BD80B5FFF790
S11336E0EAFF01BD80B523488068002807D14FF464
S11336F0787214492248FEF7A7FEC046C0461D480A
S113370081681648FFF7E1FE01BD80B5FFF7EAFFC7
S113371001BD80B51748C068002807D140F2EF32D8
S113372008491848FEF790FEC046C0461148C168D3
S11337300B48FFF7CAFE01BD80B5FFF7EAFF01BDE4
S113374068DE000074C1000020D500003CE40000E5
S113375048DA000000A0064000B0064000C0064061
S113376000D0064000A00E4060C60000A0C60000C5
S11337707CDE0000CCC1FF1FECE00000FCE0000098
S11337800CE100001CE10000010C01F1804111F585
S11337908E210A68012383401A430A607047C9B224
S11337A0002904D0026832F48042026003E0026817
S11337B052F4804202607047C06A7047C162704729
S11337C0026B8A4302637047026852005208C9B20E
S11337D052EAC172026070470068C00FC0B27047FD
S11337E001684908490001607047016851F001010E
S11337F001607047036833F44063C9B253EAC123DC
S1133800D2B253EA822303607047017842781207E8
S113381012F0E04252EAC1718278120412F47C126E
S11338201143C27851EAC261007951EA806070475D
S1133830806B704738B5040000200500032D07D2C3
S1133840DFF8340850F82500A04201D06D1CF5E7DC
S1133850032D08D39A22DFF82418DFF82C08FEF78A
S1133860F3FDC046C046280032BDF8B504000D0083
S113387016002000FFF7DEFFDFF8041851F82000DF
S1133880FFF782FF01212000FFF789FF2000FFF7E7
S1133890ACFF01212000FFF797FF2068DFF8E41751
S11338A008400700A87F57EA807095F8201050EA76
S11338B08160E97F50EA016095F82110090211F452
S11338C04071084320606A7F297F200000F072F86D
S11338D033006A682978200000F080F8002808D1B5
S11338E0B622DFF89817DFF8A407FEF7ADFDC0464F
S11338F0C046287814EB8000C06830F0FE40070012
S1133900287814EB8000A968491EC90611F0F0411B
S113391039432A7B920612F0806211436A7B520675
S113392012F000721143AA7B120612F08072114346
S1133930C16028690090330001222978200000F03A
S11339401DF968690090330002222978200000F0F4
S113395015F9A8690090330003222978200000F0AB
S11339600DF92000FFF73CFFF1BD00210170DFF8E5
S113397020174160082181600021017300214173F7
S1133980002181734FF47A7101614FF47A714161BE
S11339904FF47A718161012101770121417700217E
S11339A081770021C177002180F82010002180F860
S11339B02110704710B404682300D2B2012A05D143
S11339C0C9B20C0414F47C14234304E0C9B20C04FB
S11339D014F47C14A343036010BC70472DE9F74F23
S11339E082B01C000298FFF7F7FE002801D10020E6
S11339F06CE0DDF810905FF0FF3CE0465FF0000AF9
S1133A00CDF800A05FF0000C63465FF0010C664641
S1133A105FF0000C60465FF0000C6146042933D26D
S1133A20B8F1000F30D05FF0000C6246102A29D2A2
S1133A30B8F1000F26D05FF0010C6546032D1FD2AC
S1133A40B8F1000F1CD005FB04FCDFF848A65AF8B7
S1133A5021A0DFF844B65BF822B00BFB0AFABCFBEA
S1133A60FAFC6746B94509D3B9EB070CE646C645E7
S1133A7004D2F0460091130038002E006D1CDDE7DF
S1133A80521CD3E7491CC9E7DDF808C09DF80CA017
S1133A901CEB8A0CDCF80CC0DFF800A61AEA0C0A4E
S1133AA0CDF804A0DDF804C0B6F1010A5CEACA7CD2
S1133AB0DDF800A05CEA0A4C53EA0C0CDDF808A01F
S1133AC09DF80CB01AEB8B0ACAF80CC005B0BDE81F
S1133AD0F08F2DE9F04105000E0017009846069C72
S1133AE02800FFF779FE002846D0E4B2012C04D068
S1133AF042D3032C2BD015D33EE0F6B215EB86004F
S1133B00C068DFF89C150840B90511F4400108436A
S1133B105FEA083111F470410843F6B215EB8601EF
S1133B20C86029E0F6B215EB8600C068DFF87415AA
S1133B300840390511F4401108435FEA082111F4E3
S1133B4070610843F6B215EB8601C86014E0F6B262
S1133B5015EB8600C068DFF850150840B90411F46D
S1133B60402108435FEA081111F0F0010843F6B25E
S1133B7015EB8601C860FFE7BDE8F0812DE9F64F3B
S1133B8085B004001D00109E2000FFF725FE0028CC
S1133B9001D1002069E05FF0FF30834603200290EA
S1133BA00F200190DFF80405B0FBF5F0DFF80015F5
S1133BB0029A51F822104843DFF8F814019A51F898
S1133BC02210484380080490DFF8EC04B0FBF5F0C1
S1133BD0400003900398B0420BD39DF81800009066
S1133BE0002300229DF814102000FFF772FF0398B1
S1133BF03BE000200700042F2CD2BBF1000F29D09A
S1133C0000208046B8F1100F22D2BBF1000F1FD064
S1133C10DFF89804B0FBF5F0DFF8941451F827109E
S1133C204843DFF8901451F828104843800881462F
S1133C30B1450AD3B9EB06008246DA4505D2D3462C
S1133C400297CDF80480CDF8109018F10108D9E757
S1133C507F1CD0E79DF818000090019B029A9DF804
S1133C6014102000FFF735FF049807B0BDE8F08F6B
S1133C702DE9F24F86B004000698002809D140F2DD
S1133C803122DFF8F813DFF8AC04FEF7DDFBC046A1
S1133C90C0465FF000085FF0000B00208DF80000C4
S1133CA006988068002801D10420E1E12000FFF794
S1133CB09CFDDFF884142000FFF782FD012201211E
S1133CC02000FFF797FDDFF874142000FFF776FD5E
S1133CD001200699C968C1F3031188408DF80600D4
S1133CE000208DF8070000208DF808000698007B5E
S1133CF010F00F008DF805000698C068C00203D5C7
S1133D0001208DF8040002E000208DF8040001A8D1
S1133D10FFF77BFD04900698C068800203D501205C
S1133D208DF8040002E000208DF8040001A8FFF7DC
S1133D306CFD03909DF8050014EB8000C068C00E74
S1133D4010F00F00401C8DF80100069800688146B1
S1133D50069840688246069880680600069880683F
S1133D6007002068C00402D42068800402D5012022
S1133D70050013E0DFF8F403844201D104250DE0CB
S1133D80DFF8EC03844201D1012507E0DFF8E40306
S1133D90844201D1012501E05FF0FF352000FFF7E7
S1133DA01FFD9DF80100092880F29B80002E00F081
S1133DB05E81012E59D1B81BA84219D32000FFF708
S1133DC0FBFC8003F7D5BAF1000F07D02000FFF702
S1133DD02FFD8AF800001AF1010A02E02000FFF723
S1133DE027FD7F1E5FF400312000FFF7E7FCE2E7C8
S1133DF02000FFF7E1FC800105D45FF00071200092
S1133E00FFF7DCFCF4E7B9F1000F07D099F80000E4
S1133E1003990843606319F1010904E003989DF8CC
S1133E200010084360635FF000712000FFF7C6FCD8
S1133E30761E002FBAD02000FFF7BEFC8003F8D511
S1133E40BAF1000F07D02000FFF7F2FC8AF8000057
S1133E501AF1010A02E02000FFF7EAFC7F1E5FF47A
S1133E6000312000FFF7AAFCE3E72000FFF7A4FCE1
S1133E70800105D45FF000712000FFF79FFCF4E798
S1133E80B9F1000F07D0049899F800100843606353
S1133E9019F1010904E004989DF8001008436063D7
S1133EA0761E5FF000712000FFF788FC2000FFF70A
S1133EB083FC80037FF57AAFBAF1000F07D02000AE
S1133EC0FFF7B6FC8AF800001AF1010A02E02000AC
S1133ED0FFF7AEFC7F1E5FF400312000FFF76EFC9D
S1133EE064E7002E00F0C380032E78D2B81B40088C
S1133EF0A8421DD32000FFF75FFC8003F6D5200005
S1133F00FFF796FC8346BAF1000F0AD08AF800B096
S1133F101AF1010A584680B2000A8AF800001AF120
S1133F20010ABF1E5FF400312000FFF747FCDDE704
S1133F302000FFF741FC800105D45FF000712000F0
S1133F40FFF73CFCF4E7B9F1000F0DD099F800003D
S1133F50804619F10109022E09D399F8000058EAA4
S1133F60002819F1010902E09DF800008046039839
S1133F701FFA88F858EA000060635FF000712000BF
S1133F80FFF71CFC00200600002FAAD02000FFF73A
S1133F9013FC8003F8D52000FFF74AFC8346012F69
S1133FA00FD0BAF1000F0AD08AF800B01AF1010A52
S1133FB0584680B2000A8AF800001AF1010ABF1EAE
S1133FC007E0BAF1000F03D08AF800B01AF1010A31
S1133FD07F1E5FF400312000FFF7F0FBD4E72000E0
S1133FE0FFF7EAFB800105D45FF000712000FFF7C2
S1133FF0E5FBF4E7B9F1000F0BD099F80000804617
S113400019F1010999F8000058EA002819F1010989
S113401002E09DF80000804604981FFA88F858EAE8
S113402000006063B61E5FF000712000FFF7C6FB5E
S11340302000FFF7C1FB80037FF553AF2000FFF79B
S1134040F7FB8346BAF1000F0AD08AF800B01AF1E0
S1134050010A584680B2000A8AF800001AF1010ADF
S1134060BF1E5FF400312000FFF7A8FB39E70020F2
S113407007B0BDE8F08F0000E8E2000018C00000BF
S1134080F4E20000FFCCFFBA3CCB0000DCE300000C
S113409020A107009CE00000E0C50000F0FFFC7FC9
S11340A0FF0F3FFFFFF0CFFF0FFFF3FF00286BEE82
S11340B0ACE0000020C6000000CA9A3B38B50400FA
S11340C00D002000FFF788FB002805D02900200000
S11340D0294A1268904704E029002000284A1268FF
S11340E0904731BD000080B51F480068002807D103
S11340F040F24C6221492348FEF7A6F9C046C04667
S1134100194801681948FFF7D9FF01BD80B5164861
S11341104068002807D140F2546218491A48FEF753
S113412093F9C046C046104841681148FFF7C6FFDE
S113413001BD0000DCE2000000000A9A00000ADA77
S113414080B509488068002807D140F25C620B49B9
S11341500E48FEF779F9C046C04603488168054811
S1134160FFF7ACFF01BD000000C1FF1F00C002400B
S113417000D0024000C00A400CC1FF1F18C000005C
S113418010C1FF1F6CE000007CE000008CE0000028
S1134190012110F01F029140DFF8D42840B24309F6
S11341A042F823107047010C01F1804111F58E2172
S11341B00A68012383401A430A60704710B504005B
S11341C0200040B2FFF7E4FF10BDCA0403D5827992
S11341D00B0A1A4382714A0403D582790B0A1A43E3
S11341E08271C170704738B5040000200500042DA9
S11341F007D2DFF8800850F82500A04201D06D1CDA
S1134200F5E7042D08D3A622DFF86C18DFF86C0854
S1134210FEF71AF9C046C046280032BD2DE9F8431E
S113422004000D001600002796F805804FF6FF796C
S113423096EC060B85EC060B7069A861287B0028B8
S113424007D0022028777079012804D10020804605
S113425001E001202877E078000606D4B9F10109CD
S11342601FFA89F9B9F1000FF5D11FFA89F9B9F1EB
S1134270000F02D14FF48A6017E045F212012000CA
S1134280FFF7A3FF2878800707D54246D2B22979E1
S1134290200000F0CFF9070006E04246D2B22979A7
S11342A0200000F0A9F907003800BDE8F2830200FD
S11342B00020CB0605D51023D37040F24F431800DD
S11342C004E0CB0702D540F24E43180070472DE9B5
S11342D0F84304000D001600002794F80380002022
S11342E0307000208DF80000287F032802D168690F
S11342F0002805D0287F052805D16869012802D146
S11343005FF0010901E05FF000099DF80000401C26
S11343108DF8000041462000FFF7C9FF070040F276
S11343204E40874206D15FFA89F9B9F1000F01D0F6
S113433000200700002F01D0380083E0287F0128E7
S11343400DD15FEAC87002D540F24E407AE0687938
S1134350002802D10320287701E004202877287F51
S1134360022806D06DD304283BD02AD3052849D08F
S113437067E0287B002809D0287B401E2873A868A2
S1134380297BC9B2C900C840207119E068790028A6
S11343900ED1032028776869002811D02869007895
S11343A020712869401C28616869401E686107E023
S11343B001222979200000F03DF907000420287724
S11343C03FE06869002809D02869007820712869CD
S11343D0401C28616869401E686101E0012030705A
S11343E02FE0A07810F0E700A0706869012803D1DD
S11343F0A07850F00800A07020798DF80000052006
S113440028771EE06869411E6961002818D0686930
S1134410002808D1012030702878400703D42000F8
S113442000F03AF907006869012803D1A07850F038
S11344300800A0702869217901702869401C28614E
S1134440FFE73800BDE8F28338B504000D00E078DA
S1134450C00602D4A078800606D529002000DFF823
S11344605C261268904705E029002000DFF85026FA
S11344701268904731BD2DE9F04104000D0016008B
S1134480002D01D0002E09D14FF4CF72DFF8E815CA
S1134490DFF83006FDF7D8FFC046C0462000FFF71E
S11344A0A2FEDFF8241651F82000FFF77CFEA07866
S11344B010F07F00A07045F212012000FFF785FE86
S11344C032006968200000F050F86079804618F0E6
S11344D0DF08687858EA401884F80580A079070056
S11344E017F07F07A87857EAC01717F0F007287A63
S11344F010F00F000743A7712878C001A070BDE831
S1134500F08110B50400002C09D140F2D912DFF873
S11345106815DFF8B805FDF797FFC046C046DFF819
S1134520B0056060002060700020A0700020207240
S11345300120207010BD4A0603D5827852F0400253
S113454082708A0603D5827952F020028271704704
S11345504A0603D5827812F0BF0282708A0603D518
S1134560827912F0DF02827170472DE9F0435FF027
S1134570FF3600275FF0000C5FF00009CE465FFABB
S11345808EFEBEF1030F2FD2002E2DD05FF0010955
S113459019FA0EF94B465FF00009C8465FFA88F82D
S11345A0B8F1400F1DD2DFF82C955FFA88F839F87E
S11345B0189009FB03F9B2FBF9F94C468C4201D27D
S11345C00D1B00E0651AB54208D25FFA8EFE7746ED
S11345D05FFA88F8C4462E00002D02D018F10108B5
S11345E0DCE71EF1010ECAE71CF03F0959EA8719FE
S11345F080F80190BDE8F083F8B504000D001600C2
S11346000027200000F05EF80100880603D540F280
S11346104C4007000CE0A07850F03000A070F6B2D7
S1134620012E01D1012000E0002050EA4500207154
S11346303800F2BD2DE9F04104000D0016000027FA
S1134640200000F03FF801000622880606D5A07875
S1134650800603D440F24C4007001AE0607880469C
S113466018F03F006070A07850F00400A07084F847
S113467001801000421EC0B2002801D000BFF8E73C
S1134680F6B2012E01D1012000E0002050EA4500DD
S113469020713800BDE8F081010000204FF6FF7260
S11346A08B7813F0C7038B70CB789B0603D5521E0F
S11346B092B2002AF8D192B2002A02D14FF48A634E
S11346C0180070470100C8788A79520601D550F461
S11346D080408A79D20601D550F48050704730B4B6
S11346E0030000200024DD782D06FCD50225DD70B2
S11346F09D7855F010059D7015006A1E002D19D087
S11347000D781D71491CDD78AD07FCD5DD782C00D2
S11347100225DD70E50604D51025DD7040F24F4515
S11347202800E50704D50125DD7040F24E45280038
S11347300028E1D030BC7047F8B504000D00160025
S1134740002700208DF800009DF80000401C8DF823
S11347500000E0780006FCD50220E070A07810F09C
S1134760E700A070012E03D1A07850F00800A070DB
S113477020798DF800003000461E002814D0E0781F
S11347808007FCD50220E070002E03D12000FFF743
S113479083FF0700012E03D1A07850F00800A07019
S11347A0207928706D1CE6E73800F2BDF8B50400E6
S11347B00D00002D09D14FF44A72DFF8BC12DFF866
S11347C01803FDF741FEC046C0466E79002745F246
S11347D012012000FFF7F9FCE0780006FCD5287BE5
S11347E0002804D06879012801D100200600287827
S11347F0800707D53200D2B229792000FFF71AFFCB
S1134800070006E03200D2B229792000FFF7F4FE57
S11348100700002F01D0380082E0287B002844D014
S1134820E0788007FCD50220E070E1782000FFF7F3
S11348303EFD0700002F08D040F24E40874202D1CF
S11348402000FFF729FF38006AE0287B401E287308
S1134850A868297BC9B2C900C8402071287B0028F8
S113486001D0002FDCD0687901281ED1E0788007C0
S1134870FCD50220E070E1782000FFF718FD070066
S1134880002F08D040F24E40874202D12000FFF7AB
S113489003FF380044E0012229792000FFF7CAFE13
S11348A00700002F01D038003AE0E0788007FCD5FB
S11348B0E1782000FFF7FBFC0700002F08D040F24E
S11348C04E40874202D12000FFF7E6FE380027E081
S11348D06879002817D16869002814D06A692969A1
S11348E02000FFF7FCFE0700002F02D128784007C4
S11348F003D540F24E40874205D10220E0702000EB
S1134900FFF7CAFE07006879012808D16869002802
S113491005D06A6929692000FFF70EFF07003800F7
S1134920F2BD2DE9F04704000D0016001F00002D14
S113493009D140F2BD32DFF84011DFF8A001FDF7E4
S113494083FDC046C0462000FFF74DFC80465FF063
S113495028095FF0000A52464946280002F0B4FDD7
S11349602E626F62DFF8780140F828500FF27D0064
S1134970DFF848110860DFF86C0118F90000FFF750
S11349801DFCBDE8F087F8B504000D001600002DED
S113499009D14FF47572DFF8E010DFF84001FDF73C
S11349A053FDC046C046002E09D140F2D532DFF88F
S11349B0C810DFF82401FDF747FDC046C0460027B4
S11349C0287F002803D040F24C4007000BE032005F
S11349D029002000FFF722FC0700002F03D140210B
S11349E02000FFF7A8FD3800F2BD0000F8B5040070
S11349F00D00002D08D14FF481621F49DFF8E80053
S1134A00FDF722FDC046C0462E0000270220E070BC
S1134A106A4631002000FFF75AFC07009DF80000A9
S1134A20002801D1002F21D03078400703D540F26F
S1134A304E4087420AD1A078800607D52000FFF7B0
S1134A402BFE002802D04FF48A6007000020307744
S1134A5040212000FFF77CFD306A002806D0736AED
S1134A603A0031002000D6F820C0E047F1BD000034
S1134A7000E100E0CCE0000000C100008CCB0000AD
S1134A8080B5174801681948FFF7DEFC01BD80B501
S1134A90134841681648FFF7D7FC01BD80B510489C
S1134AA081681448FFF7D0FC01BD80B50C48C1688B
S1134AB01148FFF7C9FC01BD00000000C0C1FF1F81
S1134AC0C4C1FF1F04D50000DCE00000BCE000000E
S1134AD0A08601009CBE000024E400002CE4000039
S1134AE0B0C1FF1F94E600000CE300000060064024
S1134AF00070064000600E4000700E40010C01F191
S1134B00804111F58E210A68012383401A430A600B
S1134B10704701627047006B08407047016370473B
S1134B20826A8A4382627047C9B2002907D0026848
S1134B305200520802600268D202FCD406E0026805
S1134B4052F0004202600268D202FCD5704738B5C8
S1134B50040000200500022D07D2DFF8200750F8DA
S1134B602500A04201D06D1CF5E7022D08D3B9221F
S1134B70DFF80C17DFF89407FDF766FCC046C04663
S1134B80280032BD016851F080410160016851F094
S1134B90805101600168C901FCD57047016831F09A
S1134BA080510160016831F0804101600168C901F0
S1134BB0FCD470470200106880000FD5506B000EC3
S1134BC010F00F000300DBB25800C31DDBB2C9B202
S1134BD08B4201D3012002E0002000E00020704756
S1134BE038B504000D00EDB2102D08DBF422DFF817
S1134BF09016DFF8D407FDF727FCC046C046A06A2C
S1134C00E840C00701D5012000E0002032BD10B506
S1134C1004002068002809D540F21312DFF860165A
S1134C20DFF8A807FDF710FCC046C0462168C9029A
S1134C30FCD4216851F00071216021688901FCD401
S1134C40216841F4201151F00F012160802161603D
S1134C505FF43301616300210800C0B2102808DA50
S1134C607FF04041C0B214EB8002C2F88018401CAF
S1134C70F3E77FF0404121617FF0404161617FF0C3
S1134C804041A1617FF04041A16400210800C0B20D
S1134C90102807DA0021C0B214EB0012C2F8801009
S1134CA0401CF4E710BDF0B583B004000D001600FD
S1134CB00A2000FB06F7DFF85806864209D34FF4B2
S1134CC0A872DFF8BC15DFF84C06FDF7BDFBC04643
S1134CD0C046BD4209D24FF4A972DFF8A415DFF82B
S1134CE0F006FDF7B1FBC046C046002F01D10120FC
S1134CF00700B5FBF7F0471EFF2F01D9FF2007007F
S1134D0038008DF8000003208DF8020002208DF891
S1134D10030001208DF8040001208DF8010069468C
S1134D20200000F084F8F7BDF8B504000D0016006B
S1134D30002D09D140F27312DFF84415DFF8940610
S1134D40FDF782FBC046C0466879002802D0687926
S1134D50112809DB4FF4BA72DFF82415DFF83006A6
S1134D60FDF772FBC046C0462000FFF7F0FEDFF8F7
S1134D70681651F82000FFF7C1FE00212000FFF75C
S1134D80D3FE2879002803D1606830F4005002E093
S1134D90606850F40050606001212000FFF7C4FEF9
S1134DA02000FFF734FF206807006879401E60F395
S1134DB00607A879002803D0606850F4805002E008
S1134DC0606830F480506060E879002802D057F4BD
S1134DD0800701E037F48007287A002802D057F4CE
S1134DE0803701E037F4803727602A6831002000DB
S1134DF0FFF759FFF1BD10B50400002C09D14FF4A1
S1134E00D972DFF87C14DFF8CC05FDF71DFBC04632
S1134E10C04600202071DFF88C07206010206071EC
S1134E200020A0710020E0710020207210BD38B570
S1134E3004000D00002D09D140F2C312DFF8401424
S1134E40DFF89005FDF700FBC046C0462000FFF7E1
S1134E5099FE60684FF6F8710840606060682978D0
S1134E606A78920512F4400252EA0161AA78D204E7
S1134E7012F460121143EA78120412F4E02211438E
S1134E802A7912F007021143084360602000FFF7FB
S1134E9085FE31BD70B504000D001600206810F0C9
S1134EA07F00EDB2A84209D24FF40072DFF8D013AC
S1134EB0DFF8C406FDF7C8FAC046C0462900C9B2E7
S1134EC02000FFF777FE002809D04FF40172DFF8C5
S1134ED0B013DFF8FC06FDF7B7FAC046C046F6B2D9
S1134EE0002E07D05FF00060EDB214EB0511C1F89D
S1134EF0800005E00020EDB214EB0511C1F880003C
S1134F000020EDB214EB0511C1F884000020EDB2CD
S1134F1014EB0511C1F888000020EDB214EB051163
S1134F20C1F88C0070BD2DE9F04104000D0016009D
S1134F301F00206810F07F00EDB2A84209D240F2B1
S1134F401A22DFF83C13DFF83006FDF77DFAC0467D
S1134F50C046002E0CD1FFB2002F09D040F21B2214
S1134F60DFF81C13DFF86C06FDF76EFAC046C04686
S1134F705FF000082900C9B22000FFF71BFE0028DB
S1134F8009D040F22122DFF8F812DFF84406FDF7D9
S1134F905BFAC046C0460020EDB214EB0511C1F81F
S1134FA080000020EDB214EB0511C1F8840000204C
S1134FB0EDB214EB0511C1F888000020EDB214EB3A
S1134FC00511C1F88C00FFB2002F16D03068EDB285
S1134FD014EB0511C1F884003079012801D158F48B
S1134FE000187079012801D158F4801858F08068AD
S1134FF0EDB214EB0510C0F88080BDE8F081F8B57F
S113500004000D001600206810F07F00EDB2A842E5
S113501009D240F2CB22DFF86812DFF85C05FDF715
S113502013FAC046C046002E09D14FF43372DFF89C
S11350305012DFF8A405FDF707FAC046C0463068F1
S1135040C0F30340092809DB40F2CD22DFF8301217
S1135050DFF88805FDF7F8F9C046C04600272900A7
S1135060C9B22000FFF7A6FD002809D040F2D322E0
S1135070DFF80C12DFF85805FDF7E6F9C046C04624
S1135080EDB214EB0510D0F8800010F07060B0F1B0
S1135090406F3CD0EDB214EB0510D0F8800030F036
S11350A0706050F00060EDB214EB0511C1F880009F
S11350B07068C000C008EDB214EB0511C1F884009B
S11350C03068C0F34050002801D057F4C00730685E
S11350D0C0F30050002801D057F48017306810F452
S11350E0702050F040600743B068EDB214EB051136
S11350F0C1F88800F068EDB214EB0511C1F88C001A
S1135100EDB214EB0510C0F88070002000E001201F
S1135110F2BD2DE9F04104000D001600206810F0E6
S11351207F00EDB2A84208D24FF440725449DFF830
S11351304804FDF789F9C046C046002E08D140F264
S113514001324F49DFF89804FDF77EF9C046C046A6
S11351502900C9B22000FFF72DFD002808D04FF424
S113516042724749DFF86804FDF76EF9C046C0464D
S1135170EDB214EB0510D0F880000700380E10F0E3
S11351800F0080465FFA88F8B8F1020F04D05FFA86
S113519088F8B8F1060F30D1EDB214EB0510D0F851
S11351A08400C000C008716860F31C017160780D50
S11351B0316860F355513160380D316860F3145132
S11351C03160380C316860F313413160EDB214EB97
S11351D00510D0F88800B060EDB214EB0510D0F8DB
S11351E08C00F060A0685FFA88F8B8F1020F01D172
S11351F0002004E041F2B94001E0A0680120BDE8CC
S1135200F08138B504000D00002D08D140F23B3286
S11352101B49DFF8CC03FDF717F9C046C0462068E8
S1135220800028D5D4F880000100D4F88400C000A0
S1135230C0086A6860F31C026A60480D2A6860F35B
S113524055522A60080D2A6860F314522A60080C2B
S11352502A6860F313422A60D4F88800A860D4F85E
S11352608C00E860E06CC0B22A6860F3DF522A6008
S1135270A068002000E0012032BD00000CE4000022
S11352809CBF000070B504000D001600002D08D16D
S113529040F23442DFF85413D248FDF7D5F8C04643
S11352A0C046206810F07F00F6B2B04208D240F247
S11352B03542DFF83813B048FDF7C6F8C046C0469B
S11352C03100C9B22000FFF775FC002807D040F276
S11352D03942C649BE48FDF7B7F8C046C04601206A
S11352E010FA06F12000FFF71BFC0020F6B215EBC4
S11352F08601886001223100C9B22000FFF7CAFD8F
S11353000020F6B2711981F84C0070BD60CA00002B
S113531041420F00CCD4000070B504000D0016000B
S1135320002D07D140F24B42B049AE48FDF78CF84E
S1135330C046C046206810F07F00F6B2B04207D2E3
S113534040F24C42A9498C48FDF77EF8C046C0465D
S11353503100C9B22000FFF72DFC002807D04FF41C
S11353608A62A2499A48FDF76FF8C046C0460120F8
S113537010FA06F12000FFF7D3FB0020F6B215EB7C
S1135380860188600020F6B2711981F84C0070BD66
S113539034C3000038B504000D00002D07D140F2DD
S11353A05E4292498F48FDF74FF8C046C0462068D8
S11353B0800005D5E0212000FFF7B2FB0020A8649F
S11353C0002085F85C0031BD9CC5000024CF00009E
S11353D0E8D40000E4E3000014E40000F8B504009D
S11353E00D00002D07D140F2714280497D48FDF740
S11353F02BF8C046C04641F2BF46206A07007C48ED
S1135400074207D041F2BE40060079492000FFF769
S113541080FB93E000200700102F10D2012010FA27
S113542007F12000FFF777FB002806D03900C9B246
S11354302000FFF7D5FB002801D17F1CECE7102FDB
S113544000F0998095F85C00002826D00120B8402F
S1135450812822DA0120B84020280BD0402805D02A
S1135460802816D141F2BC40060061E041F2B4400C
S113547006005DE0A96C2000FFF7C3FE0600002EC5
S113548002D141F2BB40060029002000FFF782FF51
S11354904EE041F2BF4006004AE0781990F84C0013
S11354A0012806D041D303282DD017D3042834D0A3
S11354B03BE015EB870082683900C9B22000FFF792
S11354C028FE0600002E02D141F2B84006003A0040
S11354D0D2B229002000FFF71FFF29E015EB870057
S11354E082683900C9B22000FFF713FE0600002EBF
S11354F002D141F2B84006003A00D2B2290020009D
S1135500FFF70AFF14E041F2B54006003A00D2B2B8
S113551029002000FFF7B6FE0AE00220791981F87D
S11355204C0041F2B640060002E041F2BF400600E2
S1135530012010FA07F12000FFF7F0FA286800288C
S113554008D0686800903B00320029002000D5F89C
S113555000C0E04741F2BF400600206A07005FF048
S1135560FF312000FFF7D7FA00287FF448AF204826
S113557007427FF444AFF1BD8CCA000080B51A48DD
S11355800068002807D140F2FC4218491948FCF78A
S11355905BFFC046C046144801681748FFF71EFF6A
S11355A001BD000048E8010080B50F4840680028AC
S11355B007D140F205520D491048FCF745FFC0469B
S11355C0C046094841680E48FFF708FF01BD0000C6
S11355D0ECE30000CCD10000F4E3000030DA00007A
S11355E0FCE3000004E40000A8C1FF1F9CBF00000E
S11355F00700030018DE0000004002402CDE00001B
S113560000400A4000F10103810704D010F8011B97
S113561089B18107FAD10268B2F10131914311F0E5
S1135620803F04BF50F8042FF6E710F8011B11B1B6
S113563010F8011BFBE7C01A70475AA10EB400B55D
S113564082B003A9009102466B46012103487844C5
S11356500A30FCF75FFE06BC5DF810FB7D87000096
S1135660012001F0BBBF4D601B4213D1094236D16A
S11356702AB18446B0FBF2F002FB10C2704701F07D
S1135680B3BFFCD30022002370470B0002000021AB
S113569000207047904271EB030CF6D370B5B1FA59
S11356A081F4B3FA83F52C1BA340C4F1200532FA2C
S11356B005F63343A2405FF00046E64002E05B0893
S11356C05FEA3202841A71EB030524BF204629469F
S11356D07641F4D302000B003000002170BD012A92
S11356E0CFD970B5140C20D0B1FA81F4B2FA82F596
S11356F0C4F120046419B4F12006D6D3B2405FF09B
S11357000044F440002502E052085FEA3303C61A5D
S113571071EB020E24BF3046714664416D41F3D3F0
S113572002000B002000290070BD0C46B1FBF2F111
S113573002FB11452D0445EA1045B5FBF2F402FBCA
S1135740145580B240EA0545B5FBF2F002FB105255
S113575040EA044070BD4C5FD2B2002A03D1012359
S11357608B40836002E001238B404360704738B56F
S1135770040000200500052D06D2284850F8250015
S1135780A04201D06D1CF6E7052D06D3442224491E
S11357902448FCF759FEC046C046280032BD70B507
S11357A004000D001600002E06D14B221C491E4891
S11357B0FCF74AFEC046C0463078002805D160692F
S11357C00121A9408843606109E072782900200022
S11357D0FFF7C2FF60690121A9400843606170BD01
S11357E070B504002000FFF7C2FF05000F48EDB2BA
S11357F050F825000600D6F8A00070BDF8B50400E6
S11358000D002000FFF7B3FF06000848F6B250F879
S113581026000700C7F8A050F1BD000054DE0000C8
S11358208CC0000064CB00001CE4000040DE0000DB
S113583002002948086012204860002070470200D6
S1135840087A002805D125480860202048600020F7
S113585000E00520704770B40200887A002806D161
S11358601F48006808601E484068486031E0002412
S11358700423E4B2042C11D20889194DAD68E4B2B2
S11358800C2606FB04552D89A84205D1887A0428E4
S113589001D2887A030001E0641CEAE7DBB2042B3E
S11358A001D1052016E00E488068E4B20C2505FB02
S11358B004000068DBB250F82300086008488068E0
S11358C0E4B20C2505FB04004068DBB250F8230069
S11358D04860002070BC7047C004FF1FD404FF1F41
S11358E0D405FF1F2DE9F84304000D0016001F0026
S11358F0DDF82080EDB2F6B256EA450901F076FEF5
S113590014EB0910C06A50F4804014EB0911C8620A
S11359106068400A4002EDB215F00F0150EA4110F0
S1135920F6B216F0010150EA011014EB0911C96A2C
S1135930490A11F00801084347606068400A4002C0
S1135940EDB215F00F0150EA4110F6B216F0010164
S113595050EA011014EB0911C96A490A11F008014F
S113596008435FEA8851890D14EB0912D26A52097F
S113597012F0400252EA014151F08801016001F045
S113598041FEA06890F8940010F0DF00A16881F84F
S113599094000020BDE8F28310B582B00400E06AF0
S11359A0C0F3003014EBC0000C3020620020A06271
S11359B008206062E06A50F40050E062E06A30F46B
S11359C00060E06208200090236A00220021200089
S11359D0FFF788FF13BD10B4FF22836883F8882083
S11359E0826892F8942052F00202836883F894202B
S11359F00022836883F898200022D2B2042A44D279
S1135A0043685B0A5B02D2B212F00F0453EA4413F8
S1135A1000241C6043685B0A5B02D2B212F00F04DC
S1135A2053EA441353F0080300241C6043685B0AE0
S1135A305B02D2B212F00F0453EA441353F0100382
S1135A4000241C6043685B0A5B02D2B212F00F04AC
S1135A5053EA441353F0180300241C60D2B25300D9
S1135A6010EB03130024DC62D2B2530053F00103A1
S1135A7010EB03130024DC628368D2B213EB8203BD
S1135A80002483F8C040521CB7E7002280F8A0200D
S1135A90826892F8942012F0FD02836883F89420BF
S1135AA0FF22836883F88C2089221100826882F89F
S1135AB08410002280F8A120826892F8942012F0C9
S1135AC0DF02836883F8942010BC70472DE9F84303
S1135AD004000D002E88A87810F00F07A8785FEA5C
S1135AE0D01858EA4709E878012807D1B6B2B6F5C4
S1135AF0806F16D340F2FF30060012E0B6B2412E9A
S1135B0001D340200600A068FFB210EB8700A16813
S1135B10FFB211EB870191F8C01051F0010180F838
S1135B20C0105FFA89F914EB0910C06A30F48040A0
S1135B305FFA89F914EB0911C862B6B25FFA89F900
S1135B4014EB0910C06A66F309005FFA89F914EBD3
S1135B500911C8625FFA89F914EB0910C06A30F4BC
S1135B6000605FFA89F914EB0911C8625FFA89F9D8
S1135B7014EB0910C06A30F480605FFA89F914EB01
S1135B800911C8625FFA88F8B8F1010F01D1042045
S1135B9000E00820A168FFB211EB8701A268FFB200
S1135BA012EB870292F8C020104381F8C000FFB2C4
S1135BB0002F07D15FFA88F8B8F1000F02D1200056
S1135BC0FFF7EAFE0020BDE8F2832DE9F04104006E
S1135BD00D0015F00F06EDB2EF0957EA460829004B
S1135BE0C9B2200000F00DFCA068F6B210EB8600EC
S1135BF0002180F8C0105FFA88F814EB0810C06A1E
S1135C00800A80025FFA88F814EB0811C862002049
S1135C10BDE8F0812DE9F04104000D0015F00F06F8
S1135C20EDB2EF0957EA46082900C9B2200000F096
S1135C30E8FB5FFA88F814EB0810C06A50F480603F
S1135C405FFA88F814EB0811C8626068400A4002E1
S1135C50F6B216F00F0150EA4110FFB217F001013D
S1135C6050EA01105FFA88F814EB0811C96A490A6E
S1135C7011F0080108435FFA88F814EB0811C96AA7
S1135C808905890D090451F08C010160A06890F820
S1135C90940010F0DF00A16881F894000020BDE8B2
S1135CA0F0812DE9F84304000D0015F00F07EDB263
S1135CB05FEAD51858EA47095FFA89F914EB091025
S1135CC0C06A30F480605FFA89F914EB0911C86284
S1135CD05FFA89F914EB0910C06A30F400605FFAC6
S1135CE089F914EB0911C8620020C0B2022836D227
S1135CF06168490A4902FFB217F00F0251EA4211E2
S1135D005FFA88F818F0010251EA0211C0B210F0EB
S1135D10010251EAC20109680E0071071DD56168CC
S1135D20490A4902FFB217F00F0251EA42115FFA21
S1135D3088F818F0010251EA0211C0B210F0010211
S1135D4051EAC2015FFA89F914EB0912D26A920589
S1135D50920D120452F008020A60401CC5E7A068C4
S1135D60FFB210EB8700A168FFB211EB870191F835
S1135D70C01011F0FD0180F8C010FFB2002F07D150
S1135D805FFA88F8B8F1000F02D12000FFF704FE93
S1135D90A06890F8940010F0DF00A16881F89400E6
S1135DA00020BDE8F2832DE9F04F85B00400A0681F
S1135DB090F890905FFA89F95FEA19100700C9F327
S1135DC0C0008DF80000C9F380008DF801000820A0
S1135DD0A16881F880006068400A4002FFB217F0B1
S1135DE00F0150EA41109DF8001011F0010150EA32
S1135DF001109DF8011011F0010150EAC100006882
S1135E0001900198C0F3094005000198C0F3830094
S1135E100D2802D15FF0010A01E05FF0000A9DF84D
S1135E20000050EA470080465FFA88F814EB081037
S1135E30C06AC0F38030002800F060815FFA8AFAFB
S1135E40BAF1000F03D09DF8010084F8A3009DF877
S1135E500000012840F085805FFA88F814EB0810F0
S1135E60806A28185FFA88F814EB081188625FFAD0
S1135E7088F814EB0810406A5FFA88F814EB0811EC
S1135E80896A401A06005FFA88F814EB0810C06AA1
S1135E9090F400605FFA88F814EB0811C8625FFAA6
S1135EA088F814EB0810C06A90F480505FFA88F800
S1135EB014EB0811C862002E08D05FFA88F814EBBE
S1135EC00810C06A8005800D85423DD25FFA88F8CB
S1135ED014EB0810806A03905FFA88F814EB08103A
S1135EE0006A02905FFA88F814EB0810C06A30F474
S1135EF080405FFA88F814EB0811C8625FFA88F8EA
S1135F0014EB0810C06A8005800D854240F0E280E1
S1135F10FFB2002F40F0DE8094F8A30014EBC00021
S1135F2010F10C0B5FFA88F814EB0810406ABBF808
S1135F300610884280F0CE80002300223900C9B2C6
S1135F40206801F071F9D9E033005FFA88F814EBA6
S1135F500810026A57F08001C9B2200000F077F9F6
S1135F60CCE0FFB255EA0700002804D100200390DA
S1135F7000200290AEE05FFA88F814EB0810C06AC3
S1135F80C0F34030002828D16068400A4002FFB2C4
S1135F9017F00F0150EA41105FFA88F814EB08116A
S1135FA0C96A490A11F00801084340685FFA88F891
S1135FB014EB0811096A5FFA88F814EB0812926A64
S1135FC05118884206D00022AA4203D2135C5354CB
S1135FD0521CF9E7002284F8A0205FFA88F814EB39
S1135FE00810806A28185FFA88F814EB0811886290
S1135FF05FFA88F814EB0810406A5FFA88F814EB2B
S11360000811896A401A0600FFB2002F13D15FFA03
S11360108AFABAF1000F0ED057F08001C9B22000FD
S113602000F0EFF9E06A50F40060E062E06B50F4D5
S11360300060E0630BE05FFA88F814EB0810C06AB4
S113604090F400605FFA88F814EB0811C8625FFAF4
S113605088F814EB0810C06A90F480505FFA88F84E
S113606014EB0811C8625FFA88F814EB0810406A50
S113607000280AD0002E08D05FFA88F814EB081024
S1136080C06A8005800D854218D25FFA88F814EB47
S11360900810806A03905FFA88F814EB0810006A0D
S11360A002905FFA88F814EB0810C06A30F480405C
S11360B05FFA88F814EB0811C8620BE033005FFA4A
S11360C088F814EB0810026A3900C9B2200000F005
S11360D017F913E08DF811A09DF8000057EAC010DD
S11360E08DF8100002A9206800F0DDFFA06890F888
S11360F0940010F0DF00A16881F8940005B0BDE8B9
S1136100F08F10B584B00400012084F8A1000120B0
S1136110A16881F880000020009010208DF808000C
S11361200020019000208DF809006946206800F0E5
S1136130BAFF1FBD10B504008020A16881F880005B
S1136140E06BC0F38020002804D1E06AC0F3802013
S1136150002807D080212000FFF7A3FD00212000A4
S1136160FFF79FFD10BDF8B504000D00160068464A
S113617021490A680260E4B2002C02D1E4B2002C86
S113618001D0062037E01D48E4B2A42101FB04003D
S1136190070087F8A2406846E4B250F82400B860CB
S11361A01748E4B2402101FB0400F861FF20B968FC
S11361B081F8800000220121380000F052F91148D2
S11361C0E4B24FF4007101FB040078607868000ABF
S11361D0B96881F89C007868000CB96881F8B0004F
S11361E07868000EB96881F8B4003800FFF7F3FB53
S11361F037603D600020F2BDCCE60000F4C5FF1F0F
S113620098C6FF1F0006FF1F01000A00002901D1E4
S113621003201BE0FF20936883F88000906890F8C7
S113622084000020936883F884000020936883F836
S113623098000020936883F89400906890F8000117
S113624050F0C000936883F80001002070472DE9E6
S1136250F04782B004000D0016001F00A046EDB206
S113626015F00F00400050F001095FF0010A18EB2F
S11362700910C06AC0F38030002811D1002018EB47
S11362800911886218EB0910066218EB09104762BD
S113629018EB0910C06A50F4005018EB0911C862D9
S11362A018EB0910C06A8005800DB84205D218EBBE
S11362B00910C06A8005800D070098F8A100002825
S11362C00ED1009718EB0910006A18EB0911896ABE
S11362D00B18012215F00F014046FFF703FB82461D
S11362E018EB0910806A3843002805D10F210D42AC
S11362F002D14046FFF750FB5046C0B2BDE8F687D6
S11363002DE9F04782B004000D0016001F00A046DE
S1136310EDB215F00F005FEA40095FF0010A18EBD7
S11363200910C06AC0F38030002809D1002018EB9E
S11363300911886218EB0910066218EB091047620C
S113634018EB0910C06A50F4005018EB0911C86228
S113635018EB0910C06A8005800DB84205D218EB0D
S11363600910C06A8005800D070018EB0910806AC7
S11363708619D8F81C0000281AD098F8A000002824
S113638016D1412F14D217F0030F03D116F00300D6
S113639000280DD018EB0910C06A30F4005018EB37
S11363A00911C862D8F81C000600012088F8A00072
S11363B098F8A100002808D100973300002215F0B6
S11363C00F014046FFF78EFA8246002F15D10F21A8
S11363D00D4212D118EB0910C06A90F4805018EBEA
S11363E00911C86218EB0910C06A30F4804018EB38
S11363F00911C8624046FFF7CFFA5046C0B2BDE863
S1136400F687FEB504000D00260015F00F012800E4
S1136410C0B2C00950EA4107FFB216EB0710C06AC8
S1136420C0F3803000281AD05FF0FF300190FFB233
S113643016EB0710006A00908DF8085000208DF8C4
S11364400900FFB216EB0710C06A30F48040FFB2B7
S113645016EB0711C8626946306800F024FE00207C
S1136460FEBD2DE9F84F04000D00160027005FF073
S11364700108002C01D10320D6E0EDB2002D1FD07D
S1136480022D53D03DD3042D62D057D3062D73D0A3
S113649068D3082D00F0928077D30A2D00F09A80FB
S11364A0C0F097800C2D00F0B180C0F094800E2DC8
S11364B000F0B680C0F0B3800F2D00F0B280B1E0E0
S11364C00020B96881F80001B868007F400705D54D
S11364D0B868007F50F08000B9680877B86890F811
S11364E0080150F01000B96881F80801B86890F804
S11364F0940050F00100B96881F8940000208046AF
S113650090E0B868007F400705D5B868007F10F0B8
S11365107F00B9680877B86890F8080110F0EF00B8
S1136520B96881F80801002080467BE0002E04D081
S113653031003800FFF7CAFA804673E0002E06D017
S1136540B2469AF800103800FFF73FFB804669E036
S1136550002E06D0B2469AF800103800FFF75AFB16
S113656080465FE0002E06D0B2469AF8001038004C
S1136570FFF797FB804655E0002E05D0B146012079
S1136580A9F80000002080464CE0002E15D0300011
S1136590017811F00F0104290FD2017811F00F01D5
S11365A00278D20952EA410117EB0111C96A890A3A
S11365B011F0010141800021884633E0002E07D00C
S11365C0B2469AF80000B96881F898000020804625
S11365D028E027E026E05FF0000B5FFA8BFBBBF1BD
S11365E0040F0DD25BF08001C9B23800FFF7EDFA59
S11365F05946C9B23800FFF7E8FA1BF1010BECE782
S11366003800FFF7E8F9002080460BE0002E05D0A3
S1136610B24600208AF800000020804602E001E033
S113662000E0FFE74046C0B2BDE8F28FF8B50400D1
S11366302500002C1ED028680600B06890F8800061
S11366400700380702D53000FFF7ADFBF80702D585
S11366503000FFF756FD380602D53000FFF76AFD1B
S1136660B06890F85C010700FFB2002F02D0B06858
S113667080F85C71F1BD4B5EDFF8E803006850F40C
S11366807000DFF8E01308604CF22050DFF8D813F4
S113669008804DF62810DFF8D01308804FF4E97015
S11366A0DFF8C8130880DFF8C8030078C0070DD5E9
S11366B0DFF8C003007800072FD5DFF8B8030078AF
S11366C050F00800DFF8AC13087026E0DFF8A803E8
S11366D0006850F00050DFF8A0130860DFF89C0356
S11366E00068C00519D4DFF89403006830F47050D2
S11366F050F44070DFF884130860DFF8800300680A
S113670050F48070DFF874130860DFF870030068D9
S113671030F40070DFF864130860AA20DFF8601317
S113672008705FF08A70DFF85C130860DFF85803C4
S1136730006830F4402050F40020DFF84C13086067
S1136740DFF84803006830F4403050F48030DFF85C
S11367503C130860DFF83403006830F0407050F0F8
S11367608070DFF828130860DFF82403006850F411
S11367700070DFF81C130860DFF818030068DFF806
S113678018130840DFF80C130860DFF810030068E2
S1136790C1490840C14908600020C1490870C14886
S11367A00078C0B210F0BF0050F02400BD4908705A
S11367B08020BD4908700020BC490870A220BC4953
S11367C00870BC4800788007FBD5BA480078C0063A
S11367D0FBD4B948007810F01F00B74908700120B5
S11367E0B64908700E20B64908700020B5490870F3
S11367F0B348007850F04000B1490870AD480078C3
S11368004006FBD5AA48007810F03F00A84908705C
S1136810A8480078C0B210F00C000C28F8D1AA489F
S11368200078C0B20028FAD1A84800680009000125
S113683050F00200A5490860A5480068000900015D
S1136840A349086070479A4A1278C0231A4240F05C
S1136850C7809B4A1278520600F18180944A1278CC
S1136860520742D4914A1278D2B212F00302002A9B
S113687002D0012A03D006E0964A100005E04FF446
S11368800042100001E0944A1000864A1278302336
S11368901A421FD0854A1278D2B212F00302012A9A
S11368A018D0834A1278D2B212F03802302A05D0B6
S11368B0382A07D14FF4C062110012E04FF4A062ED
S11368C011000EE020227A4B1B78C3F3C2039A40D6
S11368D0110006E00122764B1B78C3F3C2039A40F1
S11368E0110089B2B0FBF1F002E04FF40042100055
S11368F0714A1278D2B212F0E002002A0ED0202A95
S113690010D0402A12D0602A14D0802A16D0A02A8F
S113691018D0C02A1AD0E02A1CD01FE04FF42072ED
S1136920504395E04FF4A062504391E04FF4F0627D
S113693050438DE04FF42062504389E04FF43772A6
S1136940504385E04FF4B762504381E040F695022E
S113695050437DE040F67132504379E078E0594A83
S11369601278D20616D4554A1278D2B212F007021F
S1136970521C1100574A89B2B2FBF1F21000504A7E
S11369801278D2B212F01F021032110089B24843B9
S113699040085DE0514A126812F00C0F02D14D4AD2
S11369A0100055E04D4A1268C2F3051211004B4A1B
S11369B0126812F00C02042A02D189B2890007E09D
S11369C0464A126812F00C02082A01D189B2490021
S11369D0434A89B292FBF1F210001222504337E08D
S11369E0334A1278D2B212F0C002402A14D12D4A8E
S11369F01278D20703D44FF40042100028E0012299
S1136A00274B1B78C3F342039A401100354A89B2DD
S1136A10B2FBF1F210001BE0254A1278D2B212F058
S1136A20C002802A13D1214A1278D2B212F0030292
S1136A30002A02D0012A03D006E0264A100007E00B
S1136A404FF40042100003E0234A100000E007E086
S1136A500C4A1268120F521CB0FBF2F2224B1A605D
S1136A607047000088ED00E00E200540002005403E
S1136A7000F0074002D007403C80044010D003409F
S1136A8000E0074044800440007004400480044057
S1136A903880044048900440FFF8FFFE4C900440C6
S1136AA00840064001400640005006400C400640A5
S1136AB000400640064006400340064004400640AD
S1136AC005400640104006401240064048800440FD
S1136AD0648004400024F400006CDC0200210A40BD
S1136AE000389C1C00093D008804FF1F70B5040099
S1136AF00D0000F07BFD00200600002E16D1DFF80B
S1136B007403142101FB0600006800280CD0DFF890
S1136B106403142101FB0600807CE4B2844203D1A7
S1136B2000F070FD012022E0761CE6E7002006005C
S1136B30002E19D1DFF83C03142101FB0600006884
S1136B4000280FD1DFF82C03142101FB0600847404
S1136B50DFF82003142101FB0600286000F052FD39
S1136B60002004E0761CE3E700F04CFD022070BD39
S1136B7038B50400002500F039FD002D2BD1DFF8D5
S1136B80F402142101FB05000068002821D0DFF87D
S1136B90E402142101FB0500807CE4B2844218D194
S1136BA00020DFF8D012142202FB05110860002037
S1136BB0DFF8C012142202FB051148600020DFF840
S1136BC0B412142202FB0511887400F01BFD00208E
S1136BD004E06D1CD1E700F015FD042032BD70B552
S1136BE004000D00002600F001FD002E11D1A14883
S1136BF0142101FB06000068844208D19D48142139
S1136C0001FB0600286000F0FDFC002004E0761C77
S1136C10EBE700F0F7FC042070BD70B504000D0034
S1136C20002600F0E3FC002E1AD19248142101FB47
S1136C3006000068002811D08E48142101FB0600CC
S1136C40807CE4B2844209D18A48142101FB060005
S1136C500068286000F0D6FC002004E0761CE2E71F
S1136C6000F0D0FC042070BD2DE9F04782B0040090
S1136C700D0016005FF001095FF0010A002E01D13A
S1136C80042053E069462000FFF7A9FF81465FFA1C
S1136C9089F9B9F1000F01D0042047E000208046B3
S1136CA000984068007A5FFA88F880453CD200205A
S1136CB00700FFB2022F34D26F48FFB210EB071067
S1136CC0007B0099496809685FFA88F80C2202FB86
S1136CD0081189680979884221D13200EDB229006E
S1136CE00098406800685FFA88F80C2303FB0800EA
S1136CF04068614BFFB213EB07139B6898478146CA
S1136D005FFA89F9B9F1050F01D105200EE05FFAA8
S1136D1089F9B9F1000F01D10020824601E07F1CFE
S1136D20C7E718F10108BBE75046C0B2BDE8F687D3
S1136D30F8B504000D001600012769462000FFF78E
S1136D404EFF0700FFB2002F02D03800C0B214E09B
S1136D50012D08D10099200000F0F1FF009A0221D2
S1136D602000FFF781FF320029002000009B5B68B0
S1136D705B68984707003800C0B2F2BD2DE9F843BC
S1136D8004000D0016005FF00109002E04D0002D50
S1136D9002D06868002801D1042069E06946200017
S1136DA0C0B2FFF7A3FE81465FFA89F9B9F1000F7B
S1136DB002D04846C0B25BE000984560009A2F4973
S1136DC02000C0B200F084F981465FFA89F9B9F174
S1136DD0000F0AD00098006800F011FA2000C0B239
S1136DE0FFF7C6FE4846C0B242E000208046009845
S1136DF04068007A5FFA88F8804534D200200700A2
S1136E00FFB2022F2CD20098406800685FFA88F81D
S1136E100C2101FB0800806800791749FFB211EBCF
S1136E200711097B884219D10098406800685FFA0D
S1136E3088F80C2101FB0800021D009840680068D6
S1136E405FFA88F80C2101FB08012000C0B20A4B4C
S1136E50FFB25FEA071C5CF8033098477F1CCFE75A
S1136E6018F10108C3E70098006830604846C0B2D2
S1136E70BDE8F28390C5FF1FACD40000316D000063
S1136E8070B504000D0000F0B1FB00200600002ED8
S1136E9015D12948502101FB0600006800280CD0B8
S1136EA02548502101FB060090F84D00E4B28442CD
S1136EB003D100F0A7FB012020E0761CE7E70020C7
S1136EC00600002E17D11C48502101FB0600006863
S1136ED000280ED11848502101FB060080F84D40CF
S1136EE01548502101FB0600286000F08BFB0020B0
S1136EF004E0761CE5E700F085FB022070BD10B5C8
S1136F00040000F073FB00202060002084F84D0092
S1136F1000F078FB002010BD10B402000620D2B2AD
S1136F201300002B012B04D8044B0B600023180022
S1136F30FFE7C0B210BC7047A4C5FF1FC0DD00004E
S1136F402DE9F84304000D0016001F00A0465FF071
S1136F500109B8F1000F01D1032023E0D8F804009F
S1136F6000281BD028060CD53B0032002900C9B2EA
S1136F70D8F80000D8F804C0DCF808C0E04781461F
S1136F800EE03B0032002900C9B2D8F80000D8F85E
S1136F9004C0DCF80CC0E047814601E006208146CD
S1136FA04846C0B2BDE8F2832DE9F04104000D006B
S1136FB0160027005FF00108002F01D103200FE025
S1136FC07868002808D032002900C9B238687B6884
S1136FD05B699847804601E0062080464046C0B27F
S1136FE0BDE8F08138B504000D0000220B2120001B
S1136FF0FFF7DAFF022084F84E00002084F84C00EA
S11370000020082809D2002114EBC002D16000211D
S113701014EBC0021161401CF3E70022012120009F
S1137020A3689847002032BD2DE9F04184B00400E4
S11370300D00287A10F00F06287AC7095FF00108BE
S1137040287A102805D129002000FFF7CBFF8046BD
S113705024E0F6B2042E21D27000C0B2FFB238434D
S113706014EBC000C068002818D028680090686835
S11370700190687A8DF808007000C0B2FFB23843FE
S113708014EBC0000269694620007300DBB2FFB252
S11370903B4314EBC303DB68984780464046C0B2C9
S11370A004B0BDE8F081F8B504000D0026002F00FF
S11370B0002D01D0002C01D1032008E0B068002885
S11370C001D1012003E039003000FFF7ADFFF2BD2C
S11370D02DE9F04182B004000D001600002000905C
S11370E0002E01D1032080E069462000C0B2FFF7E2
S11370F0C7FE80465FFA88F8B8F1000F02D0404618
S1137100C0B272E000988560009880F84D4000207D
S1137110009981F84C0000200700082F0BD20020B2
S1137120009911EBC701C8600020009911EBC70159
S113713008617F1CF1E70098011D2000C0B2FFF731
S1137140EBFE80465FFA88F8B8F1000F05D000988E
S1137150FFF7D5FE4046C0B247E0009840680028DB
S113716004D10098FFF7CBFE06203EE0009840686B
S11371700068002818D0009840684068002813D0A0
S113718000984068806800280ED000984068C06865
S1137190002809D0009840680069002804D00098AD
S11371A040684069002804D10098FFF7A8FE072032
S11371B01BE0009A00992000C0B2009B5B681B682A
S11371C0984780465FFA88F8B8F1000F05D0009818
S11371D000F015F84046C0B207E00220009981F89B
S11371E04E00009830604046C0B2BDE8F68110B54C
S11371F00400002200212000FFF7D6FE10BD38B5A0
S113720004002500002D01D103200CE0686800284B
S113721005D02868696849688847002068602800A4
S1137220FFF76DFE002032BDF8B504000D00160016
S11372301F003B00320015F00F0050F08001C9B26E
S11372402000FFF77DFEF2BDF8B504000D00160026
S11372501F003B00320015F00F012000FFF770FE05
S1137260F2BDF8B504000D0026000127002E01D15F
S113727003200EE07068002807D02900C9B23068E6
S1137280726812699047070001E006200700380081
S1137290C0B2F2BD2DE9F84304000D00160027002A
S11372A0002F01D103202EE0002D01D0002E01D1AA
S11372B0042028E0A87810F00F008046A878C009C0
S11372C081465FFA88F8B8F1040F1BD25FEA4800E0
S11372D0C0B25FFA89F959EA000017EBC0003168BF
S11372E0C1605FEA4800C0B25FFA89F959EA000058
S11372F017EBC000716801612A0002212000FFF72A
S113730053FE00E00420BDE8F2832DE9F3410400BC
S113731025009DF8040010F00F069DF80400C7092D
S11373205FF00108002D01D103201CE001AA032114
S11373302000FFF739FE8046F6B2042E12D2700008
S1137340C0B2FFB2384315EBC0000021C160700029
S1137350C0B2FFB2384315EBC000002101614046C2
S1137360C0B200E00420BDE8F68113B504009DF826
S1137370040010F00F00042805D201AA0421200003
S1137380FFF712FE00E0042016BD13B504009DF8BB
S1137390040010F00F00042805D201AA05212000E2
S11373A0FFF702FE00E0042016BD2DE9F0410400C1
S11373B00D0016005FF00108002E01D1042040E00A
S11373C0EDB2022D0AD03AD3042D23D00DD3062DCD
S11373D012D026D3082D2BD015D330E032000C2147
S11373E02000FFF7E1FD804629E032000D21200056
S11373F0FFF7DAFD804622E037000020804694F84B
S11374004E0038701BE037000020804694F84C0092
S1137410387014E0320006212000FFF7C5FD8046D5
S11374200DE0320007212000FFF7BEFD804606E094
S1137430320009212000FFF7B7FD8046FFE74046F0
S1137440C0B2BDE8F081F8B504000D0016000127B4
S1137450EDB22800032806D006280BD0072811D047
S1137460092826D02CE032000E212000FFF79CFDD5
S1137470070025E0002E04D000200700307884F8AF
S11374804E001DE094F84E0003280AD0002E0FD0C1
S113749000200700307884F84C00032084F84E0064
S11374A006E014F14C0208212000FFF77DFD0700DF
S11374B006E032000A212000FFF776FD0700FFE70F
S11374C03800C0B2F2BDFEE762F30F2262F31F423E
S11374D0401810F0030308D0C91A1FD3DB0748BFB4
S11374E000F8012D28BF20F8022D130030B41446F3
S11374F01546103928BF20E93C00FAD8490728BFAF
S113750020E90C0048BF40F8042D890028BF20F86A
S1137510022D48BF00F8012D30BC7047C91818BFB0
S113752000F8012DCB0728BF00F8012D7047FEE7B6
S113753062B38B0708D0521E11F8013B00F8013BDF
S113754000F024808B07F6D1830740F0208000BF31
S1137550103A07D330B4B1E83810103AA0E8381024
S1137560F9D230BC530724BFB1E80810A0E80810D2
S113757044BF51F8043B40F8043BD20724BF31F820
S1137580022B20F8022B44BF0B7803707047083A93
S113759007D3B1E80810083A40F8043B40F804CB9C
S11375A0F7D25307E4E7FEE70CB41CB5044604A87D
S11375B001900A46009401AB6946074878441830A4
S11375C0FAF7A8FE009A0021117000285CBF009809
S11375D0001B16BC5DF80CFBF7A0FFFF202109037C
S11375E026311820ABBEF9E77047FEE70D48007856
S11375F0002800D172B60B480078401C0949087075
S11376007047000007480078002804D00548007837
S1137610401E0449087003480078002800D162B66F
S113762070470000DAC7FF1F2DE9FC4104000D007C
S113763016001F005FF0050801AA06212068FFF765
S1137640B4FE9DF80400012806D09DF8040000282B
S113765002D04046C0B23EE028781F2108420FD134
S113766014F1100204212068FFF79FFE8046207C5D
S113767010F003002082208A20820220386025E056
S1137680287810F01F00012806D100208046002031
S113769020820220386019E0287810F01F000228A8
S11376A014D1A8888DF800000020ADF802006A46C5
S11376B005212068FFF779FE80469DF8020010F04E
S11376C003002082208A20820220386014F11000F6
S11376D030604046C0B2BDE8F6812DE9F04182B089
S11376E004000D0016001F005FF0050800208DF84F
S11376F000000DF1010206212068FFF756FE9DF8F7
S11377000100012806D09DF80100002802D040465F
S1137710C0B24DE06878032802D101208DF8000042
S113772028781F21084209D1688801283ED16A4679
S113773010212068FFF7FCFA804637E0287810F023
S11377401F00022832D1688800282FD128790F2100
S113775008421AD19DF8000000280BD0287910F0B7
S11377600F00A98889B2C9090143C9B22068FFF78B
S1137770FCFD0AE0287910F00F00A98889B2C90934
S11377800143C9B22068FFF700FE9DF800000028FD
S113779006D02A1D05212068FFF766FA804605E019
S11377A02A1D06212068FFF75FFA80464046C0B2D2
S11377B0BDE8F6812DE9F04182B004000D00160009
S11377C01F005FF005086A4606212068FFF7EDFDFB
S11377D09DF8000003280AD09DF80000012806D077
S11377E09DF80000022802D04046C0B223E09DF874
S11377F00000032809D068888DF800006A46072134
S11378002068FFF720FE804613E00022072120684D
S1137810FFF719FE80465FFA88F8B8F1000F08D127
S113782001208DF800006A4606212068FFF70BFE50
S113783080464046C0B2BDE8F6812DE9FF4704000A
S11378400D0016001F005FF0050A68885FEA102823
S1137850B5F802906A4606212068FFF7A6FD9DF858
S1137860000001280AD09DF80000002806D09DF8E9
S11378700000022802D05046C0B231E0E8880290ED
S11378805FFA88F8B8F1010F06D101AA092120682E
S1137890FFF74EFA82461DE05FFA88F8B8F1020F4E
S11378A008D18DF80C9001AA0A212068FFF740FA4C
S11378B082460FE05FFA88F8B8F1030F0AD18DF819
S11378C00E90A888ADF80C0001AA0B212068FFF7E0
S11378D02FFA824601983060029838605046C0B250
S11378E004B0BDE8F087F8B504000D0016001F00D1
S11378F06A4606212068FFF758FD9DF8000001281C
S113790005D09DF80000002801D005200AE00120E0
S1137910386014F11000306014F110021121206855
S1137920FFF706FAF2BDF8B504000D0016001F00BB
S11379306A4606212068FFF738FD9DF800000128FB
S113794005D09DF80000002801D005201CE000208F
S11379508DF800006A4606212068FFF774FD6888E8
S1137960002807D101208DF800006A46062120680E
S1137970FFF769FDAA1C03212068FFF775F9AA1C0B
S113798007212068FFF7D4F9F2BD2DE9F04182B058
S113799004000D0016001F005FF005086A4606216A
S11379A02068FFF702FD9DF80000002802D0404641
S11379B0C0B20DE00120386014F110003060287965
S11379C0C0B2208214F1100212212068FFF7B0F92E
S11379D0BDE8F681F8B504000D0016001F006A46E4
S11379E006212068FFF7E1FC9DF80000002801D083
S11379F0052011E0A888A978C9B251EA00202082A4
S1137A0014F1100204212068FFF72EF914F110027A
S1137A1008212068FFF78CF9F2BD2DE9F04182B00E
S1137A2004000D0016001F005FF005086A460621D9
S1137A302068FFF7BAFC9DF80000002802D04046F9
S1137A40C0B20FE0A888208214F110020821206837
S1137A50FFF7ABFC804614F1100030600220386060
S1137A604046C0B2BDE8F6812DE9F84F04000D0090
S1137A7093461E000A9FDDF82C805FF001095FF039
S1137A80010A5FFA8BFBBBF1050F16D12878602140
S1137A9008420AD02878000607D4E888002804D0D1
S1137AA0F6B2002E01D1002082465FEACA11C9B2A3
S1137AB02000FFF75AFC81461EE0E888D8F8001041
S1137AC0884202D2E888C8F80000D8F800303A6842
S1137AD000212000FFF7A8FB81465FFA89F9B9F17C
S1137AE0000F09D12878000606D5002300220021C2
S1137AF02000FFF7A9FB81464846C0B2BDE8F28FDB
S1137B002DE9F0479EB004000D00160000200390FC
S1137B10002004905FF00508686810F1010F01D09F
S1137B20002E02D14046C0B206E1B2461AF1080066
S1137B30070002AA06212000FFF737FC287A002854
S1137B4000F0AF806868082802D12868002802D1B4
S1137B504046C0B2F0E0D5F80090B9F80200788051
S1137B60B9F80400B880B9F80600F88099F8010063
S1137B70787099F80000387038786021084212D182
S1137B808948797850F8210000287DD004AB03AAF5
S1137B9039005046DFF810C297F801E05CF82EC0B7
S1137BA0E047804670E0F888002842D03878000624
S1137BB03FD4F888002815D03878800612D50020E4
S1137BC0129001208DF850001197F888139011AA93
S1137BD001212000FFF748F880461398049012987A
S1137BE0039017E0F888002814D03878400611D59F
S1137BF000200E9001208DF840000D97F8880F901A
S1137C000DAA0F212000FFF793F880460F980490E7
S1137C100E9803905FFA88F8B8F1000F34D1FB880E
S1137C20039A00212000FFF70FFB80464046C0B2B4
S1137C3082E03878800612D500200A9001208DF861
S1137C4030000997F8880B9009AA01212000FFF75A
S1137C500BF880460B9804900A98039014E0387847
S1137C60400611D50020069001208DF820000597CC
S1137C70F888079005AA0F212000FFF759F88046DD
S1137C80079804900698039004A8019003A8009014
S1137C9000234246D2B239002000FFF7E5FE8046B9
S1137CA048E09DF8080003280CD104AB03AA39006E
S1137CB05046DFF8F4C097F801E05CF82EC0E047C6
S1137CC0804637E06868002834D0F888002831D02E
S1137CD0387800062ED4387880060ED528681A9095
S1137CE000208DF87000199768681B9019AA01216B
S1137CF02000FEF7B9FF804610E0387840060DD525
S1137D002868169000208DF8600015976868179011
S1137D1015AA0F212000FFF70BF8804604A8019054
S1137D2003A8009001234246D2B239002000FFF795
S1137D309BFE80464046C0B21EB0BDE8F0877FB5CA
S1137D4004000D0019480290039501208DF80400E9
S1137D5000208DF8030080208DF802004020ADF84B
S1137D60000002AA69462000FFF794FA0600F6B262
S1137D70002E02D03000C0B213E000208DF80200C3
S1137D8002AA69462000FFF785FA0600F6B2002E23
S1137D9006D080212000FFF7B8FA3000C0B200E01E
S1137DA0002004B070BD00007CC80000017B00000E
S1137DB00EB430B5040003A8050029002000F9F72B
S1137DC01DFC30BC5DF810FB80B501F0CDF8DFF888
S1137DD0540B01F0EEF8DFF8500B01F0EAF8DFF88D
S1137DE04C0B01F0E6F8DFF8980C01F0E2F801BD65
S1137DF0F0B589B004000D0000260020009001A811
S1137E001C21F9F761FC0027E4B2022C07D0DFF84B
S1137E10140B8168DFF8E80CFFF7CAFF1EE06868FE
S1137E2006003100684601F0D3FA002807D1DFF8D4
S1137E30F40A8168DFF8C80CFFF7BAFF0EE001A965
S1137E400098C0B2F8F7F0FA0700380000F008F81C
S1137E50002F03D101A9009800F039F809B0F0BD52
S1137E6038B5040000257FF00040854207D0DFF8D4
S1137E70400B50F83500844201D06D1CF3E7DFF865
S1137E80300B10EBC500436822002100DFF8740CAE
S1137E90FFF78EFF31BD010000200200DFF8100B58
S1137EA050F832007FF0004398420DD0DFF8000B09
S1137EB050F83200814205D1DFF8F40A10EBC20019
S1137EC0406803E0521CE9E7DFF83C0C7047F8B562
S1137ED004000D00BAA0FFF76BFF200001283DD07D
S1137EE002285BD0032874D0042878D005287CD0DD
S1137EF0062800F08080072800F08380082800F01E
S1137F009B800A2800F0A1800B2800F0A9800C288F
S1137F1000F0AC800E2800F0CC800F2800F0CF8059
S1137F20102800F0D280112800F0D580122800F02B
S1137F30DF80132800F0F180142800F0FB8015285E
S1137F4000F0FE80162800F00181172800F020813F
S1137F50182813D01A2800F024812BE12879C0B204
S1137F6000906868C0F307236868C0F30742686834
S1137F70010EDFF8980BFFF71BFF1FE12879C0B251
S1137F8000906868C0F307236868C0F30742686814
S1137F90010EDFF87C0BFFF70BFF0FE1DFF8740B2A
S1137FA0FFF706FF6E680027002E11D0F0070CD5EE
S1137FB0DFF8640B50F82710A2A0FFF7F9FE700851
S1137FC0002802D0A0A0FFF7F3FE76087F1CEBE7A1
S1137FD0F4E06968DFF8440BFFF7EAFEEEE0696855
S1137FE0DFF83C0BFFF7E4FEE8E06968DFF8340BE8
S1137FF0FFF7DEFEE2E06968DFF82C0BFFF7D8FE3E
S1138000DCE0DFF8280BFFF7D3FE6E680027002EB4
S113801011D0F0070CD5DFF8180B50F8271089A001
S1138020FFF7C6FE7008002802D087A0FFF7C0FE45
S113803076087F1CEBE7C1E06868FFF72CFF0100BE
S1138040DFF8F00AFFF7B4FEB8E06868002801D052
S11380507EA100E07EA1DFF8E00AFFF7A9FEADE013
S11380606968DFF8D80AFFF7A3FEA7E0A868696883
S1138070401A461C012E01D1002006002869E96837
S1138080401A471C012F01D100200700DFF8280CFB
S1138090FFF78EFE3300AA686968DFF8200CFFF74B
S11380A087FE3B002A69E968DFF8140CFFF780FEBD
S11380B084E06968DFF80C0CFDF7C0FA7EE06968BB
S11380C0DFF8040CFFF774FE78E06968DFF8FC0B56
S11380D0FFF76EFE72E06868002802D0DFF8F01B3C
S11380E001E0DFF8F01BDFF8F00BFFF761FE65E05D
S11380F0DFF8E80BFFF75CFE0126286886420BD206
S113810055F8260082B255F82600010CDFF8D00B92
S1138110FFF74EFE761CF0E750E06868002802D0B6
S1138120DFF8C01B01E0DFF8C01BDFF8740CFFF7B9
S11381303FFE43E06968DFF86C0CFFF739FE3DE071
S11381406968DFF8640CFFF733FE37E0DFF85C0C96
S1138150FFF72EFE6868002804D1DFF8540CFFF7FF
S113816027FE14E06868012804D1DFF8480CFFF703
S11381701FFE0CE06868022804D1DFF83C0CFFF70E
S113818017FE04E06968DFF8340CFFF711FE15E010
S11381906868FFF780FE0100DFF8240CFFF708FE93
S11381A00CE06868FFF777FE0100DFF8180CFFF7B2
S11381B0FFFD03E0DFF8100CFFF7FAFDF1BD00004E
S11381C00D0A2000F0B583B004000D000026002045
S11381D00190002000900027E4B2032C07D0DFF8C0
S11381E048078168DFF8E00CFFF7E2FD28E06868E3
S11381F00600310001A801F0EBF8002807D1DFF8F0
S113820028078168DFF8C00CFFF7D2FD18E0A868E2
S113821006003100684601F0DBF8002807D1DFF8DA
S113822008078168DFF8A00CFFF7C2FD08E0009999
S11382300198C0B2F8F752F907003800FFF710FEB2
S1138240F7BD0000257300002C2000004F4E0000F5
S11382504F46460070B504000D000026F8F782F979
S113826006003000FFF7FCFD70BD30B583B004009C
S11382700D00DFF8580CD0E90023CDE90023E4B267
S1138280022C07DB6A4629002000C0B200F054F833
S1138290002850D19DF80000012809D1DFF8300CE6
S11382A0FFF786FD0199DFF82C0CFFF781FD38E01C
S11382B09DF80000022809D1DFF81C0CFFF778FDB7
S11382C00199DFF8100CFFF773FD2AE09DF8000018
S11382D0032810D10198B0F5964F02D24FF46140B3
S11382E00190DFF8F80BFFF763FD0199DFF8F00B5D
S11382F0FFF75EFD15E09DF80000042809D1DFF8C2
S1138300E40BFFF755FD0199DFF8C80BFFF750FDAB
S113831007E0DFF86C078168DFF8AC0BFFF748FD76
S113832009E001A99DF80000F8F73FFF01999DF8C5
S11383300000F8F778FF37BD2DE9F04104000D0087
S1138340160000275FF00008012080465FFA88F8D5
S1138350E4B2A0455DD25FFA88F855F828000078A9
S11383602D2825D15FFA88F855F82800407862282E
S11383701ED15FFA88F855F828008078002811D0BB
S11383805FFA88F855F82800801C0700310038008F
S113839000F042F8002839D0DFF84C0BFFF708FD55
S11383A0012037E0DFF8440BFFF702FD012031E044
S11383B05FFA88F855F8280000782D2826D15FFA4E
S11383C088F855F82800407866281FD15FFA88F8A5
S11383D055F828008078002812D05FFA88F855F8FC
S11383E02800801C0700321D3178380000F042F864
S11383F000280BD0DFF8F80AFFF7DAFC012009E0C7
S1138400DFF8F00AFFF7D4FC012003E018F10108BB
S11384109CE70020BDE8F08138B504000D00210080
S1138420BBA000F0BBFF012803D10120287000206D
S11384301FE02100B7A000F0B1FF012803D1022002
S11384402870002015E02100DFF8AC0A00F0A6FF38
S1138450012803D10320287000200AE02100AEA0E7
S113846000F09CFF012803D104202870002000E0C4
S1138470012032BD70B582B004000D00160000204A
S113848000902100684600F0A3FF002801D10120DC
S11384902FE00098642810D30098B0F57A7F0CD8A8
S11384A0EDB2012D05D0EDB2022D02D0EDB2042DB6
S11384B003D10098306000201BE0EDB2032D17D1EA
S11384C00098B0F5964F0FD00098B0F5164F0BD02A
S11384D00098B0F5614F07D00098B0F5E13F03D0A4
S11384E00098B0F5613F03D100983060002000E0AF
S11384F0012076BD70B504000D000026002001F0B7
S113850038F80600002E04D1DFF8F409FFF750FC18
S113851011E0032E04D1DFF8EC09FFF749FC0AE06F
S1138520042E04D1DFF8E009FFF742FC03E0DFF892
S1138530DC09FFF73DFC70BD2DE9F04782B0040073
S11385400D0000260020009000275FF000085FF077
S11385500009E4B2032C07D0DFF8B4098168DFF81E
S11385606809FFF725FC5DE068680600310068468D
S113857000F02EFF002807D1DFF894098168DFF8A6
S11385804809FFF715FC4DE0A86806003000FDF728
S113859039F807005FF0000ABA4518D21AF8060045
S11385A001F016F800280FD11AF806007B280BD02A
S11385B01AF806007D2807D0DFF854098168DFF82F
S11385C00809FFF7F5FB2DE01AF1010AE4E730781A
S11385D07B2824D170787B2821D1B61C3000FDF78C
S11385E011F807007F1EB85D7D2818D17F1EB85D85
S11385F07D2814D15FF0000ABA450AD251463000F2
S113860000F051FF08F8060018F101081AF1020AF7
S1138610F2E7424631000098F8F7FCF881464846F4
S1138620FFF71EFCBDE8F3872DE9F0438BB004008F
S11386300D0000260020019002A82021F9F744F83B
S11386400027002000905FF00008E4B2032C07D05C
S1138650DFF8C0088168DFF8A804FFF7A9FB54E03D
S113866068680600310001A800F0B2FE002807D1B6
S1138670DFF8A0088168DFF88804FFF799FB44E07D
S1138680A86806003100684600F0A2FE002807D161
S1138690DFF880088168DFF86804FFF789FB34E0BD
S11386A00098002831D00098212802D32020070008
S11386B001E0009807003A0002A90198F8F7EFF8E2
S11386C080464046FFF7CCFBB8F1000F1DD100985F
S11386D0C01B00900198381801905FF00009B9455B
S11386E0DED2082099FBF0F101FB1091002902D1A0
S11386F0AEA0FFF75DFB02A819F80010DFF8180818
S1138700FFF756FB19F10109E9E70BB0BDE8F08367
S1138710737069006932630063616E00FEB5040022
S11387200D000026002002900020009000200190FF
S11387300027E4B2052C07D0DFF8E0078168DFF8F2
S11387408807FFF735FB70E068680600310002A86F
S113875000F03EFE002807D1DFF8C0078168DFF88B
S11387606807FFF725FB60E0A8680600310001A850
S113877000F02EFE002807D1DFF8A0078168DFF89B
S11387804807FFF715FB50E0E8680600310068462B
S113879000F01EFE002807D1DFF880078168DFF8AB
S11387A02807FFF705FB40E0286906003100DFF8E1
S11387B0700700F0F3FD012802D1009800902BE02F
S11387C03100DFF8600700F0E9FD012805D10098C9
S11387D0009950EA014000901EE03100DFF848079C
S11387E000F0DCFD01280FD10098009950EA012027
S11387F000900098009950EA012000900098009998
S113880050EA0120009007E0DFF810078168DFF8E4
S1138810B806FFF7CDFA08E0019A00990298F8F734
S113882083F807003800FFF71BFBF7BD2DE9F84F6D
S113883004000D00002600275FF000085FF0000927
S11388405FF0000AE4B2022C07D0DFF8E00681688A
S1138850DFF87406FFF7ACFA62E0686806003000DF
S1138860FCF7D0FE8246BAF1100F07D0DFF8BC0641
S11388708168DFF85406FFF79BFA51E05FF0000BC4
S1138880D34510D21BF8060000F0A2FE002807D141
S1138890DFF898068168DFF83006FFF789FA3FE0D1
S11388A01BF1010BECE70021300000F0FCFD000699
S11388B007000221300000F0F6FD57EA00400700EF
S11388C00421300000F0EFFD57EA002007000621E4
S11388D0300000F0E8FD384307000821300000F0C4
S11388E0E2FD000680460A21300000F0DCFD58EA73
S11388F0004080460C21300000F0D5FD58EA0020ED
S113890080460E21300000F0CEFD50EA080080467B
S113891041463800F8F74FF881464846FFF7A0FA79
S1138920BDE8F18F8400FF1FDC02FF1FF402FF1F6C
S1138930F0B583B004000D00002600200190002053
S113894000900027E4B2032C07D0DFF8E405816827
S1138950DFF87405FFF72CFA27E068680600310099
S113896001A800F035FD002807D1DFF8C4058168AF
S1138970DFF85405FFF71CFA17E0A8680600310079
S1138980684600F025FD002807D1DFF8A4058168BA
S1138990DFF83405FFF70CFA07E000990198F7F7C0
S11389A092FE07003800FFF75BFAF7BD0D0A2000BE
S11389B09C00FF1F70B504000D000026F7F748FE69
S11389C006003000FFF74CFA70BD70B504000D00CE
S11389D00026F7F702FE06003000FFF741FA70BDEB
S11389E0FEB504000D000026002002900020019036
S11389F0002000900027E4B2042C07D0DFF83405EF
S1138A008168DFF8C404FFF7D3F938E0686806002A
S1138A10310002A800F0DCFC002807D1DFF81405BF
S1138A208168DFF8A404FFF7C3F928E0A86806000A
S1138A30310001A800F0CCFC002807D1DFF8F404D1
S1138A408168DFF88404FFF7B3F918E0E8680600EA
S1138A503100684600F0BCFC002807D1DFF8D404DC
S1138A608168DFF86404FFF7A3F908E0009A01992C
S1138A700298F7F7E3FF07003800FFF7F1F9F7BDB5
S1138A800C03FF1FF0B583B004000D000026002086
S1138A900190002000900027E4B2032C07D0DFF8F7
S1138AA098048168DFF82004FFF782F927E06868FA
S1138AB00600310001A800F08BFC002807D1DFF884
S1138AC078048168DFF80004FFF772F917E0A868FA
S1138AD006003100684600F07BFC002807D1DFF86F
S1138AE058048168DFF8E003FFF762F907E00099B2
S1138AF00198F7F7EAFF07003800FFF7B1F9F7BD6F
S1138B0020D0000044D00000A0DC0000ACD3000062
S1138B1084D80000A0D800006CD40000BCD80000A9
S1138B20B8DC0000CCD30000D0DC0000E8DC00009E
S1138B3000C4000000DD000018DD0000D8D80000EB
S1138B402DE9F04784B004000D005FF00009002017
S1138B5002900020019000260020009000275FF082
S1138B600008E4B2042C06D0DFF8D0038168D648AC
S1138B70FFF71EF99EE068688146494602A800F0A6
S1138B8027FC002806D1DFF8B4038168CE48FFF73C
S1138B900FF98FE0A8688146494601A800F018FC47
S1138BA0002806D1DFF894038168C748FFF700F96D
S1138BB080E0E8688146019804280FD14946684658
S1138BC000F006FC002806D1DFF870038168BE4877
S1138BD0FFF7EEF86EE00020070061E00198082836
S1138BE058D199F80000302805D199F80100782867
S1138BF001D119F102095FF0000ABAF1100F0ED287
S1138C001AF8090000F0E4FC002805D1CB4881687B
S1138C10AD48FFF7CDF84DE01AF1010AEDE7002168
S1138C20484600F040FC000600900221484600F04F
S1138C303AFC0099C0B251EA004000900421484631
S1138C4000F031FC0099C0B251EA002000900621E6
S1138C50484600F028FC0099C0B20843009008215F
S1138C60484600F020FC000607000A21484600F0B0
S1138C701AFC57EA004007000C21484600F013FC98
S1138C8057EA002007000E21484600F00CFC384348
S1138C90070005E0A94881688B48FFF789F809E0D7
S1138CA03B00009A01990298F7F752FF0600300042
S1138CB0FFF7D6F8BDE8FF876CDF0000ECD30000B7
S1138CC0F4D8000010D9000080DF000030DD00007F
S1138CD06CE4000054E300002CD9000094DF000091
S1138CE074E4000060E300006CE30000F0B585B0BC
S1138CF004000D00002600200390002000900027AF
S1138D000020029000200190E4B2032C05D08C488E
S1138D1081686D48FFF74CF840E068680600310050
S1138D2003A800F055FB002805D1854881686648F2
S1138D30FFF73EF832E0A86806003100684600F00C
S1138D4047FB002805D17E4881685F48FFF730F86B
S1138D5024E00098042808D00098082805D0784812
S1138D6081685948FFF724F818E001AB02AA00997A
S1138D700398F7F744FF07003800FFF771F8002F56
S1138D800CD1029A02996F48FFF712F8009805284F
S1138D9004D3019A01996C48FFF70AF805B0F0BDB5
S1138DA030CA00001CCD00000CD4000048D90000DB
S1138DB07CE4000084E400008CE40000ACE10000EA
S1138DC048DD000064D90000BCE100002DE9F04357
S1138DD08BB004000D0000260020019003A8202180
S1138DE0F8F772FC002700200090002002905FF04A
S1138DF00008E4B2042C05D0544881683248FEF7D8
S1138E00D7FF5EE068680600310001A800F0E0FAD0
S1138E10002805D14D4881682B48FEF7C9FF50E072
S1138E20A86806003100684600F0D2FA002805D18F
S1138E30464881682448FEF7BBFF42E0E868060024
S1138E40310002A800F0C4FA002805D13F48816827
S1138E501D48FEF7ADFF34E00098002831D000989B
S1138E60212802D32020070001E000980700029B7C
S1138E703A0003A90198F7F70FFF80464046FEF732
S1138E80EFFFB8F1000F1CD10098C01B00900198AF
S1138E90381801905FF00009B945DDD2082099FB2C
S1138EA0F0F101FB1091002902D114A0FEF780FF1C
S1138EB003A819F800101848FEF77AFF19F1010900
S1138EC0EAE70BB0BDE8F08320D0000094E4000092
S1138ED044CD00006CCD000094CD0000E4CA000035
S1138EE0BCCD000010CB000060C700009CC7000090
S1138EF0E8C1000058C200009CE400000D0A2000F4
S1138F0060DD000068D00000E4CD000078DD0000E2
S1138F103C03FF1F5403FF1FA4E400006C03FF1F66
S1138F20ACE40000B4E40000BCE400008403FF1FD0
S1138F30CC03FF1FE403FF1FFC03FF1F1404FF1FE8
S1138F402C04FF1F2CD400004CD400004404FF1F49
S1138F500EB430B5040003A8050029002000F8F77A
S1138F604DFB30BC5DF810FB80B5DFF8F40300F076
S1138F7020F8DFF8F003FFF7EBFFDFF8EC03FFF76F
S1138F80E7FFDFF8E003FFF7E3FFDFF8E003FFF7B5
S1138F90DFFF01BD80B56846F8F7AAFD002803D0BD
S1138FA09DF8000000F019F801BDDFF8C403007853
S1138FB07047DFF8C0231268002A03D1DFF8B42316
S1138FC0106009E0DFF8AC23126811004A69002A36
S1138FD001D04969FAE74861704770B582B004006E
S1138FE0DFF89403DFF89413096840F2011202FBDE
S1138FF00105E4B20A2C02D0E4B20D2C37D1E4B25C
S1139000200000F0F4FA2878002804D028782028DA
S113901001D16D1CF7E7287800281FD0F9F7F2F882
S1139020280000F0CEF8F9F70AF9DFF850030068D9
S1139030401C1021B0FBF1F202FB1102DFF83C03EB
S113904002600020DFF8381308600020CA49CB4AC8
S1139050126840F2011303FB02110870C44800783F
S1139060002840F0AD80C148FFF772FFA8E0E4B2E9
S1139070082C02D0E4B27F2C11D1C148006800282A
S113908000F09E80BE480068401EBD490860002074
S1139090BB4909684855B0A0FFF75AFF90E0E4B215
S11390A01B2C79D16846002101608DF80040F8F747
S11390B031FD8DF80100F8F72DFD8DF802009DF8C3
S11390C0020041282FD1AD4800680F301021B0FBB9
S11390D0F1F606FB1106A848F6B240F2011101FBB5
S11390E00600007800286BD0A5480068411EA44AF9
S11390F01160002803D098A0FFF72AFFF4E79E48E8
S1139100F6B240F2011101FB060005002800FCF74D
S113911079FA9B490860F6B2984806602900994894
S1139120FFF716FF4CE09DF8020042282FD1934828
S11391300068401C1021B0FBF1F606FB11068E48B6
S1139140F6B240F2011101FB06000078002837D086
S11391508B480068411E8A4A1160002803D07EA013
S1139160FFF7F6FEF4E78448F6B240F2011101FB82
S1139170060005002800FCF745FA81490860F6B2AC
S11391807E48066029007F48FFF7E2FE18E0694642
S113919072A0FFF7DDFE13E079480068FF280FD8BE
S11391A0E4B2200000F023FA75480068445574487E
S11391B00068401C724908600020714909684855DC
S11391C073BD30B583B0040000946A480068019010
S11391D00025694601A800F01AF80500042D07D1FE
S11391E001980028F5D00099019800F04DF80DE0A1
S11391F0052D04D100996448FFF7AAFE06E0032D6B
S113920004D100996148FFF7A3FEFFE737BD2DE9BC
S1139210F04104000D00D5F80080002798F8000004
S1139220202802D118F10108F8E798F80000002876
S113923003D1C5F80080002024E020680600002E39
S11392401FD04146306800F0A9F80700012F16D15D
S113925098F80000002806D098F80000202802D0D2
S113926018F10108F4E798F80000202802D118F159
S11392700108F8E7C5F800802660042002E076695A
S1139280DDE70320BDE8F0812DE9F043D1B004000F
S11392900D0010A84FF48071F8F716FA10AE0027ED
S11392A02800FCF7AFF980460DF140094246290039
S11392B04846FEF73DF920686946FFB241F82700A9
S11392C07F1C307800281ED0FFB2102F1BDA3078B4
S11392D0202801D1761CFAE73078002813D068469C
S11392E0FFB240F827607F1C3078002804D0307823
S11392F0202801D0761CF7E73078002803D000201E
S11393003070761CDDE7E068002804D06946380038
S1139310C0B2E268904751B0BDE8F08370B5040074
S11393200D0000261A48FFF713FE124800680600D5
S1139330002E06D07268B1681648FFF709FE7669F8
S1139340F6E770BD38B504000D0001200849087027
S11393501148FFF7FDFD31BD08200800257300000A
S11393601C00FF1FB0C80000E0C80000C4E30000F8
S1139370D8C7FF1F1800FF1FA808FF1FBC18FF1F36
S1139380B818FF1FCCE300006CD100008CD10000A2
S113939000DA00001CE000007CE200000200087813
S11393A0002806D008781378984202D1491C521C30
S11393B0F5E70878202802D00878002806D110782C
S11393C0002801D1012002E0022000E003207047C0
S11393D010B40200002300240878002801D10020E2
S11393E03EE00878302805D14878782802D1012059
S11393F00300891C0878002830D0002B01D02401F8
S113940001E00A2044430878302806DB08783A282B
S113941003DA0878303804191EE0002B09D00878E4
S1139420612806DB0878672803DA087857380419B6
S113943012E0002B09D00878412806DB0878472879
S113944003DA08783738041906E00878002805D0CC
S113945000201060002003E0491CCBE714600120C9
S113946010BC70470100C9B2302906DBC9B23A29E1
S113947003DAB1F13000C0B214E0C9B2612906DBED
S1139480C9B2672903DAB1F15700C0B20AE0C9B220
S1139490412906DBC9B2472903DAB1F13700C0B26A
S11394A000E0002070472DE9F04104000D002E5D1E
S11394B0281947783000C0B2FFF7D4FF804638003F
S11394C0C0B2FFF7CFFF50EA0810C0B2BDE8F08188
S11394D080B500215FF48030085CC0B2532801D10C
S11394E0012045E000215FF48030085CC0B23A28D6
S11394F001D102203CE014215FF48030085CC0B24A
S1139500532816D115215FF48030085CC0B254286A
S11395100FD116215FF48030085CC0B24D2808D109
S113952017215FF48030085CC0B2502801D10020BC
S11395301EE000215FF48030085CC0B2FF2814D123
S113954001215FF48030085CC0B2FF280DD10221F4
S11395505FF48030085CC0B2FF2806D103215FF4B9
S11395608030085CC0B2FF2801D0032000E0042052
S113957002BD70B50400FFF7ABFF05000326EDB292
S1139580012D05D15FF4803000F046F8060016E0A6
S1139590EDB2022D05D15FF4803000F081FA0600AF
S11395A00DE0EDB2002D05D15FF4803000F0F0FC49
S11395B0060004E0EDB2032D01D1042006002000D2
S11395C0002802D03000C0B2A0473000C0B270BD45
S11395D0A0F16101062924BFA0F14101062904D3A9
S11395E030380A288041C00F70470120704710B5F9
S11395F0044614F1010F82B00AD08DF80000012254
S113960069460120F8F799FD012801D1204616BDCD
S11396104FF0FF3016BDFEE72DE9F041C0B0040065
S11396200025002668464FF48071F8F74DF80027AE
S11396305FF00108200000F080F90020DFF84814F2
S113964008600020DFF8441408600020DFF84014AC
S113965008600020DFF83C1408605FFA88F8B8F16D
S1139660060F2CD031002000085CC0B20500761C27
S1139670EDB20A2D1BD13900C9B2684600F023F8B7
S113968080465FFA88F8B8F1000F02D04046C0B2B5
S113969016E000200700DFF8000400F0C7F8804659
S11396A05FFA88F8B8F1010FD7D1012008E0EDB2D4
S11396B00D2DD2D06846FFB23D547F1CCDE700206B
S11396C040B0BDE8F0812DE9F24F82B004005FF0B4
S11396D000095FF0000ADFF8C0539DF808000A286B
S11396E001DA0220A0E02078532801D003209BE077
S11396F060783A2802DA6078302801DA042093E0AE
S113970060783038287002212000FFF7CCFE6870A2
S1139710687819EB00099DF8080069784900091D6B
S1139720884201D002207FE0002600272878002804
S11397300ED0012811D0022814D0032817D00528F0
S11397401AD007281BD008281CD009281DD01FE0D8
S113975002200600012007001CE002200600012070
S1139760070017E0032006000120070012E0042090
S11397700600012007000DE0022006000AE0042094
S1139780060007E00320060004E00220060001E0D2
S1139790042049E05FF0000800208246F6B2B2459A
S11397A00DD25FEA4A00011D2000FFF77CFEC0B223
S11397B050EA082859FA80F91AF1010AEEE7C5F8C7
S11397C00480FFB2002F1CD0F6B27000001D009080
S11397D06878F6B2801BB0F1010B00208246DA45AE
S11397E00DD2009810EB4A012000FFF75CFE1AEB43
S11397F00501487259FA80F91AF1010AEFE785F870
S113980008B07FEA09005FFA80F99DF80800811E1C
S11398102000FFF748FE85F8090195F80901814504
S113982001D0052000E00020BDE8FE8F2DE9F047BF
S113983004000025002600272078032805D020787E
S1139840022802D02078012801D10120050014F15A
S11398500900002804D0207A002801D0012600E065
S11398600026EDB2002D47D0F6B2002E44D0864833
S1139870006800281AD084480068217A4018B0F59E
S1139880804F04D860688249096888420ED07E48B7
S1139890026882497D480068F6F7BCFF0700002093
S11398A079490860012F01D1012044E0764800681D
S11398B0002806D1606875490860744800687449D6
S11398C0086094F8088014F1090974486E4909681D
S11398D011EB000A424649465046FDF729FE6A4804
S11398E00068217A40186849086069480068217A4C
S11398F04018674908601DE02078072805D02078C3
S1139900082802D02078092814D15F48006800286C
S113991010D05D48026861495C480068F6F77AFF38
S11399200700002058490860012F01D1012002E0FE
S1139930062000E00020BDE8F0872DE9F041C0B02A
S113994004000025002668464FF48071F7F7BCFE3A
S113995000275FF001085FFA88F8B8F1080F25D0F6
S113996031002000085CC0B20500761CEDB20A2D5F
S113997014D13900C9B26846FFF7A5FE80465FFAE4
S113998088F8B8F1000F02D04046C0B20FE00020C2
S11399900700414800F00EF88046DCE7EDB20D2DDB
S11399A0D9D06846FFB23D547F1CD4E7002040B0B4
S11399B0BDE8F08170B50400002500262078032856
S11399C005D02078022802D02078012801D1012076
S11399D0050014F10900002804D0207A002801D0E1
S11399E0012600E00026EDB2002D33D0F6B2002EA1
S11399F030D025480068002814D023480068217A14
S1139A004018B0F5804F04D860682149096888423D
S1139A1008D01D4801681D480068F6F754FE002070
S1139A201949086018480068002806D16068174979
S1139A300860164800681649086013480068217ACF
S1139A4040181149086012480068217A40181049EA
S1139A50086017E02078072805D02078082802D06D
S1139A60207809280ED10848006800280AD0064842
S1139A70016806480068F6F726FE002002490860DF
S1139A80082000E0002070BDF0C0FF1FF4C0FF1FDD
S1139A90F8C0FF1FFCC0FF1F84C4FF1FF080FF1F1E
S1139AA02DE9F041C0B004000025002668464FF4BB
S1139AB08071F7F709FE00275FF00108200000F02D
S1139AC07FF90020DFF8B01408600020DFF8AC1440
S1139AD008600020DFF8A81408600020DFF8A41450
S1139AE008605FFA88F8B8F1060F2CD03100200026
S1139AF0085CC0B20500761CEDB20A2D1BD13900FA
S1139B00C9B2684600F023F880465FFA88F8B8F1D5
S1139B10000F02D04046C0B216E000200700DFF874
S1139B20680400F083F880465FFA88F8B8F1010F02
S1139B30D7D1012008E0EDB20D2DD2D06846FFB296
S1139B403D547F1CCDE7002040B0BDE8F0812DE9F5
S1139B50F84304000D005FF000080026DFF82874C5
S1139B60EDB20B2D01DA02205EE020783A2801D014
S1139B70032059E001212000FFF795FC3870387864
S1139B8058FA80F8EDB2387840000B30854201D0A5
S1139B90022049E05FF0000900200600022E0BD2EB
S1139BA07000C11C2000FFF77EFCC0B250EA0929F6
S1139BB058FA80F8761CF1E7C7F8049007212000D2
S1139BC0FFF771FC3872387A18EB0008387A0028ED
S1139BD0052803D83878002802D112E0042023E0B5
S1139BE000200600387886420BD2700010F109017B
S1139BF02000FFF758FCF119487258FA80F8761CD7
S1139C00F0E77FEA0800401C5FFA80F8EDB2A91E75
S1139C102000FFF748FC87F8090197F809018045FF
S1139C2001D0052000E00020BDE8F2832DE9F84FC3
S1139C3004000025002600275FF000085FF00009FB
S1139C40207A002802D10120050016E0207A03289A
S1139C5002D0207A052802D1012006000DE0207AE6
S1139C60022802D0207A042802D10120070004E04F
S1139C70207A012801D1012080460020DFF8041356
S1139C800860EDB2002D4BD0BB48006800281FD0FF
S1139C90B9480068217850FA81F0B0F5804F04D8B3
S1139CA06068B7490968884212D0B3480268B74966
S1139CB0B2480068B34B1B681818F6F7ABFD814631
S1139CC00020AD490860B9F1010F01D1012075E010
S1139CD0A9480068002806D16068A8490860A74818
S1139CE00068A74908602078009014F1090AA74881
S1139CF0A149096811EB000B009A51465846FDF73B
S1139D0017FC9D480068217850FA81F09A49086050
S1139D109B480068217850FA81F0994908604CE02A
S1139D20FFB2002F2BD094480068002812D092482C
S1139D300268964991480068924B1B681818F6F718
S1139D4069FD814600208C490860B9F1010F01D1F9
S1139D50012033E0607AA17A51EA00208949086041
S1139D60207A022805D187480068000185490860E7
S1139D7023E0844800680004824908601DE0F6B2CC
S1139D80002E1AD15FFA88F8B8F1000F15D07A487E
S1139D900068002811D0784802687C497748006838
S1139DA0F6F738FD8146002073490860B9F1010FC8
S1139DB001D1012002E0062000E00020BDE8F28F7E
S1139DC02DE9F041C0B004000025002668464FF498
S1139DD08071F7F779FC00275FF001085FFA88F8D3
S1139DE0B8F1080F25D031002000085CC0B205008E
S1139DF0761CEDB20A2D14D13900C9B26846FFF7BA
S1139E00A6FE80465FFA88F8B8F1000F02D04046FB
S1139E10C0B20FE0002007005B4800F00EF8804657
S1139E20DCE7EDB20D2DD9D06846FFB23D547F1C5E
S1139E30D4E7002040B0BDE8F0812DE9F0410400F2
S1139E400025002600275FF00008207A002802D1B0
S1139E500120050016E0207A032802D0207A052884
S1139E6002D1012006000DE0207A022802D0207AD7
S1139E70042802D10120070004E0207A012801D13E
S1139E800120804600203F490860EDB2002D33D008
S1139E9039480068002815D037480068217850FAFE
S1139EA081F0B0F5804F04D860683549096888426C
S1139EB008D03148016831480068F6F704FC0020F6
S1139EC02D4908602C480068002806D160682B4999
S1139ED008602A4800682A490860274800682178F1
S1139EE050FA81F02449086025480068217850FA26
S1139EF081F0234908603BE0FFB2002F21D01E48C7
S1139F000068002808D01C4801681C480068F6F75F
S1139F10DAFB002018490860607AA17A51EA00202F
S1139F2018490860207A022805D116480068000103
S1139F30144908601CE013480068000411490860D3
S1139F4016E0F6B2002E13D15FFA88F8B8F1000FCC
S1139F500ED00948006800280AD00748016807485D
S1139F600068F6F7B0FB002003490860082000E011
S1139F700020BDE8F0810000F0C0FF1FF4C0FF1F07
S1139F80F8C0FF1FFCC0FF1F6CC3FF1FF080FF1F42
S1139F9038B50400200000F00CF8050029005FF437
S1139FA08030F6F7F8FB002801D0012000E0002003
S1139FB032BD38B5040000251F212000085CC0B262
S1139FC0000605001E212000085CC0B255EA0040CE
S1139FD005001D212000085CC0B255EA00200500E0
S1139FE01C212000085CC0B228430500280132BDB2
S1139FF0010000200200002A13D1DFF8DC064FF430
S113A000807303FB02000068002808D1DFF8C8064B
S113A0104FF4807303FB02000860002002E0521C2E
S113A020E9E7022070470100002008600020486032
S113A030002081F8FC00002081F8FB00002070471C
S113A04070B504000125002614F158000600002014
S113A050B0700020307300207073206B706194F82E
S113A0603400C0B2C00986F8290094F837000028EB
S113A07033D003282CD004283ED012281ED0152813
S113A08049D01A2842D01B2859D01D284DD01E284B
S113A0902DD0232844D0252833D0282813D02A288B
S113A0A020D02F2846D0552835D05A282ED09E2887
S113A0B027D0A82807D0AA2814D045E0200001F012
S113A0C013F8050056E0200001F03BF8050051E0CC
S113A0D0200000F0F3FF05004CE0200001F0D1F86F
S113A0E0050047E0200001F07CF8050042E0200074
S113A0F001F05AFA05003DE0200001F029FA0500BC
S113A10038E0200001F04CF9050033E0200001F0B4
S113A110E6F805002EE0200001F00DF9050029E025
S113A120200001F060F9050024E0200001F070FA3D
S113A13005001FE0200001F0BBF805001AE0200034
S113A14001F07DFA050015E0200001F0A4FA0500F5
S113A150002084F8EC00002084F8ED00002084F84E
S113A160EF00002084F8EE00002084F8F4000020C2
S113A17084F8F3002800C0B270BD2DE9F04387B025
S113A18004000D00160037005FF00109686810F143
S113A190010F1ED197F8ED00002817D078680068E9
S113A1A0002813D097F83700282803D097F83700F1
S113A1B0A8280BD100200490286805900020039063
S113A1C003AA012138007B681B6898474846C0B23F
S113A1D074E0F8686968884203D3F8686968401ACB
S113A1E0F86097F8F300012810D1002087F8F300F5
S113A1F0012087F8EE00002087F8ED0097F8F910A9
S113A2003868FDF7B2F84846C0B257E097F8ED0059
S113A210002804D168680D2801D12868804697F881
S113A220ED00002831D078680068002844D06868C0
S113A2300190286802903869009097F83700282820
S113A24003D097F83700A82805D16A4601213800C1
S113A2507B681B689847F868002807D038696968E4
S113A26008183861380000F0F4FC8146F8680028CA
S113A27022D1002087F8ED000D2317F1480297F84A
S113A280F9103868FCF7D0FF16E068680D2813D180
S113A290D8F80000DFF8441488420DD1012087F873
S113A2A0F0001F2317F1280297F8FA103868FCF71A
S113A2B0CBFF012087F8F5004846C0B207B0BDE8DF
S113A2C0F0832DE9F04186B004000D00160037003C
S113A2D05FF00008686810F1010F1ED197F8ED00D7
S113A2E0002817D078680068002813D097F8370042
S113A2F02A2803D097F83700AA280BD1002004900D
S113A300286805900020039003AA022138007B6886
S113A3101B6898474046C0B213E1F86869688842F0
S113A32003D3F8686968401AF86097F8F4000128C4
S113A33013D1002087F8F400012087F8EF000020F3
S113A34087F8EC00002087F8F50097F8FA103868D1
S113A350FDF70BF84046C0B2F3E097F8EC00002894
S113A36035D0686801902868029038690090786850
S113A3700068002818D097F837002A2803D097F8E7
S113A3803700AA2805D16A46022138007B681B6879
S113A3909847F868002807D0386969680818386150
S113A3A0380000F099FC8046F868002840F0C78027
S113A3B0002087F8EC000D2317F1480297F8F910F4
S113A3C03868FCF731FF012087F8F600B7E097F80A
S113A3D0F000002800F09A8068681F2840F09680FA
S113A3E0B86ABF49884240F0918097F83500F0215F
S113A3F0084240F08B8097F83600E021084240F094
S113A400858097F8350097F8F810491C88427DDA62
S113A41097F83600002879D097F83600112875DAB5
S113A420002087F8F5000020F860AC48B8640020EC
S113A4303865F86AF864002087F8F000386B3863F0
S113A44097F83400000604D4386B002801D00120AA
S113A45000E0002087F8EC0097F83400000604D5EB
S113A460386B002801D0012000E0002087F8ED00BF
S113A47097F8ED00002808D097F8EE00002804D0E3
S113A480012080464046C0B25BE03800FFF7D8FDAB
S113A49080465FFA88F8B8F1050F1FD197F8EC00F1
S113A4A001280AD197F8EF00002802D1012087F88B
S113A4B0F400002087F8EC000DE097F8ED00012887
S113A4C009D197F8EE00002802D1012087F8F300A3
S113A4D0002087F8ED00022087F8F70097F8EC00D9
S113A4E000282CD197F8ED00002828D197F8F30024
S113A4F0002824D10D2317F1480297F8F910386881
S113A500FCF792FE012087F8F60018E097F8FA109D
S113A5103868FCF72AFF97F8F9103868FCF725FF2C
S113A520002087F8F000012087F8EF00012087F869
S113A530EE00012087F8F700012087F8F10040467B
S113A540C0B206B0BDE8F0812DE9FF410400002649
S113A550012760688068407994F8FC10884202D230
S113A5603800C0B2B4E0606880680068002802D196
S113A5703800C0B2ACE060688068006894F8FC10F1
S113A58010EBC100083805000020297888422EDA33
S113A59069680C2202FB00110978082925D10021E1
S113A5A06A680C2303FB0022127A914215DA6A6866
S113A5B00C2303FB002252680B019A5C94F8FB30D5
S113A5C09A4208D16A680C2303FB0022526812EBFA
S113A5D001110E0001E0491CE2E769680C2202FB4C
S113A5E00010C07884F8FD0001E0401CCDE7002E87
S113A5F002D13800C0B26BE0A6605FF00008307989
S113A60080452FDA00208DF80400B06810F8280087
S113A6108DF80200B06810EB88004088ADF80000A7
S113A620B06810EB880040788DF803009DF80200B4
S113A630C009012806D19DF8020084F8F9002948D0
S113A640029005E09DF8020084F8FA002648029082
S113A650039402AA69462068FCF71CFE070018F15F
S113A6600108CCE7002084F8EC00002084F8ED0019
S113A670002084F8EF00002084F8EE00002084F825
S113A680F400002084F8F300012084F8F000002096
S113A690E060002084F8F100002084F8F20000203B
S113A6A084F8F70094F8F500012804D194F8FA101E
S113A6B02068FCF7D6FD1F2314F1280294F8FA1041
S113A6C02068FCF7C1FD012084F8F5003800C0B211
S113A6D004B0BDE8F0810000D8C6FF1F55534253B3
S113A6E0555342437BA10000C3A2000070B504008F
S113A6F00125A068002802D12800C0B210E000267D
S113A700A0680079864209DAA068806810F82610EB
S113A7102068FCF7FAFD0500761CF1E72800C0B2BA
S113A72070BD2DE9F04387B004000D0016005FF002
S113A730010900275FF000086846FFF759FC8146CD
S113A7405FFA89F9B9F1000F02D04846C0B2D2E0ED
S113A75000992000C0B2FCF760FA81465FFA89F9DB
S113A760B9F1000F05D00098FFF75DFC4846C0B270
S113A770C1E000980068002804D10098FFF753FC5A
S113A7800320B8E0009845600020009981F8FC009F
S113A790FF20009981F8FB0001AA05210098009B85
S113A7A05B681B68984781460298002804D001988A
S113A7B0002801D0012000E00020C0B2002807D109
S113A7C0012081460098FFF72EFC4846C0B292E073
S113A7D09DF81400009981F8F800009858308046DC
S113A7E00198009948610298009988619DF81400C5
S113A7F0401E009981F8F8000398009908620498B3
S113A800009948620098C761702088F800000A2007
S113A81088F80700002088F80200002088F80C005F
S113A820002088F80D0000984069401E009949698D
S113A830491E11F47F41090251EA006000994969F7
S113A840491E090A11F47F41084300994969491EC8
S113A85050EA1160C8F82C00009880690099896951
S113A86011F47F41090251EA006000998969090ADB
S113A87011F47F4108430099896950EA1160C8F8CE
S113A880300000984069401E00994969491E11F43E
S113A8907F41090251EA006000994969491E090A89
S113A8A011F47F41084300994969491E50EA116037
S113A8B0C8F83800009880690099896911F47F41CB
S113A8C0090251EA006000998969090A11F47F417B
S113A8D008430099896950EA1160C8F83C000020D7
S113A8E0009981F8F5000020009981F8F60000989D
S113A8F030604846C0B207B0BDE8F08370B50400CC
S113A90001262500002D01D1032008E02800FFF7CF
S113A910EDFE06002800FFF786FB3000C0B270BDD4
S113A9202DE9F84F04000D0016000127002E01D078
S113A930002C01D103208AE1A046012D00F01D81E5
S113A940C0F08381032D0BD006D3052D50D028D31E
S113A950062D00F0878078E1002088F8FC0074E17F
S113A960B246D8F80400002800F06F819AF800007D
S113A97098F8FC10884200F0688198F8FC000028E0
S113A98003D04046FFF7B2FE07009AF8000088F8AB
S113A990FC00002088F8FB004046FFF7D5FD0700C7
S113A9A053E1D8F80400002800F04F813088814634
S113A9B048468DF8000098F8FD10484680B2000A19
S113A9C0C0B2814240F041819DF8000098F8FB102C
S113A9D0884200F03A814046FFF788FE07009DF860
S113A9E0000088F8FB004046FFF7AEFD07002CE1AD
S113A9F0D8F80400002803D0D8F80800002800D1B3
S113AA0023E1B2465FF0000BD8F8080000798345D3
S113AA1027DA9AF80000D8F80810896811F82B1082
S113AA2088421BD198F8EE00002809D19AF800104A
S113AA30D8F80000FCF799FC0700012088F8EE0024
S113AA4098F8EF00002809D19AF80010D8F800000F
S113AA50FCF78BFC0700002088F8EE001BF1010BCB
S113AA60D2E7F2E0D8F80400002807D0D8F80800AC
S113AA70002803D098F8F100012800D1E5E0B2469F
S113AA805FF0000BD8F808000079834527DA9AF8BC
S113AA900000D8F80810896811F82B1088421BD1DF
S113AAA098F8EE00012809D19AF80010D8F80000AF
S113AAB0FCF76BFC0700002088F8EE0098F8EF0024
S113AAC0012809D19AF80010D8F80000FCF75DFCC1
S113AAD00700002088F8EE001BF1010BD2E798F87C
S113AAE0F700032803D098F8F70002281CD198F83F
S113AAF0F200012818D098F8F600012805D198F83A
S113AB00F910D8F80000FCF7ACFB0D2318F148024B
S113AB1098F8F910D8F80000FCF786FB002088F8B4
S113AB20F600002088F8F70098F8F200012823D1F5
S113AB3098F8EE0000281FD198F8EF0000281BD1E8
S113AB40002088F8F20098F8F600012805D198F85A
S113AB50F910D8F80000FCF784FB1F2318F1280231
S113AB6098F8FA10D8F80000FCF76EFB002088F87B
S113AB70F600002088F8F70067E0002E64D0B346A2
S113AB80DBF80000007810F01F0001285DD1DBF82D
S113AB9000000079C0B298F8FD10884255D1DBF866
S113ABA000004078FE2802D0FF2824D04CE0DBF8D7
S113ABB00000808898F8FD1089B2884218D1DBF82B
S113ABC000004088002813D1DBF80000C088022868
S113ABD00EDADBF800000078000609D518F1F80059
S113ABE0CBF80400DBF80000C088CBF8080001E0D3
S113ABF00520070028E0DBF80000808898F8FD10A5
S113AC0089B288421DD1DBF800004088002818D1A1
S113AC10DBF80000C088002813D1DBF800000078BE
S113AC2000060ED44046FFF761FD07004046FFF7DB
S113AC308BFC0700002088F8F100012088F8F2005E
S113AC4001E005200700FFE7FFE73800C0B2BDE8D8
S113AC50F28F3EB50400002520690090206AB0F10F
S113AC60011F03D35FF48030019001E0206A01905A
S113AC700198E168884202D20198019001E0E068FD
S113AC800190002002906A460421200063681B683A
S113AC90984720696169A2695143884208D2019B9F
S113ACA0029A94F8F9102068FCF7BEFA050010E047
S113ACB0002084F8F300012084F8EE00002084F8DA
S113ACC0ED00022084F8F70094F8F9102068FCF7EE
S113ACD04CFB2800C0B23EBD3EB5040000252069EF
S113ACE00090606AB0F1011F03D35FF480300190DB
S113ACF001E0606A01900198E168884202D20198FB
S113AD00019001E0E0680190002002906A4603216E
S113AD10200063681B68984720696169A2695143F0
S113AD20884208D2019B029A94F8FA102068FCF732
S113AD308BFA050010E0002084F8F400012084F868
S113AD40EF00002084F8EC00022084F8F70094F867
S113AD50FA102068FCF709FB2800C0B23EBDF8B524
S113AD6004000D00160000277068A1694843E060E4
S113AD703068A16948432061EDB2012D04D120005F
S113AD80FFF767FF070003E02000FFF7A5FF0700B8
S113AD903800C0B2F2BDFEE7F8B50400002514F196
S113ADA06C00070014F158000600386800280CD124
S113ADB0002020657868002803D1002084F854001E
S113ADC079E1022084F8540075E1787D002800F0D0
S113ADD0C280786800281CD138687968401A2065D8
S113ADE07B68BA6894F8F9102068FCF71DFA05002E
S113ADF0EDB2002D03D1002084F8540006E00120B8
S113AE0084F854000320B07011203073052005002D
S113AE1051E1B87D002800F08E8078683968884256
S113AE2028D238687968401A206596F828000128E5
S113AE3007D117F10C0201212000FFF790FF050054
S113AE4007E07B68BA6894F8F9102068FCF7ECF91D
S113AE500500EDB2002D03D1002084F8540006E073
S113AE60012084F854000320B070112030730520B1
S113AE70050020E138687968884224D100202065E3
S113AE8096F82800012807D117F10C0201212000AF
S113AE90FFF765FF050007E07B68BA6894F8F910CE
S113AEA02068FCF7C1F90500EDB2002D03D10020A4
S113AEB084F85400FFE0012084F854000320B070AB
S113AEC011203073F7E00020206596F8280001284F
S113AED012D13868A169B0FBF1F03861386839697A
S113AEE0A26902FB1100206517F10C020121200068
S113AEF0FFF735FF050007E03B68BA6894F8F910DE
S113AF002068FCF791F90500EDB2002D0BD196F8FD
S113AF102800012803D1022084F85400CBE000204B
S113AF2084F85400C7E0012084F854000320B07072
S113AF3011203073BFE0386820650023BA6894F8A4
S113AF40F9102068FCF770F90500022084F8540019
S113AF5005200500AFE0786800280FD194F8FA10B6
S113AF602068FCF702FA38682065012084F8540050
S113AF70012084F8EF00052005009CE0B87D00283E
S113AF800FD094F8FA102068FCF7EFF938682065C0
S113AF90022084F85400012084F8EF000520050005
S113AFA089E078683968884228D238687968401A14
S113AFB0206596F82800012807D117F10C0200211A
S113AFC02000FFF7CCFE050007E07B68BA6894F820
S113AFD0FA102068FCF738F90500EDB2002D03D112
S113AFE0002084F8540006E0012084F85400032073
S113AFF0B07003203073052005005CE03868796880
S113B000884224D10020206596F82800012807D121
S113B01017F10C0200212000FFF7A1FE050007E054
S113B0207B68BA6894F8FA102068FCF70DF90500FB
S113B030EDB2002D03D1002084F854003BE0012040
S113B04084F854000320B0700320307333E00020F0
S113B050206596F82800012812D13868A169B0FB50
S113B060F1F0386138683969A26902FB1100206582
S113B07017F10C0200212000FFF771FE050007E024
S113B0803B68BA6894F8FA102068FCF7DDF805000C
S113B090EDB2002D0BD196F82800012803D102202F
S113B0A084F8540007E0002084F8540003E00320EF
S113B0B0B070032030732800C0B2F2BD70B5040034
S113B0C0002514F1580005001220A861012085F81C
S113B0D02A00ED61002085F828002000FFF75CFEBF
S113B0E006003000C0B270BD2DE9F0470400002511
S113B0F014F158000500DFF84C048046C14615F1F0
S113B100400A00200700FFB2242F07D2FFB217F82D
S113B1100900FFB207F80A007F1CF4E72420A861A5
S113B120012085F82A0015F14000E861002085F827
S113B13028002000FFF730FE06003000C0B2BDE852
S113B140F0872DE9F041040000255FF00008002796
S113B15014F15800050094F839000006804694F86C
S113B1603A0058EA004894F83B0058EA002894F85A
S113B1703C0050EA080894F83700282808D194F8CD
S113B1803E00000280B2070094F83F00074312E03B
S113B19094F83700A8280ED194F83D000006070063
S113B1A094F83E0057EA004794F83F0057EA002716
S113B1B094F840000743012085F82A00A0697843E9
S113B1C0A8610020E861012085F82800C5F82080E6
S113B1D06F622000FFF7E0FD06003000C0B2BDE85A
S113B1E0F0812DE9F041040000255FF000080027FC
S113B1F014F15800050094F839000006804694F8CC
S113B2003A0058EA004894F83B0058EA002894F8B9
S113B2103C0050EA080894F837002A2808D194F82A
S113B2203E00000280B2070094F83F00074312E09A
S113B23094F83700AA280ED194F83D0000060700C0
S113B24094F83E0057EA004794F83F0057EA002775
S113B25094F840000743002085F82A00A069784349
S113B260A8610020E861012085F82800C5F8208045
S113B2706F622000FFF790FD06003000C0B2BDE809
S113B280F08170B50400002514F158000500002079
S113B290A861012085F82A000020E861002085F8D3
S113B2A028002000FFF778FD06003000C0B270BD12
S113B2B070B50400002514F1580005000020A861B1
S113B2C0012085F82A000020E861002085F8280084
S113B2D02000FFF761FD06003000C0B270BD2DE90B
S113B2E0F0470400002514F15800050096488046F4
S113B2F0C14615F1640A00200700FFB2082F07D2E7
S113B300FFB217F80900FFB207F80A007F1CF4E740
S113B3100820A861012085F82A0015F16400E8617D
S113B320002085F828002000FFF736FD06003000D5
S113B330C0B2BDE8F0872DE9F047040000250B26D4
S113B34014F15800050080488046C14615F1640A8E
S113B35000200700FFB2082F07D2FFB217F8090038
S113B360FFB207F80A007F1CF4E70820A861012057
S113B37085F82A0015F16400E861002085F82800AA
S113B3802000FFF709FD060094F83800C00703D534
S113B3900520A870242028733000C0B2BDE8F087CF
S113B3A070B5040000250B2614F15800050094F82C
S113B3B03700252805D10820A86115F12C00E86183
S113B3C004E00C20A86115F13400E861012085F83F
S113B3D02A00002085F828002000FFF7DDFC060085
S113B3E03000C0B270BD2DE9F04F87B004000025D5
S113B3F00B208DF802005548006802905FF0000AA7
S113B4005FF0000B5FF0000914F15800050094F898
S113B4103F00ADF8000095F86C00002806D0E06904
S113B420002801D0022702E0032700E0002760691A
S113B4300390A069049095F86C00002802D05FF096
S113B440020801E05FF00108FFB2F8008DF80B007C
S113B45060690590A0690690FFB2F8000C30019075
S113B460BDF800000199884202D2BDF800000190A5
S113B47002A80600002082465FFA8AFABAF1040F95
S113B4800ED25FFA8BFB1BF806005FFA8AFA1AEBFE
S113B490050181F86D001BF1010B1AF1010AEBE7BC
S113B4A005A80600002083465FFA8BFBBBF1080F5A
S113B4B00ED25FFA8BFB1BF806005FFA8AFA1AEBCE
S113B4C0050181F86D001BF1010B1AF1010AEBE78C
S113B4D095F86C0000281FD0002083465FFA8BFB90
S113B4E0FFB2BB4518D203A806005FFA8AFABAF184
S113B4F0080F0ED25FFA89F919F806005FFA8AFA82
S113B5001AEB050181F86D0019F101091AF1010A1C
S113B510EBE71BF1010BE1E70198A861012085F835
S113B5202A0015F16D00E861002085F8280020004C
S113B530FFF732FC8DF802009DF8020007B0BDE869
S113B540F08F0000B0D00000F4E40000D0E600006A
S113B55070B50400002514F1580005000020A8610E
S113B560012085F82A000020E861002085F82800E1
S113B5702000FFF711FC060094F85400022810D0B4
S113B58094F8380010F01F00172803D1002084F825
S113B590540006E0012084F854000520A8702420FB
S113B5A028733000C0B270BDF8B50400002514F152
S113B5B05800050094F83B0010F00100070000203B
S113B5C0A861012085F82A000020E861002085F8A0
S113B5D028002000FFF7E0FB060094F8540002283E
S113B5E009D0FFB2002F06D0012084F854000520B2
S113B5F0A8702420287360680068002805D0002201
S113B6000721200063681B6898473000C0B2F2BD70
S113B61070B50400002514F1580005000020A8614D
S113B620012085F82A000020E861002085F8280020
S113B6302000FFF7B1FB06003000C0B270BD70B54A
S113B64082B00400002514F15800050094F83B0072
S113B65010F003008DF800000020A861012085F897
S113B6602A000020E861002085F828002000FFF768
S113B67093FB060094F85400022809D0606800681F
S113B680002805D06A460821200063681B68984793
S113B6903000C0B276BD0100002211F15800020052
S113B6A000200865012081F85400052090702020B6
S113B6B010730020507300207047FEE70EB430B5BD
S113B6C0040003A8050029002000F5F797FF30BC0B
S113B6D05DF810FB416070478160704780B5F6F7F4
S113B6E046F8FCF771FB00F06FF8FDF75EFC0028EC
S113B6F042D1FDF74FFC82480068012804D1102193
S113B7008048FFF7E9FFF0E77D4800680228ECD1A4
S113B710F6F778FD7C480068012804D164210120F3
S113B720F5F781FD1AE078480068022804D1642105
S113B7300220F5F778FD11E073480068032805D16D
S113B7404FF461410320F5F76EFD07E06E48006891
S113B750042803D17D210420F5F765FD0FF21D00B7
S113B760FDF707FFF6F76BFD10216648FFF7B2FF00
S113B770002063490860B8E701BD000010B504006B
S113B780E4B2002C07D020215E48FFF7A5FF5F48F4
S113B790FFF794FF17E010215A48FFF79BFF5FF073
S113B7A080515B48FFF796FF5FF000515848FFF760
S113B7B091FF20215348FFF78DFF01205249086073
S113B7C05448FFF77BFF10BD80B55348FDF7F1FBEC
S113B7D05248FDF7EEFB5248FDF7EBFB5148FDF7ED
S113B7E0E8FB5148FDF7E5FB5048FDF7E2FB504804
S113B7F0FDF7DFFB4F48FDF7DCFB4F48FDF7D9FBB6
S113B8004E48FDF7D6FB4E48FDF7D3FB4D48FDF7F8
S113B810D0FB4D48FDF7CDFB01BD10B53C48F9F711
S113B820DFFF04004FF480613948F9F7E7FF102186
S113B8303748F9F7E3FFE0060CD531480068401CAF
S113B8402F4908602E480068032857D300202C494C
S113B850086053E0600551D529480068002846D1A6
S113B86029480068401C28490860274800680528C2
S113B87002D301202449086023480068012809D123
S113B8805FF080512248FFF725FF5FF00051204808
S113B890FFF720FF1C48006802280AD15FF080519E
S113B8A01B48FFF719FF5FF000511948FFF712FF1B
S113B8B024E01548006803280AD15FF08051144839
S113B8C0FFF708FF5FF000511148FFF705FF15E08F
S113B8D00D480068042811D15FF080510C48FFF72F
S113B8E0FBFE5FF000510A48FFF7F6FE06E0002079
S113B8F00349086010210348FFF7ECFE10BD000067
S113B90078C4FF1F40F00F408404FF1FB8D9000023
S113B91000F00F408CD400002403FF1F3C03FF1FE2
S113B9205403FF1F6C03FF1F8403FF1FB403FF1F97
S113B9309C03FF1FCC03FF1FE403FF1FFC03FF1F37
S113B9401404FF1F2C04FF1F4404FF1F816807E039
S113B95002681168536889185B18C3600832026072
S113B960C2689142F4D04A1C82600878704738B5A6
S113B97004460D46A068E168884212D120686168D7
S113B980884208BFF9F76CFE2068227C016802B186
S113B9904944A16042685218E26008309142206034
S113B9A0ECD0A068401CA06000F8015D31BD2DE919
S113B9B0F0418AB000F1080100910268520801EBDD
S113B9C0C20101910021029103910168490800EB31
S113B9D0C10108310491017901F001018DF82010B1
S113B9E040680499400801EBC000059000200690CF
S113B9F0079084E06846FFF7A9FF044614F00306A5
S113BA0003D16846FFF7A2FFC61C25090F2D1BD1E1
S113BA106846FFF79BFF00F10F0515E000980168E9
S113BA200818009902904968081803900098083093
S113BA300090029803998842F0D0401C029010F8BC
S113BA40011D04A8FFF793FF761EF2D1002D51D0FB
S113BA506846FFF77BFF0646A00800F003000328B2
S113BA6004BF6846FFF772FFDDF810800699079F50
S113BA7006EB002008E0A8F10808A8F10801801AE4
S113BA800A6849688F18394658F8082C8A1A82427D
S113BA90F1D30C1AAE1C2DD0BC4206D158F8044B7D
S113BAA058F8040B0719BC42F8D00698079914F803
S113BAB0015B884217D104980599884208BFF9F7B9
S113BAC0CFFD049800689DF82010069009B1484401
S113BAD00690049906984968049A0918083288421D
S113BAE007910492E7D00698401C0690761E00F851
S113BAF0015DD1D10298039988427FF47BAF00980D
S113BB00019988427FF476AF05980AB0BDE8F081C8
S113BB1046534C204C6F616465722008000000009D
S113BB2000000000000000602C4200000000000043
S113BB30412E0066007300650076000F00DA650090
S113BB406E0074007300640000000000FFFFFFFF3C
S113BB5046534556454E7E31202020120000006099
S113BB602C422C42000000602C4202000000000025
S113BB7042650072005F0069006E000F00A8640057
S113BB80650078000000FFFFFFFF0000FFFFFFFFDC
S113BB90012E006D006500740061000F00A86400B0
S113BBA06100740061005F006E00000065007600B3
S113BBB04D45544144417E31202020220000006044
S113BBC02C422C42000000602C42000000000000C7
S113BBD0412E0054007200610073000F00256800BC
S113BBE0650073000000FFFFFFFF0000FFFFFFFF81
S113BBF05452415348457E312020202200000060E9
S113BC002C422C42000000602C4200000000000086
S113BC1042200049006E0066006F000F007272003F
S113BC206D006100740069006F0000006E00000088
S113BC3001530079007300740065000F00726D00F9
S113BC40200056006F006C00750000006D00650058
S113BC5053595354454D7E31202020160000006076
S113BC602C422C42000000602C4203000000000023
S113BC70494E464F202020205458540100000060B3
S113BC802C422C42000000602C4205000100000000
S113BC90535441545553202054585401000000601B
S113BCA02C422C42000000602C42060001000000DF
S113BCB0456D62656464656420486F737420256310
S113BCC025642E25642E25640D0A0D0A486F7374AD
S113BCD020426F6172643A2025730D0A4350552047
S113BCE0636C6F636B3A202575204D487A0D0A46C4
S113BCF06C6173682073697A653A202575206279CE
S113BD007465730D0A466C6173682072616E6765B1
S113BD103A2025732D25730D0A52414D2073697AFB
S113BD20653A2025752062797465730D0A52414D78
S113BD302072616E67653A2025732D25730D0A50B4
S113BD4065726970686572616C20737570706F726A
S113BD507465643A2025730D0A000000433A5C556B
S113BD60736572735C4232313731305C446F637592
S113BD706D656E74735C53746173685C6D63752D6B
S113BD80626F6F742D6D61737465725C322E302E28
S113BD90305F72656C656173652E6275696C645C95
S113BDA04B696E657469735F426F6F746C6F616425
S113BDB065725C76616C69646174696F6E5C656DF3
S113BDC06265646465645F686F73745C4D4B36359B
S113BDD04631385C2E2E5C2E2E5C2E2E5C737263E4
S113BDE05C647269766572735C706F72742F6673CB
S113BDF06C5F706F72742E68000000002E2020208B
S113BE002020202020202032000000602C422C42E0
S113BE10000000602C420300000000002E2E2020B1
S113BE202020202020202010000000602C422C42E2
S113BE30000000602C420000000000004247007532
S113BE40006900640000000F00FFFFFFFFFFFFFF19
S113BE50FFFFFFFFFFFF0000000000000149006E2C
S113BE60006400650078000F00FF65007200560052
S113BE706F006C00750000006D006500494E44457C
S113BE8058457E3120202020000000602C422C42A6
S113BE90000000602C4204004D0000001400160055
S113BEA018001A001C001E00220028001C0020009C
S113BEB0240028002C0030003800440030003800F2
S113BEC040004800500058006800800050006000A6
S113BED0700080009000A000C000F000A000C0002E
S113BEE0E0000001200140018001E00140018001E7
S113BEF0C0010002400280020003C003800200036C
S113BF008003000480040005000680070005000685
S113BF10000700080009000A000C000F433A5C55B2
S113BF20736572735C4232313731305C446F6375D0
S113BF306D656E74735C53746173685C6D63752DA9
S113BF40626F6F742D6D61737465725C322E302E66
S113BF50305F72656C656173652E6275696C645CD3
S113BF604B696E657469735F426F6F746C6F616463
S113BF7065725C7372635C7574696C69746965730A
S113BF805C7372635C66736C5F72746F735F61621F
S113BF90737472616374696F6E2E6300433A5C5507
S113BFA0736572735C4232313731305C446F637550
S113BFB06D656E74735C53746173685C6D63752D29
S113BFC0626F6F742D6D61737465725C322E302EE6
S113BFD0305F72656C656173652E6275696C645C53
S113BFE04B696E657469735F426F6F746C6F6164E3
S113BFF065725C7372635C647269766572735C66A5
S113C0006C657863616E5C66736C5F666C6578639F
S113C010616E2E6300000000433A5C5573657273D1
S113C0205C4232313731305C446F63756D656E74D8
S113C030735C53746173685C6D63752D626F6F74A8
S113C0402D6D61737465725C322E302E305F7265B3
S113C0506C656173652E6275696C645C4B696E65B1
S113C0607469735F426F6F746C6F616465725C7343
S113C07072635C647269766572735C647370695C24
S113C08066736C5F647370692E630000433A5C5599
S113C090736572735C4232313731305C446F63755F
S113C0A06D656E74735C53746173685C6D63752D38
S113C0B0626F6F742D6D61737465725C322E302EF5
S113C0C0305F72656C656173652E6275696C645C62
S113C0D04B696E657469735F426F6F746C6F6164F2
S113C0E065725C7372635C647269766572735C67B3
S113C0F070696F5C66736C5F6770696F2E630000B4
S113C100433A5C55736572735C4232313731305C4B
S113C110446F63756D656E74735C53746173685CAE
S113C1206D63752D626F6F742D6D61737465725CD0
S113C130322E302E305F72656C656173652E6275C8
S113C140696C645C4B696E657469735F426F6F748C
S113C1506C6F616465725C7372635C64726976654A
S113C16072735C6932635C66736C5F6932632E63FD
S113C17000000000433A5C55736572735C423231CF
S113C1803731305C446F63756D656E74735C5374E2
S113C1906173685C6D63752D626F6F742D6D61736F
S113C1A07465725C322E302E305F72656C6561731B
S113C1B0652E6275696C645C4B696E657469735F46
S113C1C0426F6F746C6F616465725C7372635C64FC
S113C1D07269766572735C756172745C66736C5FA8
S113C1E0756172742E6300000D0A20506C656173D2
S113C1F06520696E70757420726967687420747242
S113C200616E73666572206672657175656E6379B9
S113C210203A202D665B3130307E313030305D2065
S113C2206F7220626175642072617465203A202DFA
S113C230665B31393230302F33383430302F353774
S113C2403630302F3131353230302F3233303430D4
S113C250305D2E20000000000D0A20506C656173D3
S113C2606520696E707574207472616E7366657290
S113C270206672657175656E637920616674657296
S113C280202D66203A202D665B3130307E313030EF
S113C290305D206F72206261756420726174652064
S113C2A03A202D665B31393230302F333834303018
S113C2B02F35373630302F3131353230302F32335D
S113C2C0303430305D2E2000433A5C557365727310
S113C2D05C4232313731305C446F63756D656E7426
S113C2E0735C53746173685C6D63752D626F6F74F6
S113C2F02D6D61737465725C322E302E305F726501
S113C3006C656173652E6275696C645C4B696E65FE
S113C3107469735F426F6F746C6F616465725C7390
S113C32072635C6372635C7372635C637263313601
S113C3302E63000028636F6E6669672D3E6D617819
S113C3404D624E756D203E2030292026262028631C
S113C3506F6E6669672D3E6D61784D624E756D2016
S113C3603C3D2046534C5F464541545552455F463B
S113C3704C455843414E5F4841535F4D45535341EB
S113C38047455F4255464645525F4D41585F4E55BD
S113C3904D4245526E2862617365292900000000F0
S113C3A02E20202020202020202020320000006089
S113C3B02C422C42000000602C42020000000000CD
S113C3C02E2E20202020202020202010000000607D
S113C3D02C422C42000000602C42000000000000AF
S113C3E04E4F5F4C4F472020202020200800006043
S113C3F02C422C42000000602C420000000000008F
S113C4002CE1000090DE000018E300003CE1000095
S113C41024E3000060DA00004CE100005CE100006D
S113C42044E400004CE4000054E400006CE100002B
S113C4303CD50000A4DE00007CE10000B8DE000072
S113C440CCDE00008CE1000030E3000098E6000040
S113C4509CE60000A0E60000CCE10000A8DF00009C
S113C46078E30000DCE1000084E3000090DD0000DC
S113C470ECE10000FCE10000C4E40000CCE40000B6
S113C480D4E400000CE2000080D90000BCDF00000E
S113C4901CE20000D0DF0000E4DF00002CE200001A
S113C4A090E30000C0E60000C4E60000C8E6000017
S113C4B00000000010C80000360000000100000069
S113C4C06CE200000E0000001100000010BB000030
S113C4D0A001000013000000A0C3000060000000E1
S113C4E014000000FCBD0000A000000015000000C6
S113C4F004C500004D000000000000000000000022
S113C500000000007B0033003700320030003300AD
S113C5104200460038002D00460044003800330035
S113C5202D0034003300320031002D00410034006E
S113C530430034002D00390041003900410042001D
S113C54046003800460042004300460044007D0097
S113C550000000000D0A204572726F723A20496E85
S113C560697469616C2070696E67206661696C75B5
S113C57072653A204E6F20726573706F6E7365201A
S113C580726563656976656420666F722070696E92
S113C5906720636F6D6D616E640000006D624964B5
S113C5A078203C2046534C5F464541545552455FE4
S113C5B0464C455843414E5F4841535F4D455353A4
S113C5C04147455F4255464645525F4D41585F4E8F
S113C5D0554D4245526E2862617365290000000082
S113C5E00200000004000000060000000800000033
S113C5F01000000020000000400000008000000047
S113C6000001000000020000000400000008000017
S113C6100010000000200000004000000080000026
S113C62002000000040000000800000010000000E8
S113C6302000000040000000800000000001000015
S113C64000020000000400000008000000100000C8
S113C65000200000004000000080000000000100F5
S113C66046534C5F464541545552455F55415254DB
S113C6705F4649464F5F53495A456E286261736568
S113C68029203E3D20636F6E6669672D3E747846AF
S113C69069666F57617465726D61726B00000000AA
S113C6A046534C5F464541545552455F554152549B
S113C6B05F4649464F5F53495A456E286261736528
S113C6C029203E3D20636F6E6669672D3E72784671
S113C6D069666F57617465726D61726B000000006A
S113C6E066696C6C2D6D656D6F7279203C61646454
S113C6F0723E203C627974655F636F756E743E2090
S113C7003C7061747465726E3E205B776F72642056
S113C7107C2073686F7274207C20627974655D007C
S113C72019E050F8041BCB0744BFA9F101035918C1
S113C730121F0023042A41F8043BF9D25FEA827CE9
S113C7400B4604D54FF0000CA1F800C09B1CD10788
S113C75044BF0021197050F8042B002AE1D170471E
S113C7600D0A20506C6561736520696E70757420C4
S113C7707269676874207472616E73666572206290
S113C7807573206D6F6465203A202D627370692F74
S113C7906932632F756172742E2000000D0A2050D7
S113C7A06C6561736520696E707574207472616E56
S113C7B07366657220627573206166746572202DDC
S113C7C062203A202D627370692F6932632F75617C
S113C7D072742E2000000000526561647320746836
S113C7E06520636F6E74656E7473206F6620466C8B
S113C7F061736820494652206F7220466C617368E9
S113C800204669726D77617265204944000000001A
S113C810EB3C904D5357494E342E31000201010038
S113C820022000FF07F008000100010001000000E1
S113C830FF070000000029313233344B696E657400
S113C84069732055534200004E6F20726573706FF8
S113C8506E7365207061636B65742066726F6D2002
S113C86074617267657420646576696365207761B5
S113C870732065787065637465642E002976000002
S113C880DB76000000000000DB7600000000000002
S113C890B57700003B78000000000000E778000056
S113C8A0277900008B790000D57900001B7A0000FD
S113C8B00D0A202A2A2A2A2A2A2A2A2A2A2A2A2A1B
S113C8C02A2A2A2A2A2A2A2A2A2A2A2A2A2A2A2AC4
S113C8D02A2A2A2A2A2A2A2A2A2A2A200000000066
S113C8E00D0A202A2A2A2020202020202057656C87
S113C8F0636F6D6520746F20626C73682020202044
S113C90020202020202020202A2A2A200000000085
S113C910436F6D6D616E6420646973616C6C6F77D5
S113C9206564207768656E207365637572697479D0
S113C93020697320656E61626C65642E00000000DE
S113C940457261736520616C6C20666C6173682C40
S113C950206578636C7564696E672070726F7465A6
S113C9606374656420726567696F6E73000000000C
S113C970457261736520616C6C20666C6173682C10
S113C98020696E636C7564696E672070726F74657C
S113C9906374656420726567696F6E7300000000DC
S113C9A0457865637574652061742061646472659B
S113C9B0737320776974682061726720616E6420E4
S113C9C0737461636B20706F696E7465720000002C
S113C9D0666C6173682D70726F6772616D2D6F6E16
S113C9E06365203C696E6465783E203C62797465B9
S113C9F0436F756E743E203C646174613E000000B8
S113CA00666C6173682D726561642D7265736F75F0
S113CA10726365203C616464723E203C6279746593
S113CA20436F756E743E203C6F7074696F6E3E0088
S113CA30466C6173682041636365737320436F6E52
S113CA4074726F6C6C6572202846414329205375BB
S113CA5070706F727420466C6167203D20257300EE
S113CA60696E7374616E6365203C2046534C5F4667
S113CA704541545552455F534F435F464C455843D7
S113CA80414E5F434F554E54000000006D624964AF
S113CA9078203C3D2028626173652D3E4D43522031
S113CAA0262043414E5F4D43525F4D41584D425FF6
S113CAB04D41534B290000006B5374617475735FCF
S113CAC0466C61736845786563757465496E526137
S113CAD06D46756E6374696F6E4E6F7452656164F2
S113CAE0790000000D0A2020205472616E7366657F
S113CAF072206275733A20202020202020202020DC
S113CB0020202020202020554152542000000000E5
S113CB100D0A2020205472616E736665722062755E
S113CB20733A202020202020202020202020202094
S113CB3020202043414E202000000000696E7374C1
S113CB40616E6365203C2046534C5F464541545515
S113CB5052455F534F435F445350495F434F554ED3
S113CB6054000000696E7374616E6365203C204656
S113CB70534C5F464541545552455F534F435F47BD
S113CB8050494F5F434F554E54000000696E737413
S113CB90616E6365203C2046534C5F4645415455C5
S113CBA052455F534F435F4932435F434F554E54A1
S113CBB000000000517565727920766172696F75A5
S113CBC0732070726F7065727469657320616E642E
S113CBD02073657474696E67730000004E6F207271
S113CBE06573706F6E7365207061636B6574206626
S113CBF0726F6D2074617267657420646576696311
S113CC00652E00004E6F20726573706F6E73652021
S113CC10726563656976656420666F722070696EFB
S113CC206720636F6D6D616E642E00007365742DF3
S113CC30627573202D623C6275733E202D663C66DE
S113CC4072657175656E63792F62617564207261B6
S113CC5074653E005772697465206D656D6F7279F5
S113CC602066726F6D20737472696E67206F662020
S113CC706865782D76616C756573000077726974E8
S113CC80652D6D656D6F7279203C616464723E2020
S113CC905B7B7B3C6865782D646174613E7D7D5D62
S113CCA000000000466C61736820736563757269E7
S113CCB074792064697361626C65203C382D6279F3
S113CCC074652D6865782D6B65793E00666C6173BB
S113CCD0682D65726173652D726567696F6E203C9E
S113CCE0616464723E203C627974655F636F756E43
S113CCF0743E000065786563757465203C61646406
S113CD00726573733E203C6172673E203C737461AC
S113CD10636B706F696E7465723E0000466C61737C
S113CD206820416363657373205365676D656E7432
S113CD302053697A65203D202564206279746573E7
S113CD40000000000D0A2020205472616E73666595
S113CD5072206275733A2020202020202020202079
S113CD602020202020202053504920000D0A20207C
S113CD70205472616E7366657220667265717565A2
S113CD806E6379284B687A293A20202020202025B8
S113CD90640000000D0A2020205472616E736665E1
S113CDA072206275733A2020202020202020202029
S113CDB02020202020202049324320000D0A20205A
S113CDC0205472616E7366657220626175642072AC
S113CDD06174653A20202020202020202020202556
S113CDE0640000000D0A20496E76616C6964206954
S113CDF06D616765207479706520696E20686F7352
S113CE007420666C61736821000000000D0A2054D0
S113CE106865206672657175656E63792069732033
S113CE2061646A757374656420746F2031393230BB
S113CE30302E20000D0A20546865206672657175D5
S113CE40656E63792069732061646A7573746564BF
S113CE5020746F203132354B2E2000000D0A2054EF
S113CE606865206672657175656E637920697320E3
S113CE7061646A757374656420746F203235304B55
S113CE802E2000000D0A20546865206672657175B5
S113CE90656E63792069732061646A75737465646F
S113CEA020746F203530304B2E2000000D0A2054A2
S113CEB06865206672657175656E63792069732093
S113CEC061646A757374656420746F203130303026
S113CED04B2E20000D0A205468652074617267652A
S113CEE0742068617320726573657420737563635D
S113CEF065737366756C6C792E20000010B5074954
S113CF0079441831064C7C44163404E00A68081D40
S113CF10511888470146A142F8D110BD0002000013
S113CF20280200002128626173652D3E4D43522082
S113CF30262043414E5F4D43525F4D4449535F4D5C
S113CF4041534B29000000006B5374617475735F87
S113CF50466C61736850726F74656374696F6E5662
S113CF60696F6C6174696F6E000000004E6F20720F
S113CF706573706F6E736520726563656976656449
S113CF8020666F7220636F6D6D616E642E00000009
S113CF906B5374617475735F52656C6961626C651F
S113CFA0557064617465496D616765496E76616C3D
S113CFB06964000053657420766172696F7573202B
S113CFC070726F7065727469657320616E6420732A
S113CFD0657474696E67730050726F6772616D2057
S113CFE0666C6173682070726F6772616D206F6E1A
S113CFF06365206669656C6400000000666C61739B
S113D000682D726561642D6F6E6365203C696E6482
S113D01065783E203C62797465436F756E743E009A
S113D0200D0A204572726F723A20496E76616C69FE
S113D0306420617267756D656E747320272573278C
S113D040000000000D0A20526573706F6E73652036
S113D050537461747573203D20256420283078252D
S113D06058292025730000000D0A204E6F20466CBD
S113D07061736820696D61676520696E20686F73EC
S113D0807420666C61736821000000000D0A205052
S113D090696E6720726573706F6E64656420696E73
S113D0A020256420617474656D70742873290000F0
S113D0B0008004022000000046534C2053454D4993
S113D0C046534C204D4153532053544F52414745EE
S113D0D03030303172B60448044901600448804756
S113D0E062B604480047000008ED00E000000000BC
S113D0F079660000A9E300004EF68851CEF20001E3
S113D100086840F470000860BFF34F8FBFF36F8F5F
S113D1104FF00070E1EE100A7047000005F6FFFFC3
S113D120DCC100000006FF1F0000000083E8FFFFD1
S113D1300200000002000000A0150000F903000036
S113D1400000FF1FE5050000FEE70000446973705E
S113D1506C617920636F6D6D616E6473206C6973AB
S113D1607420616E64207573616765000D0A204543
S113D17072726F723A20416D6269677569747920C1
S113D180636F6D6D616E643A202573000D0A20454E
S113D19072726F723A20496E76616C696420636FB3
S113D1A06D6D616E643A2025730000000800100064
S113D1B0180020003000400060008000C000000122
S113D1C08001000200030004000600002828636FA9
S113D1D06E66696729207C7C202866616C736520F3
S113D1E03D3D20656E61626C652929006B53746155
S113D1F07475735F466C617368556E6B6E6F776E92
S113D20050726F7065727479000000006B53746122
S113D2107475735F466C617368526567696F6E45B8
S113D2207865637574654F6E6C79000049324320EC
S113D230536C61766520545820556E64657272751E
S113D2406E206572726F722E0000000053504920E8
S113D250536C61766520545820556E6465727275FE
S113D2606E206572726F722E000000005153504997
S113D27020466C61736820556E6B6E6F776E20501C
S113D280726F70657274792E000000006B537461C4
S113D290747573526F6D4C6472556E656E637279FA
S113D2A0707465644F6E6C79000000006B53746198
S113D2B07475735F417070437263436865636B4F49
S113D2C075744F6652616E67650000006B5374613C
S113D2D07475735F52656C6961626C6555706461E5
S113D2E07465537563636573730000006B537461F5
S113D2F07475735F52656C6961626C6555706461C5
S113D3007465496E616374697665000053657420C1
S113D31062757320616E64206672657175656E63F3
S113D320792F626175642072617465005772697443
S113D33065206120666F726D6174656420696D613A
S113D340676520746F20666C617368007265616440
S113D3502D6D656D6F7279203C616464723E203C72
S113D360627974655F636F756E743E00666C617399
S113D370682D73656375726974792D64697361626C
S113D3806C65203C6B65793E000000005265616469
S113D39020666C6173682070726F6772616D206FB4
S113D3A06E6365206669656C640000004375727283
S113D3B0656E742056657273696F6E203D20256317
S113D3C025642E25642E256400000000466C6173DC
S113D3D06820536563746F722053697A65203D2019
S113D3E0256420627974657300000000466C6173E3
S113D3F0683A20307825582D30782558202825641F
S113D400206279746573292C20000000466C6173D6
S113D4106820416363657373205365676D656E743B
S113D42020436F756E74203D202564000D0A205240
S113D4306573706F6E736520776F72642031203D61
S113D4402025642028307825582900000D0A205210
S113D4506573706F6E736520776F72642032203D40
S113D4602025642028307825582900005CE4000039
S113D470A4E60000A8E60000ACE60000B0E6000068
S113D480B4E60000B8E60000BCE600000D0A204641
S113D4906C61736820696D6167652073756363658A
S113D4A073732E200D0A203E2000000023A70000E5
S113D4B0FDA8000021A900000300000000000000F6
S113D4C000000000000000000000000062617564BC
S113D4D0526174655F427073203C3D2031303030BE
S113D4E03030305500000000707269446976203C89
S113D4F03D20736F75726365436C6F636B5F487A2D
S113D500000000006D6173746572436F6E66696735
S113D51020262620737263436C6F636B5F487A0026
S113D520696E7374616E6365203C20756172744129
S113D53072726179436F756E74000000666C61737A
S113D540682D65726173652D616C6C2D756E7365E4
S113D55063757265000000006B5374617475735FCA
S113D560466C617368416C69676E6D656E74457273
S113D570726F72006B5374617475735F466C617380
S113D58068416464726573734572726F720000005F
S113D5906B5374617475735F466C61736841636344
S113D5A06573734572726F72000000006B5374618F
S113D5B07475735F466C617368436F6D6D616E64FF
S113D5C04661696C7572650049324320536C61761B
S113D5D065205258204F76657272756E206572729E
S113D5E06F722E0049324320417262697472617411
S113D5F0696F6E204C6F7374206572726F722E00A7
S113D60053504920536C617665205258204F7665FB
S113D6107272756E206572726F722E00515350498A
S113D62020466C61736820416C69676E6D656E7429
S113D630206572726F722E005153504920466C61FE
S113D64073682041646472657373206572726F72CB
S113D6502E0000005153504920466C6173682043EA
S113D6606F6D6D616E64204661696C7572652E0024
S113D6705153504920436F6D6D616E64204E6F7439
S113D68020537570706F727465642E004F54464158
S113D690442053656375726974792056696F6C61AF
S113D6A074696F6E2E0000004F54464144204C6F45
S113D6B0676963616C6C792044697361626C656449
S113D6C02E0000006B537461747573526F6D4C645B
S113D6D07253656374696F6E4F76657272756E000E
S113D6E06B537461747573526F6D4C6472536563DC
S113D6F074696F6E4C656E67746800006B53746177
S113D700747573526F6D4C6472556E6B6E6F776E79
S113D710436F6D6D616E64006B5374617475735205
S113D7206F6D4C647244617461556E646572727598
S113D7306E0000006B537461747573526F6D4C64AA
S113D740724A756D7052657475726E65640000007E
S113D7506B537461747573526F6D4C64724B65795D
S113D7604E6F74466F756E64000000006B537461F5
S113D7707475734D656D6F727952616E6765496E2C
S113D78076616C69640000006B5374617475734D49
S113D790656D6F727957726974654661696C656409
S113D7A0000000006B5374617475735F41707043C3
S113D7B07263436865636B50617373656400000052
S113D7C06B5374617475735F417070437263436823
S113D7D065636B4661696C65640000006B5374613A
S113D7E07475735F417070437263436865636B491A
S113D7F06E616374697665006B5374617475735FED
S113D800417070437263436865636B496E76616C03
S113D810696400006B5374617475735F52656C695D
S113D82061626C655570646174654661696C000081
S113D8307365742D70726F7065727479203C7461B5
S113D840673E203C76616C75653E000052657365E9
S113D85074207468652074617267657420626F6FE8
S113D860746C6F616465720046696C6C206D656DE3
S113D8706F72792077697468207061747465726E50
S113D8800000000054617267657420566572736904
S113D8906F6E203D20256325642E25642E256400AB
S113D8A0417661696C61626C65205065726970686B
S113D8B06572616C73203D2000000000466C61734A
S113D8C068205374617274204164647265737320B8
S113D8D03D203078255800004D6178205061636BFD
S113D8E065742053697A65203D202564206279742B
S113D8F06573000052414D3A20307825582D307818
S113D9002558202825642062797465732900000055
S113D91052414D2053746172742041646472657382
S113D92073203D203078255800000000466C617358
S113D93068205365637572697479205374617465E2
S113D940203D202573000000466C617368207265D9
S113D9506164206D617267696E206C6576656C2008
S113D9603D20000052656C6961626C6520557064ED
S113D97061746520537461747573203D20257300B0
S113D980666C6173682D65726173652D616C6C2DB5
S113D990756E736563757265000000000D0A20459D
S113D9A07261736520666C61736820726567696F64
S113D9B06E204F4B212000000D0A20466C617368D5
S113D9C020696D616765206661696C21200D0A20FC
S113D9D03E2000000120C046002801D0FFF78EFA47
S113D9E00020C046C046FDF779FE00F000F800F0C4
S113D9F001B8350007463846F9F7F0FDFBE70000AB
S113DA000D0A20436F6D6D616E64204C6973743A26
S113DA10200D0A20000000000D0A466C6173682086
S113DA2070726F6772616D206572726F722100008F
S113DA3074784672616D652D3E6C656E67746820FE
S113DA403C3D203800000000636F6E6669672D3E20
S113DA5062617564526174655F4270730000000016
S113DA60666C6173682D73656375726974792D646E
S113DA70697361626C6500006B5374617475735FE4
S113DA80496E76616C6964417267756D656E740088
S113DA906B5374617475735F466C61736853697A10
S113DAA0654572726F7200005153504920466C6193
S113DAB073682053697A65206572726F722E000054
S113DAC051535049204E6F7420436F6E66696775D9
S113DAD07265642E000000005153504920436F6D5D
S113DAE06D616E642054696D656F7574000000008B
S113DAF04F5446414420496E76616C6964204B65FD
S113DB0079426C6F622E00006B5374617475735F9D
S113DB10556E6B6E6F776E436F6D6D616E64000052
S113DB206B5374617475735F41626F727444617492
S113DB3061506861736500006B537461747573524E
S113DB406F6D4C64725369676E6174757265000021
S113DB506B537461747573526F6D4C6472454F46A8
S113DB6052656163686564006B53746174757352C4
S113DB706F6D4C6472436865636B73756D00000070
S113DB806B537461747573526F6D4C64724372633A
S113DB9033324572726F72006B53746174757352D1
S113DBA06F6D4C647249644E6F74466F756E640099
S113DBB06B537461747573526F6D4C647243616C12
S113DBC06C4661696C6564006B537461747573525F
S113DBD06F6D4C64725365637572654F6E6C79003A
S113DBE06B5374617475734D656D6F7279526561B1
S113DBF0644661696C65640050726F706572747913
S113DC0020697320726561642D6F6E6C792E00003B
S113DC10496E76616C69642070726F706572747994
S113DC202076616C75652E00496E76616C6964209E
S113DC307061636B657420747970652E0000000058
S113DC4052656164206D656D6F727920616E642028
S113DC50646973706C617900457261736520612039
S113DC60726567696F6E206F6620666C6173680009
S113DC7043616C6C206164647265737320776974AA
S113DC80682061726700000063616C6C203C616411
S113DC9064726573733E203C6172673E000000004D
S113DCA0556E6B6E6F776E206572726F7220636F44
S113DCB06465202825642900466C617368205369D3
S113DCC07A65203D20256420627974657300000024
S113DCD0466C61736820426C6F636B20436F756E92
S113DCE074203D2025640000417661696C61626C9A
S113DCF06520436F6D6D616E6473203D20000000EC
S113DD0043524320436865636B2053746174757395
S113DD10203D2025730000005665726966792057FE
S113DD20726974657320466C6167203D2025730019
S113DD3053797374656D204465766963652049443D
S113DD40203D2030782558005153504920496E69B0
S113DD507420537461747573203D20257300000092
S113DD600D0A20466C61736820696D6167652073D4
S113DD707563636573732E000D0A20466C617368C6
S113DD8020696D616765206661696C21000000008F
S113DD90666C6173682D73656375726974792D643B
S113DDA0697361626C6500000D0A20496E6A6563DF
S113DDB07420636F6D6D616E6420272573270000E6
S113DDC067610000096200004F6200000163000007
S113DDD0036400006364000038B504460D46284619
S113DDE0FBF705FCA84218BF0024204632BD000002
S113DDF05350492C204932432C20554152542C2055
S113DE0043414E000168F02212040A430260BFF34A
S113DE106F8FBFF34F8F7047735F666C6578636174
S113DE206E48616E646C655B305D0000735F666CA8
S113DE30657863616E48616E646C655B315D00009A
S113DE400090044000A0044000B0044000C004401E
S113DE5000D0044000F00F4040F00F4080F00F402D
S113DE60C0F00F4000F10F4000A0064000B0064093
S113DE7000C0064000D0064000A00E400A00341046
S113DE800B0034100C0034100D0034100A0028105C
S113DE90666C6173682D65726173652D726567695F
S113DEA06F6E0000666C6173682D70726F677261CB
S113DEB06D2D6F6E63650000666C6173682D72650D
S113DEC061642D7265736F7572636500636F6E664E
S113DED069677572652D71756164737069000000FE
S113DEE06765742D70726F7065727479203C74610B
S113DEF0673E00006B5374617475735F52656164AF
S113DF004F6E6C79000000006B5374617475735F1D
S113DF104F75744F6652616E6765000051535049E6
S113DF20205772697465204661696C7572652E00AC
S113DF304F5446414420496E76616C6964204B65B8
S113DF40792E0000556E6B6E6F776E2070726F7055
S113DF50657274792E000000496E76616C696420E4
S113DF604352432076616C75652E000052657365DB
S113DF707276656420526567696F6E73203D200078
S113DF8052414D2053697A65203D202564206279F1
S113DF9074657300556E69717565204465766963AF
S113DFA065204944203D0000666C6173682D6572EC
S113DFB06173652D726567696F6E0000666C6173CD
S113DFC0682D70726F6772616D2D6F6E63650000EE
S113DFD0666C6173682D726561642D7265736F750B
S113DFE072636500636F6E6669677572652D71751E
S113DFF0616473706900000000A0064000B0064030
S113E00000C0064000D0064000A00E404578697468
S113E0102074686520626C736800000025730D0A23
S113E020200909092025730D0A2000005472616E2D
S113E0307366657272696E670D0A00005457522D3B
S113E0404B3635463138304D00000000D4E3000033
S113E0502CE0000094E20000A0E200002110000087
S113E060FFFF00000000000000000000675F647311
S113E070706948616E646C655B305D00675F6473F2
S113E080706948616E646C655B315D00675F6473E1
S113E090706948616E646C655B325D00020000006B
S113E0A0030000000500000007000000010000005C
S113E0B00300000005000000070000006D61737498
S113E0C06572436F6E666967000000000060064079
S113E0D00070064000600E4000700E4006003410D0
S113E0E0070034100600281007002810735F7561BC
S113E0F0727448616E646C655B305D00735F75615A
S113E100727448616E646C655B315D00735F756148
S113E110727448616E646C655B325D00735F756137
S113E120727448616E646C655B335D00666C617328
S113E130682D65726173652D616C6C00777269740A
S113E140652D6D656D6F7279000000006765742D33
S113E15070726F7065727479000000007265636597
S113E1606976652D73622D66696C65007365742D1F
S113E17070726F706572747900000000666C617370
S113E180682D726561642D6F6E63650072656C69DC
S113E19061626C652D757064617465006B537461A4
S113E1A07475735F50696E6700000000554E4B4EE6
S113E1B04F574E202825642900000000556E6B6ED1
S113E1C06F772070726F706572747900666C61731A
S113E1D0682D65726173652D616C6C00777269746A
S113E1E0652D6D656D6F7279000000006765742D93
S113E1F070726F70657274790000000072656365F7
S113E2006976652D73622D66696C65007365742D7E
S113E21070726F706572747900000000666C6173CF
S113E220682D726561642D6F6E63650072656C693B
S113E23061626C652D757064617465000D0A20451A
S113E24072617365206661696C2100000D0A2052B9
S113E25065736574206661696C00000000600640A7
S113E2600070064000600E4000700E40F0FFFFFF9B
S113E270FFFFFFFFFFFFFFFFFFFF00000D0A20422B
S113E2807965200D0A0000006372633136436F6EB6
S113E29066696700537563636573730D0A00000054
S113E2A04661696C7572650D0A0000003078303083
S113E2B03030303030300000307830303230303070
S113E2C0303000003078316666663030303000001F
S113E2D03078323030326666666600007472616E81
S113E2E0736665720000000000C0024000D0024066
S113E2F000C00A400C003C100D003C100C00301013
S113E3008021017002780A42FCD070476932634868
S113E310616E646C65000000726561642D6D656DED
S113E3206F72790066696C6C2D6D656D6F72790022
S113E330666C6173682D696D61676500537563630D
S113E3406573732E000000004661696C7572652E5A
S113E35000000000554E534543555245000000004F
S113E360535550504F52544544000000554E535598
S113E37050504F5254454400726561642D6D656D73
S113E3806F72790066696C6C2D6D656D6F727900C2
S113E390666C6173682D696D6167650000C0024039
S113E3A000D0024000C00A40C046C046FEF7A4FEAA
S113E3B0FFF710FB68656C700000000065786974F5
S113E3C0000000000D0A203E200000000D203E2029
S113E3D02573000052656164790D0A0066616C73EF
S113E3E065000000636F6E666967000066616C73A8
S113E3F06500000074784672616D6500727846723B
S113E400616D650068616E646C65000000400240E7
S113E41000400A4004003C1004003010636F6E6634
S113E42069670000786665720000000068616E64C8
S113E4306C6500007053656D00000000636F6E66CC
S113E44069670000657865637574650063616C6C69
S113E4500000000072657365740000005541525459
S113E460000000007365742D6275730053454355B5
S113E4705245000020255820255800004E4F524D8B
S113E480414C00005553455200000000464143549E
S113E4904F5259000000000064000000756172745E
S113E4A0000000003078255820000000776F726467
S113E4B00000000073686F72740000006279746574
S113E4C000000000657865637574650063616C6CB9
S113E4D00000000072657365740000001F2123258D
S113E4E0420000000040024000400A40636F6E6634
S113E4F069670000000000000000000000480047B9
S113E500D5E6000000480047D5E600000048004773
S113E510D5E6000000480047D5E600000048004763
S113E520D5E6000000480047D5E600000048004753
S113E530D5E6000000480047D5E600000048004743
S113E540D5E6000000480047D5E600000048004733
S113E550D5E6000000480047D5E600000048004723
S113E560D5E6000000480047D5E600000048004713
S113E570D5E6000000480047D5E600000048004703
S113E580D5E6000000480047814A000000480047E3
S113E5908F4A000000480047E74000000048004759
S113E5A00D41000000480047D5E600000048004740
S113E5B0D5E6000000480047AF3600000048004799
S113E5C0D5E6000000480047DD360000004800475B
S113E5D0D5E60000004800470B370000004800471C
S113E5E0D5E60000004800473937000000480047DE
S113E5F0D5E60000004800474141000000480047BC
S113E600D5E60000004800479D4A00000048004746
S113E6107D550000004800477D5500000048004734
S113E620D5E6000000480047D5E600000048004752
S113E630D5E6000000480047D5E600000048004742
S113E640D5E6000000480047D5E600000048004732
S113E650AB4A000000480047A955000000480047A5
S113E660A955000000480047A9550000004800478C
S113E670A955000000480047A9550000004800477C
S113E680A955000000000000010100000020034023
S113E6900400024018194A5B693263007370690010
S113E6A063616E00493243005350490043414E00B8
S113E6B04849440043444300444655004D534400F4
S113E6C0693263007370690063616E000020074063
S113E6D000000000FFF7FEBF2006B4E300004CD1A9
S113E6E000000890011D9300011001FF1FBC1420BD
S113E6F0020CE0000008B2451C52010D200120006C
S113E700040A52100F80028000004027721418512E
S113E7100143BD29101003B804FF1F6C6043972AFE
S113E7204A134CE180C007CB0000E0DE0000F17D1D
S113E73034433CE32412480812020812F42412035E
S113E74008300108DF007C100378DA000064081246
S113E7509008126508100358D50000660812740862
S113E76022671811082268401002CF0000690812BD
S113E770AC10126A0812ECF4126C0810030CD200EC
S113E780006D081003B8CA0000C808122C1012C982
S113E7900812C82811131300E408122C81124C1813
S113E7A0222D8912D654110812A870129108121C35
S113E7B0101292081238081293081254081294087E
S113E7C0126C3012950812C0281296081270181292
S113E7D0970812D81022983811C012F408128C1815
S113E7E022F550110812F60812301812F70812F028
S113E7F028131027E81002DB0000110812109512EC
S113E8001208122010121308169C3412140816DC75
S113E810381215081248BD12740812C4481275083B
S113E82012382812760812E010127708128C90120F
S113E8307808125018127908126808127A0812809F
S113E84008127B0812FC28127C08129810127D080A
S113E850100318D700007E08123408127F0812B083
S113E86018228040111012810812C81012D8081200
S113E8706C1022D968111012DA0812881010033CA7
S113E88028000044C8123D0812F818123E0810036C
S113E89010DC0000A00812A42012A10812C0081263
S113E8A0A20812DC0822A328110812A40812ACA89A
S113E8B01A0428100304CC00000508122838120694
S113E8C008125850120708166CC812680812CC288F
S113E8D01269081714D8D01108129018126B081274
S113E8E0EC181004FFFFFF7FF3D92C2958111812DC
S113E8F030247001C58100011754E4D042D8088344
S113E900558218126410170CD3F0117C926B181AEC
S113E910307C432CD30883F58418123C6012542CA9
S113E920127C04833985181218281240B8124C340A
S113E930832986181224181268781FE0C66C038293
S113E94087181660EC12A444126C30832D881812B8
S113E9502C604340C90893B5897819944370C90859
S113E96092CB181E901C0312587812CC4C9231187A
S113E9701244D812A03012F41892E118124C181252
S113E980703012880483858A1812A44816D8381265
S113E990D03483418B18127C88128CA412FC1C8303
S113E9A0ED8C1822B83012C7101D310383CD8D1899
S113E9B01B531B3C1104200868C2FF1F2F010302D4
S113E9C0011705220B052207052205055E004E04EA
S113E9D04C070E270781024000020242042DEC037B
S113E9E01E8C2804210D100308065000940C612C81
S113E9F012A40C12B00412030D3312012B20074091
S113EA00A215000201010102141C080902200001E0
S113EA100100C03209220422023E2307055C1107CB
S113EA20315F1009040309043A0346005200450209
S113EA3010055300430041004C0A12200C100345FA
S113EA40004D00491210054F004E004400550A12B3
S113EA50540C12521C124912100143002E6D100165
S113EA6022034D0A125514124D3A125302213A410F
S113EA702810014100474421241011300031003294
S113EA8000330034003500360037003800391E12D8
S113EA90423A12442232462412421252443E325224
S113EAA06252476A21244F5800E404223A2C91040C
S113EAB012F4FC12F80410033405FF1F5804127CEE
S113EAC00412B40412A00421F32120213857C805EC
S104EAD0340D
S903E3A970
